:020000041000EA
:1000000000001020B5360110F1360110F336011052
:10001000F5360110F7360110F93601100000000026
:10002000000000000000000000000000FB3601108E
:10003000FD36011000000000FF360110BD730010F6
:10004000033701100537011007370110CD87001065
:100050000B37011091870010A5870010B987001099
:100060001337011015370110173701101937011018
:100070001B370110E57F00105587001069870010BD
:1000800023370110253701102737011029370110B8
:100090002B3701102D3701102F3701103137011088
:1000A0004D7900105B790010697900103937011023
:1000B0003B3701103D3701103F3701104137011028
:1000C00043370110453701107D8700104937011073
:1000D000F97F00104D3701104F37011051370110D3
:1000E0005337011055370110573701105937011098
:1000F0005B3701105D3701105F3701106137011068
:100100006337011065370110673701106937011037
:100110006B3701106D3701106F3701107137011007
:100120007337011075370110777900107937011096
:100130007B3701107D3701107F37011081370110A7
:100140008337011085370110873701108937011077
:100150008B3701108D3701108F3701109137011047
:100160009337011095370110973701109937011017
:100170009B3701109D3701109F370110A1370110E7
:10018000A337011010B5054C237833B9044B13B1D4
:100190000448AFF300800123237010BD88130020B2
:1001A000000000000019021008B5034B1BB1034901
:1001B0000348AFF3008008BD000000008C1300204E
:1001C0000019021080B584B000AF7860124B1B6834
:1001D000002B02D1104B114A1A600F4B1B68FB60B9
:1001E0000D4B1A687B6813441A460D4B9A4207D987
:1001F00014F074FF03460C221A604FF0FF3306E040
:10020000054B1A687B681344034A1360FB68184661
:100210001037BD4680BD00BFA4130020C02E0020B3
:1002200000F00F2080B400AF6FF010031846BD46F9
:100230005DF8047B704780B400AF6FF01003184680
:10024000BD465DF8047B704780B485B000AF4FF0C9
:1002500080439B6803F46063BB60BB68B3F5806F49
:1002600002D11A4BFB601EE0BB68B3F5C06F03D12F
:100270004FF4FA53FB6016E0BB68B3F5006F02D190
:10028000134BFB600FE0BB68B3F5206F02D1114B3D
:10029000FB6008E0104B1B78A12B02D90F4BFB60D1
:1002A00001E00F4BFB604FF080439B689B0903F01C
:1002B00007037B60FA687B6822FA03F3094A13603C
:1002C00000BF1437BD465DF8047B704700366E01F1
:1002D000000E270700127A00AC13002080F0FA020B
:1002E000005A6202A813002080B400AF4FF0804390
:1002F0001B6823F440334FF0804243F40033136013
:1003000000231846BD465DF8047B704780B400AFFB
:1003100000231846BD465DF8047B704780B500AFEA
:1003200002F0E3FE03461A46554B1A70554B564AE7
:100330009A6062B600BF534BD3F88830514A43F4F9
:100340007003C2F88830BFF34F8F00BFBFF36F8FC9
:1003500000BF042002F078FDFFF776FF4FF08043E6
:100360001B684FF0804243F400331360474B012277
:10037000C3F8002700BF454BD3F8003103F48033A6
:10038000002BF8D0414BD3F80031404A43F0010331
:10039000C2F8003100BF3D4BD3F8003103F4803385
:1003A000002BF8D0032002F0E0FC042002F0DDFC7A
:1003B000052002F0DAFC062002F0D7FC072002F04C
:1003C000D4FC082002F0D1FC092002F0CEFC0A2067
:1003D00002F0CBFC0D2002F0C8FC0E2002F0C5FCA0
:1003E0000F2002F0C2FC102002F0BFFC112002F02E
:1003F000BCFC122002F0B9FC132002F0B6FC142061
:1004000002F0B3FC172002F0B0FC1C2002F0ADFC9F
:100410001D2002F0AAFC1E2002F0A7FC1F2002F003
:10042000A4FC212002F0A1FC222002F09EFC23204B
:1004300002F09BFC242002F098FC272002F095FC9F
:10044000282002F092FC292002F08FFC2A2002F0E2
:100450008CFC2B2002F089FC2C2002F086FC2D2045
:1004600002F083FC2E2002F080FC2F2002F07DFCA5
:10047000342002F07AFCFFF749FF00BF80BD00BFC7
:10048000AC13002000ED00E00000001000A00240CE
:1004900080B500AF1A2002F0FDFD172002F090FC9D
:1004A000024800F07FF80346184680BD0040034034
:1004B00080B584B000AF78607B689B02FB60FB680E
:1004C0001B4A934202D96FF002032DE0194B1B68BF
:1004D0005A08FB68B2FBF3F3FB72FB7A0F2B02D8CE
:1004E000FB7A012B02D86FF002031DE0124B1B6850
:1004F000114A23F4006313604FF080439B694FF06F
:10050000804223F4705393614FF080439A69FB7AE1
:100510009B024FF0804113438B617968064800F0DD
:100520009AF800F00BF8034618461037BD4680BD18
:1005300000127A00A81300200040034080B582B06A
:1005400000AF4FF080439B699B0ADBB203F00F03BF
:10055000FB71FB79184600F091F8034618460837FE
:10056000BD4680BD80B582B000AF78607968044830
:1005700000F0EAF8034618460837BD4680BD00BFC4
:100580000040034080B582B000AF786079680448CD
:1005900000F018F9034618460837BD4680BD00BF75
:1005A0000040034080B584B000AF786041F2D7606E
:1005B000FFF77EFF4FF40031786800F037F87B6872
:1005C0001B6843F002027B681A607B681B6843F07B
:1005D00008027B681A6000BF7B68DB6803F40033A5
:1005E000002BF9D04FF40031786800F01FF80C4B65
:1005F00000221A600023FB7307E0FB7B094A0021FD
:1006000042F82310FB7B0133FB73FB7B032BF4D9F4
:10061000054B00221A60002318461037BD4680BDE6
:10062000C0130020B0130020C413002080B483B096
:1006300000AF786039607B68DB6803F01F023B68BD
:1006400003F4F8131A437B68DA6000BF0C37BD4629
:100650005DF8047B704780B483B000AF7860396088
:100660007B681B6843F400627B681A6000231846AD
:100670000C37BD465DF8047B7047000080B485B040
:1006800000AF0346FB71074B1B685A08FB79B2FBAE
:10069000F3F3FB60FB689B0A18461437BD465DF810
:1006A000047B7047A813002080B483B000AF78604B
:1006B0000B46FB707B681B6823F4C0227B681A60C2
:1006C000FB78022B20D0022B2BDC002B02D0012B3D
:1006D0000DD026E07B681B6843F480727B681A604B
:1006E0007B681B6823F400727B681A6026E07B68D5
:1006F0001B6823F480727B681A607B681B6823F494
:1007000000727B681A6019E07B681B6823F48072B2
:100710007B681A607B681B6843F400727B681A6010
:100720000CE07B681B6823F480727B681A607B682E
:100730001B6823F400727B681A6000BF00BF0C378F
:10074000BD465DF8047B704780B584B000AF78602B
:1007500039607B681B6823F4F8327B681A607B6819
:100760001A683B681B781B0303F4F8331A437B6851
:100770001A603B681B78072B05D83B685B781946E5
:100780007868FFF791FF4FF480317868FFF74EFFEC
:100790007B681B6843F001027B681A6007F10A035B
:1007A0001846FFF7EFFEF860FB68002B01D0FB68EE
:1007B00004E07B891A463B685A60002318461037CC
:1007C000BD4680BD80B483B000AF786039607B687F
:1007D0005B6803F00103002B06D000BF7B68DB6879
:1007E00003F48033002BF9D07B681B6803F480137B
:1007F000002B05D17B689B689AB23B681A8005E0A4
:100800007B689B689B099AB23B681A807B685B682F
:1008100003F00803002B02D06FF00B0300E000236D
:1008200018460C37BD465DF8047B704780B500AFB5
:10083000014800F00FF880BD0080024080B582B012
:1008400000AF7860786800F021F803461846083752
:10085000BD4680BD80B485B000AF78607B68094A32
:10086000934201D1002301E04FF0FF33FB60064AC1
:10087000FB68002142F8231000BF1437BD465DF825
:10088000047B704700800240C813002080B582B00E
:1008900000AF78607B68002B43DB7B680F2B40DC6C
:1008A00023497A6813469B0013449B000B441B6842
:1008B000002B36D001211F4802F020FA0346002BFE
:1008C00002D06FF005032EE019497A6813469B00A9
:1008D00013449B000B4400221A6015497A681346A2
:1008E0009B0013449B000B440C331B6800221A60CE
:1008F0000F497A6813469B0013449B000B440C334A
:1009000019680B487A6813469B0013449B00034404
:100910000C331B684A685A60064802F016FA002336
:1009200001E06FF0020318460837BD4680BD00BFE6
:10093000CC1300200C15002080B582B000AF786089
:100940007968044800F018F8034618460837BD4691
:1009500080BD00BF0090024080B582B000AF7860DB
:100960007968044800F034F8034618460837BD4655
:1009700080BD00BF0090024080B483B000AF7860BB
:1009800039603B68B3F1845F03D33B680C4A934200
:1009900002D96FF002030DE07B6841F234221A6441
:1009A0007B68084A1A647B68074A1A647B68074AAE
:1009B0001A64002318460C37BD465DF8047B704767
:1009C000FFFF8010A35C7F3A204FE3A1C1B20896DD
:1009D00080B483B000AF786039603B68B3F1845F66
:1009E00003D33B68074A934202D96FF0020303E046
:1009F0007B68054A1A64002318460C37BD465DF82B
:100A0000047B7047FFFF8010EFBEADDE80B485B081
:100A100000AF7860134B1B78002B1CD10023FB60C8
:100A200013E00023BB600AE00F49FB685A01BB6872
:100A30001344002241F82320BB680133BB60BB682C
:100A40001F2BF1DDFB680133FB60FB68032BE8DD46
:100A5000044B01221A70002318461437BD465DF876
:100A6000047B7047101900201015002080B487B057
:100A700000AFF860B9607A60FB685B687B61002357
:100A80003B6154E07B6903F00103002B49D0FB6814
:100A90001B682C4A934217D0FB681B682A4A934272
:100AA00010D0FB681B68294A934209D0FB681B6879
:100AB000274A934201D1032307E04FF0FF3304E0BC
:100AC000022302E0012300E0002322495A013B698E
:100AD0001344BA6841F82320FB681B68194A934203
:100AE00017D0FB681B68184A934210D0FB681B683C
:100AF000164A934209D0FB681B68154A934201D1FC
:100B0000032307E04FF0FF3304E0022302E0012358
:100B100000E0002310495A013B6913447A6841F808
:100B200023203B6901333B617B695B087B617B6907
:100B3000002BA7D100BF00BF1C37BD465DF8047B6A
:100B4000704700BF008000400090004000A00040BF
:100B500000B00040101500201017002080B586B0AE
:100B600000AF78607B68002B10D07B68012B0BD026
:100B70007B68022B06D07B68032B01D1204B06E05B
:100B8000002304E01F4B02E01F4B00E01F4BFB6003
:100B9000F86800F09BF978617969F86800F0A2F9CB
:100BA00000233B6123E07B6903F00103002B18D095
:100BB00017497B685A013B69134451F82330002BD5
:100BC0000FD013497B685A013B69134451F8233015
:100BD00010487A6851013A690A4450F822201046B8
:100BE00098473B6901333B617B695B087B617B69AB
:100BF000002BD8D100BF00BF1837BD4680BD00BF55
:100C000000B0004000A00040009000400080004084
:100C1000101500201017002080B582B000AF78605A
:100C20007B68002B03D1002002F0CAF817E07B6834
:100C3000012B03D1012002F0C3F810E07B68022BE6
:100C400003D1022002F0BCF809E07B68032B03D13A
:100C5000262002F0B5F802E06FF0020303E07868A6
:100C6000FFF7D4FE034618460837BD4680BD000096
:100C700080B584B000AF78607B681B68FB607B68E0
:100C8000197A7B685B681A46F86800F0A5FAB860C4
:100C9000BB68002B01D0BB68B3E07B685B7A042B98
:100CA00000F28F8001A252F823F000BFC10C0010A7
:100CB000F70C0010290D00105B0D00108F0D0010B7
:100CC000FB681A6E7B685B68DB431A40FB681A6638
:100CD000FB685A6E7B685B68DB431A40FB685A66A8
:100CE000FB68D3F8B8207B685B68DB431A40FB687D
:100CF000C3F8B82068E0FB681A6E7B685B681A432B
:100D0000FB681A66FB685A6E7B685B68DB431A40B7
:100D1000FB685A66FB68D3F8B8207B685B681A43A7
:100D2000FB68C3F8B8204FE0FB681A6E7B685B680D
:100D3000DB431A40FB681A66FB685A6E7B685B6887
:100D40001A43FB685A66FB68D3F8B8207B685B6877
:100D50001A43FB68C3F8B82036E0FB681A6E7B685C
:100D60005B681A43FB681A66FB685A6E7B685B68AF
:100D7000DB431A40FB685A66FB68D3F8B8207B68EF
:100D80005B68DB431A40FB68C3F8B8201CE0FB68D3
:100D90001A6E7B685B68DB431A40FB681A66FB6867
:100DA0005A6E7B685B681A43FB685A66FB68D3F827
:100DB000B8207B685B68DB431A40FB68C3F8B82047
:100DC00002E06FF002031CE07B68997A7B685B6845
:100DD0001A46F86800F0ADF8B860BB68002B01D087
:100DE000BB680EE07B681B7A002B01D1002308E072
:100DF0007B68D97A7B685B681A46F86800F0ABF8C4
:100E0000034618461037BD4680BD00BF80B582B08E
:100E100000AF786039603968786800F0AEF8034652
:100E200018460837BD4680BD80B582B000AF7860F7
:100E300039603968786800F0AFF800BF0837BD4600
:100E400080BD80B582B000AF78603960396878685D
:100E500000F0B0F800BF0837BD4680BD80B582B055
:100E600000AF786039603968786800F0B1F80346FF
:100E700018460837BD4680BD80B582B000AF7860A7
:100E80000B46FB70FB781946786800F0B1F8034612
:100E900018460837BD4680BD80B582B000AF786087
:100EA00039603968786800F037F900BF0837BD4607
:100EB00080BD80B582B000AF7860396039687868ED
:100EC00000F038F900BF0837BD4680BD80B582B05C
:100ED00000AF7860786800F049F903461846083793
:100EE000BD4680BD80B582B000AF7860396039689A
:100EF000786800F02DF900BF0837BD4680BD80B589
:100F000084B000AFF860B9607A607A68B968F86850
:100F1000FFF7ACFD00BF1037BD4680BD80B582B085
:100F200000AF78607868FFF719FE00BF0837BD464C
:100F300080BD80B584B000AFF8600B467A60FB726C
:100F4000FB7A7A681946F86800F01CF903461846DF
:100F50001037BD4680BD80B584B000AFF8600B4649
:100F60007A60FB72FB7A7A681946F86800F09AF9A1
:100F7000034618461037BD4680BD80B483B000AF2D
:100F8000786039607B685A6A3B68134018460C37B2
:100F9000BD465DF8047B704780B483B000AF7860D5
:100FA00039607B683A68DA6100BF0C37BD465DF88E
:100FB000047B704780B483B000AF786039607B6891
:100FC0003A681A6200BF0C37BD465DF8047B704773
:100FD00080B483B000AF786039607B689A693B6801
:100FE000134018460C37BD465DF8047B704700007F
:100FF00080B485B000AF78600B46FB707B681B68DF
:10100000FB60FB78042B7CD801A252F823F000BFD0
:101010005510001025100010B7100010851000109A
:10102000E5100010FB68DA6A7B685B681A43FB68AE
:10103000DA62FB68DA6D7B685B68DB431A40FB6849
:10104000DA65FB689A6A7B685B68DB431A40FB6879
:101050009A6259E0FB68DA6A7B685B68DB431A4096
:10106000FB68DA62FB68DA6D7B685B68DB431A4019
:10107000FB68DA65FB689A6A7B685B681A43FB6801
:101080009A6241E0FB68DA6A7B685B68DB431A407E
:10109000FB68DA62FB68DA6D7B685B68DB431A40E9
:1010A000FB68DA65FB689A6A7B685B68DB431A4019
:1010B000FB689A6228E0FB68DA6A7B685B681A431F
:1010C000FB68DA62FB68DA6D7B685B68DB431A40B9
:1010D000FB68DA65FB689A6A7B685B681A43FB68A1
:1010E0009A6211E0FB68DA6D7B685B681A43FB6803
:1010F000DA65FB689A6A7B685B681A43FB689A62E8
:1011000002E06FF0020300E0002318461437BD46EA
:101110005DF8047B704700BF80B483B000AF786097
:1011200039607B683A689A6300BF0C37BD465DF84A
:10113000047B704780B483B000AF786039607B680F
:101140003A68DA6300BF0C37BD465DF8047B704730
:1011500080B483B000AF786039607B683A689A6485
:1011600000BF0C37BD465DF8047B704780B483B088
:1011700000AF78607B681B6C18460C37BD465DF885
:10118000047B704780B485B000AFF8600B467A608E
:10119000FB72FB7A002B02D0012B0AD012E0FB6815
:1011A000D3F8C0207B68DB431A40FB68C3F8C0203B
:1011B0000BE0FB68D3F8C0207B681A43FB68C3F8D8
:1011C000C02002E06FF0020300E00023184614374D
:1011D000BD465DF8047B704780B485B000AFF86011
:1011E0000B467A60FB72FB681A6B7B681A43FB68DC
:1011F0001A63FB687A685A60FB7A032B48D801A20D
:1012000052F823F015120010371200105912001076
:1012100075120010FB687A685A61FB687A685A6038
:10122000FB687A681A67FB687A68DA67FB687A682D
:10123000C3F888202FE0FB687A681A61FB687A6837
:101240005A60FB687A681A67FB687A68DA67FB6835
:101250007A68C3F888201EE0FB687A68C3F88820A3
:10126000FB687A68DA67FB687A681A67FB687A68ED
:101270009A6010E0FB687A68C3F88820FB687A6897
:10128000DA67FB687A68DA66FB687A689A6002E077
:101290006FF0020300E0002318461437BD465DF8E6
:1012A000047B704780B485B000AFF8600B467A606D
:1012B000FB72FB7A032B53D801A252F823F000BF34
:1012C000D1120010F71200101B1300103F13001072
:1012D000FB68D3F8B0207B68DB431A40FB68C3F897
:1012E000B020FB68D3F8B4207B68DB431A40FB686E
:1012F000C3F8B42046E0FB68D3F8B0207B681A43FB
:10130000FB68C3F8B020FB68D3F8B4207B68DB43EC
:101310001A40FB68C3F8B42034E0FB68D3F8B0206F
:101320007B68DB431A40FB68C3F8B020FB68D3F846
:10133000B4207B681A43FB68C3F8B42022E0FB6842
:10134000D3F8B0207B681A43FB68C3F8B020FB6871
:10135000D3F8B4207B681A43FB68C3F8B42011E0CB
:10136000FB68D3F8B0207B68DB431A40FB68C3F806
:10137000B020FB68D3F8B4207B68DB431A40FB68DD
:10138000C3F8B420002318461437BD465DF8047B2B
:10139000704700BF80B586B000AFF860B9607A6072
:1013A000FB681B4A934208D0FB681A4A934201D15A
:1013B000012303E04FF0FF3300E000237B617B69F2
:1013C000002B03D07B69012B07D00DE00D2001F02D
:1013D000F7FC1148FFF74CFC09E01C2001F0F0FC81
:1013E0000E48FFF745FC02E06FF002030BE07A685D
:1013F000B968F86800F03AF938613B69002B01D010
:101400003B6900E0002318461837BD4680BD00BF89
:1014100000D0014000E001407C0602108806021066
:1014200080B485B000AFF860B9607A60FB68002BCB
:1014300006D0BB68B3F5806F02D27B68002B02D068
:101440006FF0020314E0FB6800225A64BB687F2B34
:1014500005D9FB685B6C43F40042FB685A64FB6887
:101460005A6CBB68C3F309031A43FB685A64002330
:1014700018461437BD465DF8047B704780B582B0CE
:1014800000AF78607B68154A934208D07B68144AA5
:10149000934201D1012303E04FF0FF3300E000232A
:1014A000002B02D0012B07D00DE0102001F0F2FD3F
:1014B0000D2001F05AFC09E0202001F0EBFD1C207A
:1014C00001F053FC02E06FF0020303E0786800F0E3
:1014D00073F9034618460837BD4680BD00D0014069
:1014E00000E0014080B582B000AF786039603B68B1
:1014F000074A934202D96FF0100304E03968786814
:1015000000F0F0F9034618460837BD4680BD00BF1D
:1015100040420F0080B582B000AF7860786800F07C
:1015200075FA034618460837BD4680BD80B582B0BF
:1015300000AF7860786800F09FFA034618460837D5
:10154000BD4680BD80B582B000AF7860786800F09D
:10155000B7FA034618460837BD4680BD80B584B04B
:1015600000AFF860B9607A607A68B968F86800F02E
:10157000C5FA034618461037BD4680BD80B584B015
:1015800000AFF860B9607A607A68B968F86800F00E
:10159000E0FA034618461037BD4680BD80B582B0DC
:1015A00000AF7860786800F000FB00BF0837BD46E8
:1015B00080BD80B582B000AF7860786800F00DFB28
:1015C00000BF0837BD4680BD80B584B000AFF8606D
:1015D000B9607A607A68B968F86800F016FB00BFF5
:1015E0001037BD4680BD80B582B000AF78603960ED
:1015F0003968786800F01BFB034618460837BD467B
:1016000080BD80B582B000AF7860786800F0B2FB32
:10161000034618460837BD4680BD80B582B000AF8E
:10162000786039603968786800F0D4FC0346184661
:101630000837BD4680BD80B582B000AF78603960A4
:101640003968786800F0E6FC034618460837BD465E
:1016500080BD80B582B000AF78600821786800F066
:10166000EFFF00BF0837BD4680BD000080B586B0E3
:1016700000AFF860B9607A60FB68002B02D14FF0D0
:10168000FF338EE0FB68494A934208D0FB68484A22
:10169000934201D1012303E04FF0FF3300E0002328
:1016A000FB751021F868FFF79EFF38613B69002B3E
:1016B00001D03B6975E0FB681B6843F00102FB68E1
:1016C0001A60F868FFF76AFFF868FFF772FF0221F7
:1016D000F868FFF7B0FF0621F868FFF79EFFBB68C8
:1016E000002B19D100227968F868FFF799FEFB6892
:1016F0002E4A934208D0FB682D4A934201D1012320
:1017000003E04FF0FF3300E000232A4A5B0113445B
:10171000043300221A6019E0FB681B6843F00202E0
:10172000FB681A60FB68214A934208D0FB68204A94
:10173000934201D1012303E04FF0FF3300E0002387
:101740001C4A5B011344043301221A6097F91730D5
:10175000184A5B01134408336FF001021A6097F9CD
:101760001730144A5B0113440C336FF001021A6006
:1017700097F917300F4A5B011344103300221A60A7
:1017800097F917300B4A5B011344143300221A6097
:1017900097F91730074A5B011344183300221A7077
:1017A000002318461837BD4680BD00BF00D0014059
:1017B00000E001401419002080B58CB000AF7860C3
:1017C0007B68002B02D14FF0FF3381E07B68424AF7
:1017D000934208D07B68414A934201D1012303E040
:1017E0004FF0FF3300E0002387F82F307B680022A2
:1017F0001A607B680022DA607B6800225A617B688D
:101800009A687B689A607B681A697B681A617B6852
:101810000022DA617B6800221A627B6800225A6229
:101820007B6800229A6297F92F302D4A5B0113449E
:10183000184620231A46002113F024FB7868FFF78E
:10184000ADFE7868FFF7B5FE97F92F30244A5B01AB
:10185000134418331B78002B39D0FEF7E7FF97F9B4
:101860002F301F4A5B01134408331B68002B12DB27
:1018700097F92F301A4A5B01134408331B68184646
:10188000FEF7DCFF97F92F30154A5B01134408334C
:101890006FF001021A6097F92F30114A5B0113446F
:1018A0000C331B68002B12DB97F92F300C4A5B01BD
:1018B00013440C331B681846FEF7C0FF97F92F300E
:1018C000074A5B0113440C336FF001021A600023D6
:1018D00018463037BD4680BD00D0014000E00140D1
:1018E0001419002080B588B000AF786039607B683B
:1018F000002B02D14FF0FF337AE03B683E4A93421F
:1019000040D93B683D4A93423CD83D4B1B685A083E
:101910003B68B2FBF3F37B617B695B00394AA2FB56
:1019200003235B08013B3B617B69364AA2FB03232F
:101930005B08013BBB617B6903F00103002B02D014
:10194000BB690133BB61BB690F2B02DC3B690F2B09
:1019500002DD6FF002034BE03B69DBB23B61BB6928
:101960001B029BB2BB613A69BB6913431A467B6891
:10197000DA637B681B6843F400427B681A60224B81
:101980003B6006E03B681D4A934202D96FF00203B8
:101990002EE01B4B1B685A083B68B2FBF3F37B61DC
:1019A0007B695B08013BFB617B695B08013BFB607A
:1019B0007B6903F00103002B02D0FB690133FB615B
:1019C000FB69B3F5007F02D2FB68002B02D16FF0F8
:1019D00002030DE0FB68C3F308027B685A63FB69EE
:1019E000C3F308027B689A637868FFF793FD0346A8
:1019F00018462037BD4680BD40420F0040E133000D
:101A0000A8130020ABAAAAAA801A060080B485B049
:101A100000AF78600223FB607B681B6803F400431F
:101A2000002B0DD07B68DB6BDBB2FA681344FB60E4
:101A30007B68DB6B1B0ADBB2FA681344FB600DE0CA
:101A40007B685B6BC3F30803FA681344FB607B6835
:101A50009B6BC3F30803FA681344FB60054B1B68D8
:101A60005A08FB68B2FBF3F318461437BD465DF81D
:101A7000047B7047A813002080B483B000AF786067
:101A80007B68002B02D14FF0FF3313E07B681B6BA8
:101A900003F00103002B06D07B681B6B43F00202AE
:101AA0007B681A6305E07B681B6B43F001027B686F
:101AB0001A63002318460C37BD465DF8047B704757
:101AC00080B483B000AF78607B68002B02D14FF008
:101AD000FF330DE07B681B6B43F004027B681A63E5
:101AE00000BF7B681B6B03F00403002BF9D10023BC
:101AF00018460C37BD465DF8047B704780B487B04C
:101B000000AFF860B9607A6000237B61FB68002B4E
:101B100002D0BB68002B0BD14FF0FF3313E0FB6802
:101B2000D96A7B695A1C7A61BA681344CAB21A70BE
:101B30007A687B699A4205D9FB685B6803F0020307
:101B4000002BECD07B6918461C37BD465DF8047B42
:101B5000704780B487B000AFF860B9607A60002346
:101B60007B61FB68002B02D0BB68002B0CD14FF0CF
:101B7000FF3314E07B695A1C7A61BA6813441B78FE
:101B8000DBB21A46FB68DA627A687B699A4205D949
:101B9000FB685B6803F01003002BEBD07B691846F1
:101BA0001C37BD465DF8047B704780B483B000AF3E
:101BB00078607B68DB6943F080027B68DA6100BF94
:101BC0007B68DB6903F08003002BF9D100BF00BF05
:101BD0000C37BD465DF8047B704780B483B000AF1E
:101BE00078607B685B6A43F080027B685A6200BF62
:101BF0007B685B6A03F08003002BF9D100BF00BF54
:101C00000C37BD465DF8047B704780B485B000AFEB
:101C1000F860B9607A60FB68BA689A60FB687A68B5
:101C20001A6100BF1437BD465DF8047B704780B56C
:101C300086B000AF786039607B68002B02D14FF02E
:101C4000FF3393E06FF008037B617B681B6843F010
:101C500001027B681A607B681B6803F48063FB6089
:101C60007B68002B02D14FF0FF337FE07B681B685D
:101C700043F480627B681A6000233B6162E00A20C3
:101C800001F004F87B681B6823F040027B681A604F
:101C90000A2000F0FBFF7B681B6803F48073002BB5
:101CA00006D07B681B6843F0C0027B681A6046E080
:101CB0000A2000F0EBFF7B681B6823F080027B6842
:101CC0001A600A2000F0E2FF7B681B6803F40073CF
:101CD000002B06D07B681B6843F0C0027B681A604B
:101CE0002DE00A2000F0D2FF7B681B6843F08002E1
:101CF0007B681A600A2000F0C9FF7B681B6803F448
:101D00000073002B06D17B681B6843F0C0027B6820
:101D10001A6014E00A2000F0B9FF7B681B6843F0EA
:101D200040027B681A600A2000F0B0FF7B681B68E5
:101D300003F48073002B02D000237B6106E03B6933
:101D400001333B613A693B689A4298D3FB68002BA8
:101D500005D17B681B6823F480627B681A607B680E
:101D60001B6823F001027B681A607B6918461837EC
:101D7000BD4680BD80B586B000AF78607B681B68CB
:101D8000FB6000237B6100233B617B685B687F2BEA
:101D900002D96FF0100315E1FB688C4A934206D01C
:101DA000FB688B4A934202D06FF002030AE1FB68A2
:101DB0001B6803F00203002B02D16FF0060301E160
:101DC00007226FF07F41F868FFF7FEFBF868FFF726
:101DD000F0FBF868FFF7E2FBFB680022DA60FB68C3
:101DE00000225A617B685B69002B03D07B68DB684B
:101DF000002B34D07B685B685A00FB68DA62FB68B2
:101E00001B6B43F00102FB681A6328E0FB689B68C8
:101E100003F02003002B13D07B689A687B69D118EC
:101E20007B68DA687B69D31A1A46F868FFF7A6FB65
:101E300003461A467B6913447B61FB6820229A6043
:101E4000FB689B6803F4FE43002B08D07B687A692B
:101E5000DA60F868FFF776FB6FF00803B2E07B68A2
:101E6000DB687A699A42D1D300221121F868FFF722
:101E7000ABFB7B685B69002B73D07B685B69B3F558
:101E8000807F03D9FB6800221A6203E07B685A69ED
:101E9000FB681A62F868FFF749FB00BFFB681B6B21
:101EA00003F00203002BF9D17B685B685B0043F011
:101EB0000102FB68DA6254E0FB689B6803F01103DF
:101EC000002B13D07B681A693B69D1187B685A696B
:101ED0003B69D31A1A46F868FFF740FB03461A46D7
:101EE0003B6913443B61FB6810229A60FB689B6866
:101EF00003F4FE43002B08D07B683A695A61F86806
:101F0000FFF720FB6FF008035CE0FB689B6803F0C1
:101F10000103002B25D07B685B693A699A4220D97E
:101F20007B685A693B69D31AB3F5807F03D9FB6894
:101F300000221A6205E07B685A693B69D21AFB6885
:101F40001A62FB681B6B43F00202FB681A63FB68B2
:101F500001229A607B685B685B0043F00102FB68CA
:101F6000DA627B685B693A699A42A5D37B689B69B0
:101F7000002B06D0FB681B6B43F00202FB681A6360
:101F80000CE0FB681B6B43F00402FB681A6300BFA4
:101F9000FB689B6803F04003002BF9D000BFFB688F
:101FA0009B6803F00103002BF9D0FB6841229A6083
:101FB000FB689B6803F4FE43002B02D06FF008031C
:101FC00000E0002318461837BD4680BD00D0014010
:101FD00000E0014080B485B000AF786039607B6874
:101FE0009B69DBB2FB603A68FB689A4202D96FF0EA
:101FF000020309E07B68DB6923F470623B681B0223
:102000001A437B68DA61002318461437BD465DF831
:10201000047B704780B485B000AF786039607B681E
:102020009B691B0ADBB2FB603A68FB689A4202D9E3
:102030006FF0020309E07B685B6A23F470623B681F
:102040001B021A437B685A62002318461437BD46A8
:102050005DF8047B7047000080B584B000AF786005
:1020600039607B680E4A934208D07B680D4A9342E0
:1020700001D1012303E04FF0FF3300E000230A4ABF
:1020800052F82330FB60FB68DB69002B04D0FB684F
:10209000DB693968F868984700BF1037BD4680BDD6
:1020A00000D0014000E001405419002080B483B00A
:1020B00000AF78607B680022DA607B6800225A619A
:1020C0007B689A687B689A607B681A697B681A618A
:1020D0007B680B4A934208D07B680A4A934201D13D
:1020E000012303E04FF0FF3300E00023064A002104
:1020F00042F8231000BF0C37BD465DF8047B7047E3
:1021000000D0014000E001405419002080B586B0A5
:1021100000AF78608F4A7B6852F823307B618E4A2B
:102120007B6852F823303B617B68002B06D07B68CC
:10213000012B01D1894B02E0002300E0884BFB60BA
:10214000884A7B6852F82330BB60FB689B6803F4C5
:10215000FE43002B19D0FB689A68FB689A60FB6805
:102160001A69FB681A61FB680022DA60FB680022CA
:102170005A61F868FFF7E6F96FF00801F868FFF7B1
:102180006BFFF868FFF792FFF8E0BB68DB687A69DD
:102190009A4243D2FB689B6803F02003002B13D0C4
:1021A000BB689A687B69D118BB68DA687B69D31A07
:1021B0001A46F868FFF7E2F903461A467B691344AA
:1021C0007B61FB6820229A60BB68DB687A699A426F
:1021D00006D2FB68DB6843F02002FB68DA6005E0AA
:1021E000FB68DB6823F02002FB68DA60BB68DB6811
:1021F0007A699A4212D1BB685B69002B0ED0FB68EA
:102200001B6B43F00202FB681A63FB6801229A60B1
:10221000FB68DB6843F00102FB68DA60BB685B695E
:102220003A699A4219D2FB689B6803F01103002BAC
:1022300013D0BB681A693B69D118BB685A693B69FE
:10224000D31A1A46F868FFF789F903461A463B691C
:1022500013443B61FB6810229A60BB68DB687A69B3
:102260009A423AD1BB685B693A699A4235D0FB68B9
:102270009B6803F00103002B2FD0FB6801229A60BA
:102280003B69002B06D1BB685B685B0043F0010231
:10229000FB68DA62BB685A693B69D31AB3F5807F81
:1022A00003D9FB6800221A6205E0BB685A693B69E2
:1022B000D21AFB681A62BB685B693A699A4206D215
:1022C000FB68DB6843F01102FB68DA6005E0FB683D
:1022D000DB6823F01102FB68DA60BB68DB687A69AF
:1022E0009A4241D1BB685B693A699A423CD1FB682A
:1022F0000022DA60FB6800225A61FB689A68FB687A
:102300009A60FB681A69FB681A61BB689B69002BBD
:1023100006D0FB681B6B43F00202FB681A6305E002
:10232000FB681B6B43F00402FB681A63FB689B6845
:1023300003F4FE43002B05D06FF00801F868FFF7A7
:102340008BFE03E00021F868FFF786FEF868FFF7D0
:10235000ADFE13E05C1900206419002000E001408C
:1023600000D001405419002006497B687A6941F881
:10237000232005497B683A6941F823201837BD4678
:1023800080BD00BF5C1900206419002080B586B0B4
:1023900000AFF860B9607A603B60FB689B687B6166
:1023A0003B6800221A607B6903F4FE43002B30D0A7
:1023B0003B686FF008021A60BB68002B04D0BB6852
:1023C0003A680421F868984707226FF07F41F8685F
:1023D000FFF71BFCF868FFF700FCF868FFF7E5FB68
:1023E0007B6800221A607B68043300221A60FB6855
:1023F000904A934208D0FB688F4A934201D101234F
:1024000003E04FF0FF3300E000238C4A002142F844
:1024100023107B681B6803F01003002B06D17B6838
:1024200004331B6803F00103002B20D07B6903F009
:102430001003002B0AD0BB68002B04D0BB6800221D
:102440000221F8689847FB6810229A60FB681B69B4
:1024500003F00103002B0AD0BB68002B04D0BB683B
:1024600000220621F8689847FB6801221A617B6800
:102470001A6848F220031340002B06D17B6804330E
:102480001B6803F00203002B4DD07B6903F020038F
:10249000002B0AD0BB68002B04D0BB6800220321AC
:1024A000F8689847FB6820229A60FB681B6903F074
:1024B0000203002B0AD0BB68002B04D0BB680022AB
:1024C0000521F8689847FB6802221A617B6903F4CA
:1024D0000043002B27D03B6800221A60BB68002B0A
:1024E00004D0BB683A680421F8689847FB684FF449
:1024F00000429A607B6800221A607B6804330022E5
:102500001A60FB684B4A934208D0FB684A4A9342E0
:1025100001D1012303E04FF0FF3300E00023474ADD
:10252000002142F823107B681B6803F00803002B8E
:102530003DD07B6903F00803002B38D0FB681B6893
:1025400003F40063002B1BD0BB68002B04D0BB68D6
:1025500000220121F8689847FB684FF480029A60D6
:10256000FB6808229A60FB684FF400429A607B681F
:102570004FF621721A607B68043302221A6016E05B
:10258000BB68002B04D0BB6800220021F868984784
:10259000FB684FF400029A60FB6808229A607B682F
:1025A00047F611721A607B68043301221A607B6857
:1025B0001B6803F00103002B37D07B6903F0400355
:1025C000002B27D03B6800221A60BB68002B04D088
:1025D000BB683A680421F8689847FB6840229A6013
:1025E0007B6800221A607B68043300221A60FB6853
:1025F000104A934208D0FB680F4A934201D101234D
:1026000003E04FF0FF3300E000230C4A002142F8C2
:1026100023100AE07B6903F00103002B05D0FB685F
:1026200001229A607B6808221A6000BF1837BD46F5
:1026300080BD00BF00D0014000E0014054190020DF
:1026400080B588B000AF786039607B681C4A9342DF
:1026500008D07B681B4A934201D1012303E04FF06D
:10266000FF3300E00023FB61FB69002B23DB7B6869
:102670001B6803F00203002B03D0F869FFF746FD47
:102680001AE0114AFB6952F82330BB617B68DB68B2
:10269000FB607B685B693B6107F1140307F10C0287
:1026A000B9697868FFF772FEFA687B68DA603A69A0
:1026B0007B685A6100E000BF2037BD4680BD00BF87
:1026C00000D0014000E001405419002080B582B0E4
:1026D00000AF78607968044800F0EBF803461846CC
:1026E0000837BD4680BD00BF0060004080B500AF28
:1026F000024800F0F6F80346184680BD006000402E
:1027000080B500AF024800F014F90346184680BDBA
:102710000060004080B582B000AF78600B46FB706F
:1027200000F07BFB112000F0B5FCFB781A467968BD
:10273000034800F026F9034618460837BD4680BD19
:102740000060004080B582B000AF786079680448CE
:1027500000F064F8034618460837BD4680BD00BF48
:102760000060004080B582B000AF786079680448AE
:1027700000F079F8034618460837BD4680BD00BF13
:102780000060004080B500AF024800F031F9034618
:10279000184680BD0060004080B582B000AF786010
:1027A0007968044800F032F9034618460837BD46F8
:1027B00080BD00BF0060004080B500AF024800F05F
:1027C00017F80346184680BD0060004080B400AF93
:1027D00000BF064B1B6903F00803002BF9D100BFB3
:1027E00000BFBD465DF8047B704700BF006000403D
:1027F00080B483B000AF7860074B1B6903F0080317
:10280000002B02D06FF0050300E0002318460C37C0
:10281000BD465DF8047B70470060004080B582B023
:1028200000AF786039603B6803F026033B603B688B
:10283000002B02D16FF0020311E0FFF7C7FF7B68A6
:102840001A693B681A437B681A613B6823F02003CE
:102850003B603B68002B01D0FFF7B8FF0023184610
:102860000837BD4680BD80B582B000AF7860396062
:102870003B6803F026033B603B68002B02D16FF0FE
:10288000020312E0FFF7A2FF7B681A693B68DB4393
:102890001A407B681A613B6823F020033B603B6869
:1028A000002B01D0FFF792FF002318460837BD46E2
:1028B00080BD80B582B000AF786039607868FFF77E
:1028C00097FF0346002B02D06FF0050305E03B683D
:1028D000C3F313027B689A60002318460837BD468D
:1028E00080BD80B582B000AF78607868FFF780FF68
:1028F0000346002B02D06FF0050316E07B681B69CE
:1029000043F400427B681A61FFF760FF7B681B6934
:1029100043F001027B681A61FFF758FF7B681B696F
:1029200023F400427B681A61002318460837BD462D
:1029300080BD80B582B000AF78607868FFF758FF3F
:102940000346002B02D06FF0050316E07B681B697D
:1029500043F400427B681A61FFF738FF7B681B690C
:1029600023F001027B681A61FFF730FF7B681B6967
:1029700023F400427B681A61002318460837BD46DD
:1029800080BD80B584B000AFF860B9607A60F86847
:10299000FFF72EFF0346002B02D06FF0050323E064
:1029A000FB684FF400421A61FFF710FFFB6800223A
:1029B0001A61FFF70BFFFB681B6943F40042FB68D9
:1029C0001A61FFF703FFFB687A685A60FFF7FEFEA3
:1029D000FB68BA681A60FFF7F9FEFB681B6923F40D
:1029E0000042FB681A61002318461037BD4680BDBF
:1029F00080B483B000AF78607B681B6903F0D003BC
:102A000018460C37BD465DF8047B704780B483B030
:102A100000AF786039607B681B693A6802F0D002C9
:102A2000D2431A407B681A61002318460C37BD4612
:102A30005DF8047B7047000080B500AF0F4B1B684A
:102A400003F48033002B16D00D4B1B68002B05DDE3
:102A50000B4B1B68013B0A4A13600CE000F0F6F8D0
:102A6000084B1B68002B06D0064B1B6800209847BC
:102A7000044B00221A6000BF80BD00BF10E000E0E0
:102A800000000020741900202DE9B04386B000AF8B
:102A900078603649896879613449096821F4803160
:102AA000334801603149096801F00101002911D161
:102AB0002E496FF07F4048602C496FF07F4088605E
:102AC0002A49052008606FF07F4179614FF08071DD
:102AD000396103E02549496801313961796800208D
:102AE000884681462349096800200A46034602FBBE
:102AF00009F008FB03F10144A8FB02454B191D46F0
:102B00001D4A4FF000032046294610F0AFFE024652
:102B10000B461346FB60FA683B69B2FBF3F31A46B7
:102B2000164B1A60FB683A69B3FBF2F2396901FB94
:102B300002F29B1ABB60BA687B699A420CD30F4BB6
:102B40001B6801330D4A13607A69BB68D21A3B696E
:102B500013440B4A136004E07A69BB68D31A084A2D
:102B6000136000BF1837BD46BDE8B08310E000E039
:102B700070190020A813002040420F000000002020
:102B80006C19002080B582B000AF78603960104ABF
:102B90003B6813600F4B1B68002B02DD6FF00503D1
:102BA00012E07B68002B01D100230DE07868FFF76D
:102BB0006BFF084B1B68002B05DD074B1B68064AA3
:102BC00043F002031360002318460837BD4680BD5A
:102BD000741900200000002010E000E080B500AF74
:102BE000164B1B68002B0CDA154B1B68002B06D00C
:102BF000134B1B6800209847114B00221A600023DA
:102C00001AE00E4B1B68002B14D10E4B9A680E4B2A
:102C10001B689A420ED800F019F8094B1B68002B6C
:102C200006D0074B1B6800209847054B00221A600E
:102C3000002301E06FF00503184680BD000000206E
:102C40007419002010E000E06C19002080B500AF7E
:102C50000A4B1B68002B07D0084B1B686FF00F0056
:102C60009847064B00221A60054A064B1B68136002
:102C7000054B4FF0FF321A6000BF80BD7419002071
:102C800010E000E0701900200000002080B582B044
:102C900000AF7860164B1B68002B02DD6FF0050358
:102CA00021E07B68002B01D100231CE07868FFF74E
:102CB000EBFE0AE00F4B1B6803F48033002B04D0BB
:102CC0000B4B1B68013B0A4A1360094B1B68002B26
:102CD000F0DC00BF074B9A68074B1B689A42F9D893
:102CE000FFF7B4FF002318460837BD4680BD00BF7C
:102CF0000000002010E000E06C19002080B489B0D2
:102D000000AF786039607B68FB61FB6953E8003F86
:102D1000BB61BB69002B02D06FF005030FE03B687D
:102D20007B617B683B6139697A6941E80023FB601C
:102D3000FB68002BE7D1BFF35F8F00BF002318466D
:102D40002437BD465DF8047B704780B483B000AF84
:102D50007860BFF35F8F00BF7B6800221A6000BFFE
:102D60000C37BD465DF8047B704780B483B000AF7C
:102D70000346FB71FB791F2B0FD9FB79203BFB71BD
:102D80004FF080439B6CFA79012101FA02F211465F
:102D90004FF080420B4393640BE04FF080435B6A3B
:102DA000FA79012101FA02F211464FF080420B43F9
:102DB0005362002318460C37BD465DF8047B70470C
:102DC00080B483B000AF0346FB71FB791F2B10D991
:102DD000FB79203BFB714FF080439B6CFA7901211A
:102DE00001FA02F2D24311464FF080420B40936445
:102DF0000CE04FF080435B6AFA79012101FA02F29C
:102E0000D24311464FF080420B40536200231846D4
:102E10000C37BD465DF8047B704780B500AF4FF0BE
:102E200080439B684FF0804243F4003393604FF03F
:102E3000007000F00FF90346002B02D06FF0090379
:102E400000E00023184680BD80B584B000AF034683
:102E5000FB714FF080439B6803F46063FB60FB7978
:102E6000062B00F2968001A252F823F0892E001062
:102E7000932F00105D2F0010BF2E0010E92E0010C0
:102E8000232F00105D2F00104FF080439B684FF000
:102E9000804243F4802393604FF0806000F0DAF8C2
:102EA0000346002B02D06FF00903CFE04FF08043C0
:102EB0009B684FF0804223F4606393606CE04FF0B6
:102EC000005000F0C7F80346002B02D06FF0090352
:102ED000BCE04FF080439B6823F460634FF0804276
:102EE00043F4C063936057E04FF080439B684FF01A
:102EF000804243F4002393604FF0006000F0AAF892
:102F00000346002B02D06FF009039FE04FF080438F
:102F10009B6823F460634FF0804243F40063936046
:102F20003AE04FF080439B684FF0804243F48013B7
:102F300093604FF0805000F08DF80346002B02D0D4
:102F40006FF0090382E04FF080439B6823F46063D5
:102F50004FF0804243F4206393601DE04FF08043C4
:102F60009B684FF0804243F4003393604FF0007051
:102F700000F070F80346002B02D06FF0090365E003
:102F80004FF080439B684FF0804223F4606393606E
:102F900002E06FF0020359E04FF4005000F05AF8DD
:102FA0000346002B0ED04FF080439B6823F46062F1
:102FB000FB6803F460634FF0804113438B606FF054
:102FC000090343E0FB79062B3DD801A252F823F018
:102FD000ED2F00104730001035300010FF2F00108B
:102FE0001130001023300010353000104FF08043B6
:102FF0009B684FF0804223F4D013936023E04FF09E
:1030000080439B684FF0804223F4F01393601AE0F2
:103010004FF080439B684FF0804223F4B0139360DD
:1030200011E04FF080439B684FF0804223F460230F
:10303000936008E04FF080439B684FF0804223F498
:10304000E013936000BFFDF7FFF800231846103728
:10305000BD4680BD80B582B000AF786000214FF4DE
:103060007A70FFF78FFD4FF080439A687B681340BA
:10307000002B03D0FFF7EAFD002307E0FFF7AEFDCA
:10308000034613F1060FEED06FF009031846083718
:10309000BD4680BD80B483B000AF0346FB71FB79B1
:1030A0001F2B0FD9FB79203BFB71FB7901229A4042
:1030B0004FF080435A6400BF4FF080435B6C002B9D
:1030C000FAD10BE0FB7901229A404FF080435A601D
:1030D00000BF4FF080435B68002BFAD100231846F5
:1030E0000C37BD465DF8047B704780B584B000AFF7
:1030F0003B460D21184600F01DF83B789E2B94BFEF
:1031000001230023DAB23B7803F00F03092BCCBF75
:1031100001230023DBB21343DBB2002B04D04FF0BA
:1031200080431B6DDBB200E03B7818461037BD468C
:1031300080BD000080B588B000AF786039603B6822
:103140000D2B02D06FF0020386E07B68002B02D1CA
:103150004FF0FF3380E04FF08450FDF7EDFB4FF070
:1031600084531B68BB603E4B1B68FB603D4B1B6878
:103170003B613D4B1B687B613C4B1B68BB613C4B1F
:103180001B68FB614FF08450FDF7E6FBBB68DB0B6F
:10319000DAB27B681A70BB68DA0D7B680133D2B291
:1031A0001A70BB68DA0F7B680233D2B21A707B6880
:1031B00002331978FB68DBB25B00DAB27B6802335A
:1031C0000A43D2B21A70FB68DA097B680333D2B2C1
:1031D0001A70FB68DA0B7B680433D2B21A70FB6892
:1031E000DA0D7B680533D2B21A703B69DA0B7B6863
:1031F0000633D2B21A703B69DA0D7B680733D2B25C
:103200001A703B69DA0F7B680833D2B21A707B6898
:10321000083319787B69DBB25B00DAB27B6808336C
:103220000A43D2B21A707B69DA097B680933D2B2D9
:103230001A707B69DA0B7B680A33D2B21A707B6929
:10324000DA0D7B680B33D2B21A70BB69DA0B7B687C
:103250000C33D2B21A70002318462037BD4680BD09
:1032600004008010080080100C00801010008010F6
:103270001400801080B582B000AF7860786800F0EC
:1032800004F800BF0837BD4680BD80B483B000AFEE
:1032900078607B680122DA6000BF0C37BD465DF8BC
:1032A000047B704780B582B000AF786000BF78685B
:1032B00000F018FA0346002BF9D0786800F0C6F940
:1032C000034618460837BD4680BD80B582B000AFC2
:1032D00078600B46FB7000BF786800F035FA034653
:1032E000002BF9D0FB781946786800F0BBF903464B
:1032F00018460837BD4680BD80B584B000AF786001
:103300003960786800F084F8F860FB68002B01D021
:10331000FB6869E07B68364A93420ED07B68354A89
:10332000934208D07B68344A934201D1022305E0DE
:103330004FF0FF3302E0012300E00023022B14D002
:10334000022B19DC002B02D0012B07D014E02B48F4
:10335000FDF78EFC0920FFF733FD10E02848FDF74C
:1033600087FC0A20FFF72CFD09E02648FDF780FCCA
:103370002120FFF725FD02E06FF0020334E07B68B7
:103380001B4A93420ED07B681A4A934208D07B684E
:10339000194A934201D1022305E04FF0FF3302E0C6
:1033A000012300E00023184A002142F823107B6823
:1033B0000F4A93420ED07B680E4A934208D07B6836
:1033C0000D4A934201D1022305E04FF0FF3302E0A2
:1033D000012300E000230D4A002142F82310396840
:1033E000786800F0DCFA034618461037BD4680BD09
:1033F0000020044000300440004004403406021025
:103400004C0602106406021078190020841900206E
:1034100080B582B000AF78607B681C4A93420ED0C2
:103420007B681B4A934208D07B681A4A934201D1B9
:10343000022305E04FF0FF3302E0012300E0002308
:10344000022B14D0022B19DC002B02D0012B07D049
:1034500014E00B20FFF71EFE0920FFF786FC10E0AA
:103460000C20FFF717FE0A20FFF77FFC09E01C2065
:10347000FFF710FE2120FFF778FC02E06FF0020357
:1034800000E0002318460837BD4680BD00200440F8
:10349000003004400040044080B582B000AF786046
:1034A00039603968786800F0C1FA03461846083771
:1034B000BD4680BD80B582B000AF7860786800F00E
:1034C0009DFB034618460837BD4680BD80B582B0D7
:1034D00000AF786039603968786800F01BFC0346FB
:1034E00018460837BD4680BD80B582B000AF786011
:1034F0000B46FB70FB781946786800F043FC0346E6
:1035000018460837BD4680BD80B582B000AF7860F0
:103510000B46FB70FB781946786800F06DFC03469B
:1035200018460837BD4680BD80B584B000AFF8604E
:103530000B467A60FB72FB681A4A93420ED0FB6816
:10354000194A934208D0FB68184A934201D10223DA
:1035500005E04FF0FF3302E0012300E00023022BDF
:103560000ED0022B10DC002B02D0012B04D00BE07C
:103570000F48FDF77DFB0AE00E48FDF779FB06E0FA
:103580000D48FDF775FB02E06FF0020306E0FB7AE1
:103590007A681946F86800F01DFD03461846103792
:1035A000BD4680BD0020044000300440004004407F
:1035B00040060210580602107006021080B582B054
:1035C00000AF78607B680B4A93420AD07B680A4A56
:1035D000934206D07B68094A934202D06FF00203FF
:1035E00003E07868FFF75EFE034618460837BD46DD
:1035F00080BD00BF00200440003004400040044073
:1036000080B582B000AF78600B46FB707B680C4AD7
:1036100093420AD07B680B4A934206D07B680A4AE1
:10362000934202D06FF0020305E0FB7819467868F8
:10363000FFF74BFE034618460837BD4680BD00BF66
:1036400000200440003004400040044080B582B0B7
:1036500000AF7860786800F025FD0346184608370B
:10366000BD4680BD80B582B000AF78600B46FB7070
:10367000FB781946786800F03FFD03461846083786
:10368000BD4680BD80B584B000AFF860B9607A6097
:103690007A68B968F86800F05DFD0346184610378F
:1036A000BD4680BD80B584B000AFF860B9607A6077
:1036B0007A68B968F86800F078FD03461846103754
:1036C000BD4680BD80B584B000AFF860B9607A6057
:1036D0007A68B968F86800F092FD0346184610371A
:1036E000BD4680BD80B582B000AF78607B680B4A74
:1036F00093420AD07B680A4A934206D07B68094A03
:10370000934202D06FF0020303E0786800F09DFD61
:10371000034618460837BD4680BD00BF0020044060
:10372000003004400040044080B584B000AFF86031
:10373000B9607A607A68B968F86800F095FD034668
:1037400018461037BD4680BD80B582B000AF7860A6
:103750007B680B4A93420AD07B680A4A934206D0A0
:103760007B68094A934202D06FF0020303E0786855
:1037700000F0A0FD034618460837BD4680BD00BFD7
:1037800000200440003004400040044080B582B076
:1037900000AF786039603968786800F09FFD0346B3
:1037A00018460837BD4680BD80B582B000AF78604E
:1037B0007B680B4A93420AD07B680A4A934206D040
:1037C0007B68094A934202D06FF0020303E07868F5
:1037D00000F0B8FD034618460837BD4680BD00BF5F
:1037E00000200440003004400040044080B582B016
:1037F00000AF786039603968786800F0B1FD034641
:1038000018460837BD4680BD80B582B000AF7860ED
:103810007B680B4A93420AD07B680A4A934206D0DF
:103820007B68094A934202D06FF0020303E0786894
:1038300000F0CEFD034618460837BD4680BD00BFE8
:1038400000200440003004400040044080B582B0B5
:1038500000AF786039603968786800F0C5FD00BF56
:103860000837BD4680BD80B582B000AF7860396052
:103870003968786800F0DCFD00BF0837BD4680BDC0
:1038800080B582B000AF786039603968786800F040
:10389000F7FD00BF0837BD4680BD000080B582B08F
:1038A00000AF78607B680B4A93420AD07B680A4A73
:1038B000934206D07B68094A934202D06FF002031C
:1038C00003E0786800F004FE034618460837BD465A
:1038D00080BD00BF00200440003004400040044090
:1038E00080B582B000AF7860786800F0FDFD0346D7
:1038F00018460837BD4680BD80B582B000AF7860FD
:1039000039603968786800F04BFF00BF0837BD4662
:1039100080BD80B582B000AF786039603968786862
:1039200000F0FCFE00BF0837BD4680BD80B582B008
:1039300000AF786039603968786800F0ADFE00BF8C
:103940000837BD4680BD80B582B000AF786078682A
:1039500001F004F800BF0837BD4680BD80B582B0D5
:1039600000AF7860786800F081FF00BF0837BD467F
:1039700080BD80B582B000AF7860786800F0B2FF9B
:1039800000BF0837BD4680BD80B582B000AF78600B
:10399000786801F031F800BF0837BD4680BD80B5BA
:1039A00084B000AF7860396001217868FFF7EEFEDF
:1039B000F860FB68002B01D0FB6832E002217868D8
:1039C000FFF714FFF860FB68002B01D0FB6828E0CC
:1039D00008217868FFF77AFDF860FB68002B01D0BA
:1039E000FB681EE000217868FFF78EFDF860FB6839
:1039F000002B01D0FB6814E000217868FFF774FD0C
:103A0000F860FB68002B01D0FB680AE07B681B684C
:103A100043F001027B681A6039687868FFF73CFD63
:103A2000002318461037BD4680BD000080B586B023
:103A300000AF786039607B686B4A93420AD07B683C
:103A40006A4A934206D07B68694A934202D06FF07B
:103A50000203C4E07B681B6803F40043002B03D01F
:103A60004FF4E1037B6103E0624B1B685B087B6101
:103A70007B6907EE903AF8EEE76A3B6807EE903A0A
:103A8000B8EE677AC6EE877AC7ED027A08233B6103
:103A900016E03B6907EE903AB8EEE77AD7ED026A96
:103AA000C6EE877AB7EE007AF4EEC77AF1EE10FA36
:103AB00003D53B695B103B6105E03B695B003B6103
:103AC0003B69802BE5DD3B69802B01DD80233B6179
:103AD0003B69072B02DC6FF0020380E03B6907EED5
:103AE000903AB8EEE77AD7ED026AC6EE877AC7ED6C
:103AF000027AD7ED027AFDEEE77AF8EEE77A97EDF3
:103B0000027A77EE677A9FED3C7A67EE877AFDEE70
:103B1000E77A17EE903AFB60FB68032B03DDFB6846
:103B2000033BFB6002E0FB680333FB603B69802BD7
:103B300021D03B69802B21DC3B69402B18D03B69AD
:103B4000402B1BDC3B69202B0FD03B69202B15DC65
:103B50003B69082B03D03B69102B03D00EE00423F4
:103B60003B610EE003233B610BE002233B6108E075
:103B700001233B6105E000233B6102E06FF0070396
:103B80002DE03B691B043B617B685B6923F4403299
:103B90003B6903F440331A437B685A617B685B6975
:103BA00023F47F6323F00F03D7ED027AFDEEE77A6B
:103BB00017EE902AC2F30B021A437B685A617B68A6
:103BC0009B6923F47F6323F00F03FA68C2F30B02AF
:103BD0001A437B689A617868FFF76CFC03461846C5
:103BE0001837BD4680BD00BF0020044000300440AF
:103BF00000400440A81300200000004380B487B0B8
:103C000000AF786000237B614FF00003FB604FF052
:103C100000033B617B681B6803F40043002B03D067
:103C20004FF4E1037B6103E0384B1B685B087B6169
:103C30007B685B69C3F30B0307EE903AF8EE677A93
:103C400097ED037A77EE277AC7ED037A7B689B6955
:103C5000C3F30B0307EE903AF8EE677AC7ED047AE8
:103C6000D7ED047AB0EE087AF4EEC77AF1EE10FAE6
:103C700011DDD7ED047AB1EE087AF4EEC77AF1EEF1
:103C800010FA08D8D7ED047AB0EE087A77EEC77A42
:103C9000C7ED047A07E0D7ED047AB0EE087A77EE44
:103CA000877AC7ED047A97ED047ADFED196AC7EEDB
:103CB000267A97ED037A77EE277AC7ED037A7B6849
:103CC0005B6903F44033C3F10703012202FA03F3F3
:103CD00007EE903AF8EEE77A97ED037A67EE277AE7
:103CE000C7ED037A7B6907EE903AF8EEE76A97ED45
:103CF000037AC6EE877AFDEEE77A17EE903A184619
:103D00001C37BD465DF8047B704700BFA813002038
:103D10000000004380B483B000AF786039607B68F6
:103D2000154A93420AD07B68144A934206D07B68B6
:103D3000134A934202D06FF0020317E03B68042B52
:103D400002DD3B68082B02DD6FF002030EE03B68EA
:103D5000053B1B023B607B681B6823F440723B6899
:103D600003F440731A437B681A60002318460C372B
:103D7000BD465DF8047B70470020044000300440DD
:103D80000040044080B483B000AF78600B46FB7005
:103D90007B68164A93420AD07B68154A934206D044
:103DA0007B68144A934202D06FF0020317E0FB785D
:103DB000002B02D0012B07D00DE07B681B6823F499
:103DC00080627B681A6009E07B681B6843F480624C
:103DD0007B681A6002E06FF0020300E000231846DF
:103DE0000C37BD465DF8047B704700BF00200440DF
:103DF000003004400040044080B483B000AF7860DD
:103E00000B46FB707B68704A93420AD07B686F4A0E
:103E1000934206D07B686E4A934202D06FF0020351
:103E2000CBE0FB780C2B00F2C48001A252F823F007
:103E3000653E0010733E0010BF3E0010133F00109F
:103E4000673F0010733E0010993E0010BF3E001007
:103E5000E93E0010133F00103D3F0010673F001087
:103E60008D3F00107B681B6823F002027B681A609C
:103E7000A2E07B681B6843F002027B681A607B68E3
:103E80001B6823F00C027B681A607B681B6823F0B8
:103E900010027B681A608FE07B681B6843F00202A7
:103EA0007B681A607B681B6823F00C027B681A60D1
:103EB0007B681B6843F010027B681A607CE07B68BB
:103EC0001B6843F002027B681A607B681B6823F062
:103ED0000C0343F004027B681A607B681B6823F0C4
:103EE00010027B681A6067E07B681B6843F002027F
:103EF0007B681A607B681B6823F00C0343F00402A4
:103F00007B681A607B681B6843F010027B681A604C
:103F100052E07B681B6843F002027B681A607B6892
:103F20001B6823F00C0343F008027B681A607B686F
:103F30001B6823F010027B681A603DE07B681B68F9
:103F400043F002027B681A607B681B6823F00C0355
:103F500043F008027B681A607B681B6843F010021C
:103F60007B681A6028E07B681B6843F002027B686C
:103F70001A607B681B6843F00C027B681A607B68E0
:103F80001B6823F010027B681A6015E07B681B68D1
:103F900043F002027B681A607B681B6843F00C02E6
:103FA0007B681A607B681B6843F010027B681A60AC
:103FB00002E06FF0020300E0002318460C37BD4614
:103FC0005DF8047B704700BF0020044000300440CF
:103FD0000040044080B485B000AFF8600B467A60C2
:103FE000FB72FB682C4A93420AD0FB682B4A93422F
:103FF00006D0FB682A4A934202D06FF0020344E0E5
:10400000FB7A022B1AD0022B25DC002B02D0012BCD
:1040100007D020E0FB681B6823F40062FB681A608D
:104020001CE0FB681B6843F40062FB681A60FB68D5
:104030001B6823F48052FB681A600FE0FB681B6862
:1040400043F40062FB681A60FB681B6843F480520B
:10405000FB681A6002E06FF0020316E07B68002B39
:1040600002DD7B68202B02DD6FF002030DE07B6830
:104070001B047B60FB685B6823F47C127B6803F4A1
:104080007C131A43FB685A60002318461437BD4658
:104090005DF8047B704700BF0020044000300440FE
:1040A0000040044080B483B000AF78607B680F4A62
:1040B00093420AD07B680E4A934206D07B680D4A31
:1040C000934202D06FF002030AE07B689B6803F022
:1040D0001003002B02D06FF00C0301E07B68DB695A
:1040E00018460C37BD465DF8047B7047002004403D
:1040F000003004400040044080B483B000AF7860DA
:104100000B46FB707B68104A93420AD07B680F4ACB
:10411000934206D07B680E4A934202D06FF00203AE
:104120000CE07B689B6803F08003002B02D06FF0EB
:104130000B0303E0FA787B68DA61002318460C373A
:10414000BD465DF8047B7047002004400030044009
:104150000040044080B586B000AFF860B9607A6076
:1041600000237B6114E0F868FFF728FA38613B69A7
:10417000002B04DA7B687A691A603B6911E07B697D
:10418000BA6813443A69D2B21A707B6901337B6111
:104190007B681B687A699A42E5DB7B687A691A60FA
:1041A000002318461837BD4680BD80B586B000AFE5
:1041B000F860B9607A6000237B6113E07B69BA68BC
:1041C00013441B781946F868FFF71AFA38613B69FF
:1041D000002B04D07B687A691A603B690BE07B692D
:1041E00001337B617B681B687A699A42E6DB7B68F6
:1041F0007A691A60002318461837BD4680BD80B41E
:1042000087B000AFF860B9607A6000237B610FE08F
:10421000FB689B6803F01003002B0ED1FB68D96983
:10422000BA687B691344CAB21A707B6901337B6137
:104230007A697B689A42EBD300E000BF7B6918463D
:104240001C37BD465DF8047B704780B483B000AF77
:1042500078607B689B681B0A03F03F0318460C37A5
:10426000BD465DF8047B704780B487B000AFF8604E
:10427000B9607A6000237B610FE0FB689B6803F004
:104280008003002B0ED1BA687B6913441B781A4651
:10429000FB68DA617B6901337B617A697B689A42EA
:1042A000EBD300E000BF7B6918461C37BD465DF8C4
:1042B000047B704780B485B000AF78607B689B68F2
:1042C0001B0C03F03F03FB60FB68C3F1200318469F
:1042D0001437BD465DF8047B7047000080B483B09E
:1042E00000AF786039607B68134A93420AD07B68DC
:1042F000124A934206D07B68114A934202D06FF073
:10430000020313E03B68002B02D03B68202B02D94C
:104310006FF002030AE07B685B6823F03F023B68B2
:1043200003F03F031A437B685A60002318460C379A
:10433000BD465DF8047B7047002004400030044017
:104340000040044080B483B000AF78607B685B6855
:1043500003F03F0318460C37BD465DF8047B7047F9
:1043600080B483B000AF786039607B68154A9342AF
:104370000AD07B68144A934206D07B68134A934262
:1043800002D06FF0020316E03B68002B02D03B68BE
:10439000202B02D96FF002030DE03B681B023B604B
:1043A0007B685B6823F47C523B6803F47C531A43BC
:1043B0007B685A60002318460C37BD465DF8047BC5
:1043C000704700BF0020044000300440004004401B
:1043D00080B483B000AF78607B681B6918460C37E7
:1043E000BD465DF8047B704780B483B000AF786051
:1043F00039607B680B4A93420AD07B680A4A934231
:1044000006D07B68094A934202D06FF0020303E0B2
:104410007B683A681A61002318460C37BD465DF880
:10442000047B7047002004400030044000400440FA
:1044300080B483B000AF786039607B680D4A9342E6
:104440000AD07B680C4A934206D07B680B4A9342A1
:1044500002D06FF0020306E07B68DA683B681A431B
:104460007B68DA60002318460C37BD465DF8047B94
:10447000704700BF0020044000300440004004406A
:1044800080B483B000AF786039607B680D4A934296
:104490000AD07B680C4A934206D07B680B4A934251
:1044A00002D06FF0020307E07B68DA683B68DB4309
:1044B0001A407B68DA60002318460C37BD465DF869
:1044C000047B70470020044000300440004004405A
:1044D00080B483B000AF78607B689B6818460C3767
:1044E000BD465DF8047B704780B584B000AF78604E
:1044F0007B681B68634A93420CD07B681B68624AE6
:10450000934207D07B681B68604A934202D06FF0E9
:104510000203B3E07B68DB68002B4BD07B685B68F1
:10452000002B02D16FF00203A8E07B6800225A61E1
:104530007B681B68534A934210D07B681B68524AC1
:10454000934209D07B681B68504A934201D10223F1
:1045500005E04FF0FF3302E0012300E000234C4967
:104560007A6841F823207B681B6840211846FFF7D2
:104570007AF97B681B681846FFF7E6F8F8607B68F5
:10458000DA687B685B69D31AFA68934228BF1346DE
:10459000FB607B6818687B685A687B685B691344BA
:1045A000FA681946FFF7C0F802467B685B691A444F
:1045B0007B685A617B681B69002B5ED07B689B68B7
:1045C000002B09D17B681B684FF0FF311846FFF7BD
:1045D00057F96FF0020351E07B6800229A617B6813
:1045E0001B68284A934210D07B681B68264A934276
:1045F00009D07B681B68254A934201D1022305E05C
:104600004FF0FF3302E0012300E0002321497A68E4
:1046100041F823207B681B680B211846FFF723F91C
:104620007B681B6810211846FFF71DF97B681B6823
:104630001846FFF757F8B8607B681A697B689B6972
:10464000D31ABA68934228BF1346BB607B681868C8
:104650007B689A687B689B691344BA681946FFF7C0
:1046600031F802467B689B691A447B689A617B68D3
:104670001B6810211846FFF7E9F800231846103789
:10468000BD4680BD0020044000300440004004408E
:10469000901900209C19002080B584B000AF78608C
:1046A00039607B68194A93420AD07B68184A934262
:1046B00006D07B68174A934202D06FF0020321E0D4
:1046C0007B68124A93420ED07B68114A934208D00D
:1046D0007B68104A934201D1022305E04FF0FF337B
:1046E00002E0012300E000230B4A52F82330FB6074
:1046F000FB68DB69002B04D0FB68DB693968F8686C
:104700009847002318461037BD4680BD002004405E
:1047100000300440004004409C19002080B584B063
:1047200000AF786039607B68194A93420AD07B6891
:10473000184A934206D07B68174A934202D06FF022
:10474000020321E07B68124A93420ED07B68114A33
:10475000934208D07B68104A934201D1022305E0BE
:104760004FF0FF3302E0012300E000230B4A52F830
:104770002330FB60FB68DB69002B04D0FB68DB693E
:104780003968F8689847002318461037BD4680BD41
:1047900000200440003004400040044090190020F4
:1047A00080B586B000AF786039607B682A4A934252
:1047B0000ED07B68294A934208D07B68284A9342EE
:1047C00001D1022305E04FF0FF3302E0012300E0B6
:1047D0000023244A52F823207B681F498B420ED0C5
:1047E0007B681E498B4208D07B681D498B4201D1F2
:1047F000022305E04FF0FF3302E0012300E0002335
:10480000194951F823309A4202D10123FB7401E087
:104810000023FB7439687868FFF780FFF860FB7C41
:1048200083F00103DBB2002B05D039687868FFF70D
:1048300033FF786101E000237B61FB68002B01D02E
:10484000FB6805E07B69002B01D07B6900E0002359
:1048500018461837BD4680BD002004400030044093
:1048600000400440901900209C19002080B582B0BF
:1048700000AF78607B68174A93420AD07B68164A7B
:10488000934206D07B68154A934202D06FF0020330
:104890001CE040217868FEF7F3FF7B680D4A9342E5
:1048A0000ED07B680C4A934208D07B680B4A934237
:1048B00001D1022305E04FF0FF3302E0012300E0C5
:1048C0000023074A002142F8231000231846083726
:1048D000BD4680BD0020044000300440004004403C
:1048E0009019002080B582B000AF78607B68174ACD
:1048F00093420AD07B68164A934206D07B68154AD9
:10490000934202D06FF002031CE01B217868FEF78F
:10491000B7FF7B680D4A93420ED07B680C4A9342E6
:1049200008D07B680B4A934201D1022305E04FF087
:10493000FF3302E0012300E00023074A002142F890
:104940002310002318460837BD4680BD00200440D0
:1049500000300440004004409C19002080B584B021
:1049600000AF78607B681F4A93420AD07B681E4A7A
:10497000934206D07B681D4A934202D06FF0020337
:104980002BE07B68174A93420ED07B68164A93420D
:1049900008D07B68154A934201D1022305E04FF00D
:1049A000FF3302E0012300E00023FB60104AFB68B4
:1049B00052F82330BB60BB68002B02D07868FEF74A
:1049C000CDFF0C4AFB6852F82330BB60BB68002B5C
:1049D00002D07868FEF7CDFF002318461037BD4699
:1049E00080BD00BF0020044000300440004004406F
:1049F000901900209C19002090B589B000AF786014
:104A00007B68704A93420ED07B686F4A934208D00D
:104A10007B686E4A934201D1022305E04FF0FF33D9
:104A200002E0012300E00023FB617B68654A9342BA
:104A30000AD07B68644A934206D07B68634A9342FB
:104A400002D06FF00203B8E07868FEF7DDFEB861CF
:104A50007B68DA68BB69134003F00B03002B0AD0B4
:104A60006FF008017868FEF747FF7868FEF76BFF84
:104A70006FF00303A1E0564AFB6952F823307B61D3
:104A8000BB6903F04003002B2DD07B69002B2AD09B
:104A90007B69DB68002B26D07B691B681846FEF714
:104AA00053FE38617B69DA687B695B69D31A3A69BE
:104AB000934228BF13463B617B6918687B695A683B
:104AC0007B695B6913443A691946FEF72DFE02467D
:104AD0007B695B691A447B695A617B691B68402169
:104AE0001846FEF7B3FE7B695A697B69DB689A4218
:104AF00006D100217868FEF70CFF7868FEF72EFFDC
:104B0000344AFB6952F823307B61BB6903F0100320
:104B1000002B44D07B69002B41D07B691B69002BA3
:104B20003DD07B691B681846FEF7DCFDF8607B69A9
:104B30001A697B699B69D31AFA68934228BF1346A6
:104B4000FB607B6918687B699A687B699B69134481
:104B5000FA681946FEF7B6FD02467B699B691A445E
:104B60007B699A617B691A697B699B69D41A7B6945
:104B70001B681846FEF718FE03469C4209D27B6963
:104B800018687B691A697B699B69D31A1946FEF715
:104B9000FDFD7B691B6810211846FEF757FE7B69F7
:104BA0009A697B691B699A4206D100217868FEF7F1
:104BB000BDFE7868FEF7DDFE002318462437BD46AB
:104BC00090BD00BF0020044000300440004004407D
:104BD000901900209C19002080B584B000AF786047
:104BE0003960012108200AF0E9FCF860FB68002B1D
:104BF00002D16FF00B0312E0FB683A6811461846C9
:104C000000F0A8FBB860BB68002B04D0F8680AF07D
:104C1000E3FCBB6803E07B68FA681A60BB6818466F
:104C20001037BD4680BD80B584B000AF78600B46BC
:104C3000FB701346BB7097F90230002B0DDABB787E
:104C40003B73FB787B737B68186807F10C010123C9
:104C5000022200F059FC034637E0FB78042B02D017
:104C6000FB78082B0BD17B6801221A717B681868CE
:104C7000F91C0123012200F047FC034625E0FB78E4
:104C8000012B02D0FB78022B0BD17B6800221A711A
:104C90007B681868F91C0123012200F035FC0346EB
:104CA00013E0FB78052B02D0FB780A2B0BD17B6835
:104CB00002221A717B681868F91C0123012200F096
:104CC00023FC034601E06FF0150318461037BD467C
:104CD00080BD80B586B000AFF860B9607A6096207C
:104CE00002F07EFBFB681B79022B4BD0022B7DDC94
:104CF000002B24D0012B79D17B68002B02D16FF0DF
:104D0000150375E0FB68186807F110010123022202
:104D100000F031FC78617B69002B01D07B6967E092
:104D20003B7C1BB21B011AB27B7C1B09DBB21BB2A2
:104D300013431BB29AB27B681A80002358E0BB6809
:104D4000002B02D16FF0150352E0FB68186807F1E1
:104D500010010123022200F00EFC78617B69002B18
:104D600001D07B6944E03B7C1BB21B011AB27B7C07
:104D70001B09DBB21BB213431BB29AB2BB681A8089
:104D8000002335E0BB68002B02D07B68002B02D1EA
:104D90006FF015032CE0FB68186807F11001012380
:104DA000032200F0E8FB78617B69002B01D07B696E
:104DB0001EE03B7C1BB21B011AB2BB7C1B09DBB2A1
:104DC0001BB213431BB29AB2BB681A807B7C1BB226
:104DD0001B011AB2BB7C1BB203F00F031BB21343BF
:104DE0001BB29AB27B681A80002301E06FF01503B2
:104DF00018461837BD4680BD80B58CB002AFF8604C
:104E0000B9607A603B60FB687B627B6A1B683B62CF
:104E10003B68DB78002B02D0012B11D021E007F199
:104E2000140207F116031946386AFFF752FFF861BA
:104E3000FB69002B01D0FB6920E0FB8ABB6113E01A
:104E400007F1140207F116031946386AFFF741FF0C
:104E5000F861FB69002B01D0FB690FE0BB8ABB61E5
:104E600002E06FF0150309E007F118030093012336
:104E700001227968B86807F0ADF80346184628376C
:104E8000BD4680BD80B58AB002AFF860B9607A6077
:104E90003B60FB68002B02D16FF015033DE0FB681F
:104EA000FB61FB691B68002B02D16FF0150334E036
:104EB000FB691B68BB613B68DB78002B02D0012BD0
:104EC00019D028E0BB695B79002B03D146F2EE6371
:104ED0003B6102E041F6FA133B61124B5B787B6168
:104EE00007F11003009302230B227968B86807F0DA
:104EF00071F8034611E00C4B3B614FF4C8337B6102
:104F000007F11003009302230A227968B86807F0BA
:104F100061F8034601E06FF0150318462037BD46DF
:104F200080BD00BF04000020709D010080B584B0EA
:104F300000AF786039607B68002B02D16FF01503F9
:104F40000EE07B68FB60FB683A689A603B68DBB206
:104F500018460BF0A6FD0346DAB2FB681A7300236D
:104F600018461037BD4680BD80B58CB000AFF860E4
:104F7000B9607A600023FB62FB68002B02D16FF0FE
:104F8000150346E0FB68BB62BB6A1B68002B02D1BD
:104F90006FF015033DE0BB6A1B687B622FE007F1F1
:104FA000140207F116031946786AFFF792FE386279
:104FB0003B6A002B01D03B6A2BE0FB8AFB61BB8A7A
:104FC000BB61BB6A9B6803F00103002B08D0FB6A3E
:104FD0009B00BA681344FA691A60FB6A0133FB62EA
:104FE000BB6A9B6803F00203002B08D0FB6A9B009E
:104FF000BA681344BA691A60FB6A0133FB62BB6A80
:105000001B7B1A467B6802FB03F3FA6A9A42C6D3FB
:105010007B6818463037BD4680BD000080B584B03F
:1050200000AF78603960102101200AF0C7FAB8603B
:10503000BB68002B02D16FF00B0324E0BB68144A5D
:105040005A60BA683B681B6819461046FFF7C4FDF2
:10505000F860FB68002B0FD1BB681B68002205219C
:105060001846FFF7E0FDF860FB68002B06D17B686F
:10507000BA681A60002306E000BF00E000BFB8680D
:105080000AF0AAFAFB6818461037BD4680BD00BF7B
:105090009000002080B584B000AF786039603B6834
:1050A000002B03D03B685B68002B02D16FF0150327
:1050B00019E03B685B681B68002B02D16FF0570357
:1050C00011E03B685B681B68396878689847F8604E
:1050D000FB68002B01D0FB6805E07B681B683A6821
:1050E00052685A60002318461037BD4680BD90B5FF
:1050F00085B000AFF860B9607A607B80FB68002BF8
:1051000006D0FB685B68002B02D07B68002B02D1C5
:105110006FF0150310E0FB685B685B68002B02D141
:105120006FF0570308E0FB685B685C687B887A680F
:10513000B968F868A047034618461437BD4690BDC5
:1051400090B585B000AFF860B9607A607B80FB688D
:10515000002B06D0FB685B68002B02D07B68002B1D
:1051600002D16FF0150310E0FB685B689B68002BB1
:1051700002D16FF0570308E0FB685B689C687B888E
:105180007A68B968F868A047034618461437BD46E0
:1051900090BD80B584B000AF786039603B68002B6B
:1051A00003D03B68DB68002B02D16FF0150319E0D8
:1051B0003B68DB681B68002B02D16FF0570311E0DE
:1051C0003B68DB681B68396878689847F860FB685B
:1051D000002B01D0FB6805E07B681B683A68D26849
:1051E000DA60002318461037BD4680BD80B582B016
:1051F00000AF78607B68002B15D07B68DB68002BE4
:1052000002D16FF015030FE07B68DB689B68002B11
:1052100002D16FF0570307E07B68DB689B68786812
:105220009847034600E0002318460837BD4680BD76
:1052300080B582B000AF78607B68002B15D07B68AA
:10524000DB68002B02D16FF015030FE07B68DB6891
:10525000DB68002B02D16FF0570307E07B68DB6847
:10526000DB6878689847034600E000231846083753
:10527000BD4680BD80B582B000AF78600B46FB7044
:105280007B68002B17D07B68DB68002B02D16FF0A6
:10529000150311E07B68DB681B69002B02D16FF0FE
:1052A000570309E07B68DB681B69FA781146786868
:1052B0009847034600E0002318460837BD4680BDE6
:1052C00080B582B000AF78600B46FB707B68002B26
:1052D00017D07B68DB68002B02D16FF0150311E05B
:1052E0007B68DB689B69002B02D16FF0570309E0F4
:1052F0007B68DB689B69FA781146786898470346B3
:1053000000E0002318460837BD4680BD80B582B056
:1053100000AF786039607B68002B16D07B68DB6853
:10532000002B02D16FF0150310E07B68DB689B69EE
:10533000002B02D16FF0570308E07B68DB68DB6964
:10534000396878689847034600E000231846083714
:10535000BD4680BD80B584B000AF786039603B68E1
:10536000002B03D03B68DB68002B02D16FF01503E4
:105370003FE03B68DB681B68002B02D16FF05703EE
:1053800037E03B681B68042B02D96FF0150330E04F
:105390003B681B68194A52F82330002B08D1386843
:1053A00000F02EF8F860FB68002B01D0FB6820E0CD
:1053B0003B68DB681B68396878689847F860FB6869
:1053C000002B01D0FB6814E03B681A687B681B68FF
:1053D0000A4951F822201A607B681B681B681A79F9
:1053E0000132D2B21A717B681B683A68D2681A61BE
:1053F000002318461037BD4680BD00BFA819002005
:1054000080B584B000AF7860182101200AF0D6F88A
:10541000F860FB68002B02D16FF00B031DE0FB6806
:1054200018460BF0A7F8FB6800221A717B681A680F
:10543000FB689A607B685A68FB68DA607B68DA68A8
:10544000FB681A617B681A69FB685A617B681B6894
:105450000449FA6841F82320002318461037BD4656
:1054600080BD00BFA819002080B582B000AF786071
:105470007B681B689B68184600F01CF87B68002B53
:1054800003D07B681B69002B02D16FF015030DE080
:105490007B681B69DB68002B02D16FF0570305E0C6
:1054A0007B681B69DB6878689847034618460837AD
:1054B000BD4680BD80B584B000AF7860114A7B687E
:1054C00052F82330FB60FB681B79002B05D0FB688A
:1054D0001B79013BDAB2FB681A71FB681B79002B60
:1054E0000CD1FB681B6818460BF062F8FB68002BB8
:1054F00004D0F8680AF070F80023FB6000BF103792
:10550000BD4680BDA819002090B587B000AFF860F7
:10551000B96011461A460B46FB711346BB71FB6816
:10552000002B03D0FB681B69002B02D16FF0150321
:105530001DE0FB681B695B68002B02D16FF057030D
:1055400015E0FB681B681B6818460BF01DF8FB682C
:105550001B695C68BB79FA79B968F868A04778611B
:10556000FB681B681B6818460BF018F87B69184627
:105570001C37BD4690BD90B587B000AFF860B960EC
:1055800011461A460B46FB711346BB71FB68002B94
:1055900003D0FB681B69002B02D16FF015031DE0DF
:1055A000FB681B699B68002B02D16FF0570315E065
:1055B000FB681B681B6818460AF0E6FFFB681B695E
:1055C0009C68BB79FA79B968F868A0477861FB688C
:1055D0001B681B6818460AF0E1FF7B6918461C37F8
:1055E000BD4690BD80B584B000AF786039603B683F
:1055F000002B03D03B685B68002B02D16FF01503D2
:1056000019E03B685B681B68002B02D16FF0570301
:1056100011E03B685B681B68396878689847F860F8
:10562000FB68002B01D0FB6805E07B681B683A68CB
:1056300052685A60002318461037BD4680BD80B5B9
:1056400082B000AF78607B68002B03D07B685B681A
:10565000002B02D16FF015030DE07B685B685B6A7D
:10566000002B02D16FF0570305E07B685B685B6A33
:1056700078689847034618460837BD4680BD80B510
:1056800084B000AFF860B9607A60FB68002B03D08B
:10569000FB685B68002B02D16FF015030FE0FB681D
:1056A0005B685B68002B02D16FF0570307E0FB6873
:1056B0005B685B687A68B968F8689847034618467B
:1056C0001037BD4680BD80B584B000AFF860B960CA
:1056D0007A60FB68002B03D0FB685B68002B02D16B
:1056E0006FF015030FE0FB685B689B68002B02D12D
:1056F0006FF0570307E0FB685B689B687A68B968DE
:10570000F8689847034618461037BD4680BD80B5F7
:1057100084B000AFF860B9601346FB71FB68002BE2
:1057200003D0FB685B68002B02D16FF015030FE01C
:10573000FB685B685B69002B02D16FF0570307E0E1
:10574000FB685B685B69FA79B968F8689847034653
:1057500018461037BD4680BD80B582B000AF786076
:1057600039607B68002B03D07B685B68002B02D11B
:105770006FF015030EE07B685B689B69002B02D11C
:105780006FF0570306E07B685B689B69396878684F
:105790009847034618460837BD4680BD80B582B09D
:1057A00000AF786039607B68002B03D07B685B6852
:1057B000002B02D16FF015030EE07B685B68DB699C
:1057C000002B02D16FF0570306E07B685B68DB6952
:1057D000396878689847034618460837BD4680BD43
:1057E00080B584B000AFF860B9607A60FB68002BC8
:1057F00003D0FB685B68002B02D16FF015030FE04C
:10580000FB685B681B6A002B02D16FF0570307E04F
:10581000FB685B681B6A7A68B968F8689847034652
:1058200018461037BD4680BD80B584B000AF7860A3
:1058300039603B68002B03D03B689B68002B02D18A
:105840006FF0150328E03B689B681B68002B02D1B2
:105850006FF0570320E03B689B681B6839687868E5
:105860009847F860FB68002B01D0FB6814E07B6868
:105870001B683A6812681A607B681B683A6812797C
:105880001A717B681B683A6852795A717B681B6889
:105890003A6892689A60002318461037BD4680BD6A
:1058A00080B582B000AF78607B68002B03D07B6846
:1058B0009B68002B02D16FF015030DE07B689B689D
:1058C000DB68002B02D16FF0570305E07B689B6813
:1058D000DB6878689847034618460837BD4680BDA0
:1058E00080B584B000AFF860B9601346FB80FB68F8
:1058F000002B03D0FB689B68002B02D16FF01503CF
:105900000FE0FB689B685B68002B02D16FF05703C8
:1059100007E0FB689B685B68FA88B968F868984795
:10592000034618461037BD4680BD80B584B000AF31
:10593000F860B9607A60FB68002B03D0FB689B6855
:10594000002B02D16FF015030FE0FB689B689B688A
:10595000002B02D16FF0570307E0FB689B689B6840
:105960007A68B968F8689847034618461037BD4604
:1059700080BD000080B584B000AF786039603B68BE
:10598000002B07D03B685B69002B03D03B681B787A
:105990000A2B02D96FF015032AE03B685B691B688C
:1059A000002B02D16FF0570322E03B685B691B6854
:1059B000396878689847F860FB68002B01D0FB686D
:1059C00016E07B681B683A6852695A613B681B782D
:1059D0009B00094A134418460AF0CCFD3B681B782B
:1059E00019467B681B68044A52F821201A6000237C
:1059F00018461037BD4680BDBC19002080B582B066
:105A000000AF78607B68002B03D07B685B69002B5C
:105A100002D16FF0150319E07B685B695B69002BAD
:105A200002D16FF0570311E07B681B6818460AF03B
:105A3000BFFD7B681B791946064B002243F82120E5
:105A40007B685B695B697868984703461846083746
:105A5000BD4680BDBC19002080B586B000AFF8609F
:105A6000B9607A60FB68002B06D0FB685B69002B8D
:105A700002D0BB68002B02D16FF015031AE0FB685F
:105A80005B695B68002B02D16FF0570312E0FB6883
:105A90001B6818460AF078FDFB685B695B687A68EA
:105AA000B968F86898477861FB681B6818460AF07F
:105AB00075FD7B6918461837BD4680BD80B586B038
:105AC00000AFF860B9607A60FB68002B06D0FB6815
:105AD0005B69002B02D0BB68002B02D16FF015036D
:105AE0001AE0FB685B699B68002B02D16FF05703DB
:105AF00012E0FB681B6818460AF046FDFB685B690C
:105B00009B687A68B968F86898477861FB681B6891
:105B100018460AF043FD7B6918461837BD4680BD1C
:105B200080B586B000AF786039607B68002B02D00A
:105B30003B68002B02D16FF0150338E00C210120E7
:105B400009F03CFD38613B69002B02D16FF00B037B
:105B50002DE03B681A683B691A600421012009F0B6
:105B60002DFDF860FB68002B03D16FF00B037B6108
:105B700019E03B689B68BB60FA68BB681B68194604
:105B80001046FFF7E7FB78617B69002B07D13B6983
:105B9000FA689A607B683A691A60002307E000BFE0
:105BA000F86809F019FD386909F016FD7B69184697
:105BB0001837BD4680BD80B58AB000AFF860B960C7
:105BC0007A607B80BB683B62FB68002B06D0FB6879
:105BD0009B68002B02D07B68002B02D16FF015036D
:105BE00035E0FB689B68FB610023FB842AE03B6A8D
:105BF0009BB207F11402114618460AF0A9FFFB698F
:105C0000186807F1140101230222FFF77DFCB86137
:105C1000BB69002B01D0BB6919E0FB691868FB8CDC
:105C20007A68D11801230122FFF7A5FCB861BB698E
:105C3000002B01D0BB690AE03B6A01333B62FB8C5D
:105C40000133FB84FA8C7B889A42D0D30023184618
:105C50002837BD4680BD80B592B000AFF860B9600E
:105C60007A607B807B885B099BB2DBB27A8802F02A
:105C70001F0292B2002A14BF01220022D2B21344A2
:105C800087F83F30BB683B64FB68002B06D0FB689D
:105C90009B68002B02D07B68002B02D16FF01503AC
:105CA00075E0FB689B68BB63BB6803F01F03002BB8
:105CB0003CD1002387F8453031E097F845309BB25E
:105CC0005B019AB2BB689BB213449BB207F110020E
:105CD000114618460AF03CFF97F845305B011A461A
:105CE0007B68991807F110030233202218460FF041
:105CF00025FCBB6B186807F1100101232222FFF776
:105D000003FC78637B6B002B01D07B6B3FE00520AD
:105D100001F071FB97F84530013387F8453097F86B
:105D2000452097F83F309A42C7D32FE00023A7F8C9
:105D3000463026E03B6C9BB207F110021146184634
:105D40000AF006FFB7F846307A6813441B78BB7434
:105D5000BB6B186807F1100101230322FFF7D4FB86
:105D600078637B6B002B01D07B6B10E0052001F08A
:105D700042FB3B6C01333B64B7F846300133A7F874
:105D80004630B7F846207B889A42D3D30023184682
:105D90004837BD4680BD80B584B000AF78607B6871
:105DA000002B03D07B689B68002B02D16FF015039A
:105DB00016E07B689B68FB60FB681B681846FFF772
:105DC00053FBB860BB68002B01D0BB6808E07B6860
:105DD0009B68184609F000FC786809F0FDFB002379
:105DE00018461037BD4680BD80B586B000AF7860DC
:105DF00039607B68002B02D03B68002B02D16FF02A
:105E00001503A9E00821012009F0D8FB38613B699E
:105E1000002B02D16FF00B039EE03B691A1D3B681B
:105E2000043319461046FFF7FFFC78617B69002BAD
:105E300040F084803B681B68002B0FD03A693B68B8
:105E40001B6819461046FFF7A4F978617B69002B9F
:105E50007DD1386900F0AEF8786103E0386900F070
:105E60007FF878617B69002B6AD107F10E031A462F
:105E70000221386900F0D8F87861FB8940F283226A
:105E8000934203D06FF00D037B6151E007F10E03E5
:105E90001A460321386900F0C7F87861FB894BF690
:105EA0003042934203D06FF00D037B6140E03B68CA
:105EB0005969386900F002F978617B69002B2ED1AD
:105EC0003B68197E3B685B7E1A46386900F06AF9C8
:105ED00078617B69002B24D13B689B7E1946386929
:105EE00000F0B0F978617B69002B1CD13B68DB7E48
:105EF0001946386900F0CEF978617B69002B14D11E
:105F00003B681B7F1946386900F07FFA78617B692E
:105F1000002B0CD17B683A691A6000231CE000BF9B
:105F200006E000BF04E000BF02E000BF00E000BFE9
:105F30003B695B681846FFF7B3FC02E000BF00E076
:105F400000BF3B691B681846FFF750F900E000BF2F
:105F500038690DF045FE7B6918461837BD4680BD8F
:105F600080B584B000AF78604FF0FF33FB60FB6812
:105F7000DB06FB60FB68DB0AFB60FB681E21184642
:105F80000AF06AFD02460A4B13430122194678685B
:105F900000F037F8B860BB68002B01DABB6803E09B
:105FA000142001F028FA002318461037BD4680BDA2
:105FB0000CFF008080B584B000AF78607B681B6800
:105FC00000211846FFF756F9F860FB68002B01D056
:105FD000FB6812E0012001F00EFA7B681B680121CA
:105FE0001846FFF747F9F860FB68002B01D0FB6803
:105FF00003E0142001F0FFF9002318461037BD46D6
:1060000080BD80B584B000AFF860B9601346FB80F6
:10601000FB685B68FA88B9681846FFF761FC0346BD
:1060200018461037BD4680BD80B584B000AFF8601B
:10603000B9607A60FB685B687A68B9681846FFF7F0
:1060400074FC034618461037BD4680BD80B586B047
:1060500000AFF860B96011461A460B46FB80134644
:10606000BB80FB685B6807F11202B9681846FFF74E
:106070005CFC78617B69002B01D07B6919E0B7F982
:106080000430DB431AB27B8A1BB213401BB29BB2B3
:106090007B82FA88BB8813409AB27B8A13439BB2F7
:1060A0007B82FB685B687A8AB9681846FFF718FC40
:1060B000034618461837BD4680BD000090B587B02E
:1060C00000AF78603960012101200AF0C5FC034669
:1060D0009CB201214FF400700AF0BEFC03469BB253
:1060E00023439CB201214FF480600AF0B5FC0346C3
:1060F0009BB22343FB823B78002B19D00121022065
:106100000AF0AAFC04464FF0FF333B613B695B0792
:106110003B613B699B0E3B613B697A7811461846AF
:106120000AF09AFC034623439AB2FB8A1343FB828C
:10613000BB78002B19D0012104200AF08DFC044605
:106140004FF0FF33FB60FB685B07FB60FB68DB0D18
:10615000FB60FB68FA78114618460AF07DFC03469E
:1061600023439AB2FB8A1343FB824FF0FF33BB6099
:10617000BB68DB06BB60BB68DB0ABB60BB681E217B
:1061800018460AF069FC0246054B1343FA8A194681
:106190007868FFF736FF034618461C37BD4690BDAA
:1061A00023FF008080B586B000AF78600B46FB709F
:1061B0001346BB703723FB824FF0FF333B613B69D3
:1061C000DB063B613B69DB0A3B613B691E211846EC
:1061D0000AF042FC03461A491943FB8A00227868F8
:1061E000FFF734FFF860FB68002B01D0FB6823E069
:1061F000FB78002B1FD04FF0FF33BB60BB68DB0682
:10620000BB60BB68DB0ABB60BB681E2118460AF096
:1062100023FC03460A491943BB78012202FA03F31F
:106220009AB2BB78012000FA03F39BB27868FFF7BB
:106230000DFF034600E0002318461837BD4680BD19
:106240001FFF008080B584B000AF78600B46FB7004
:106250004FF0FF33FB60FB68DB06FB60FB68DB0A8B
:10626000FB60FB681E2118460AF0F6FB034608494E
:106270001943FB78002B01D0082200E000220823FC
:106280007868FFF7E3FE034618461037BD4680BD29
:106290001FFF008080B588B000AF78600B46FB70B0
:1062A0004FF0FF33BB61BB69DB06BB61BB69DB0E33
:1062B000BB61BB699BB243F4F073FB824FF0FF33C9
:1062C0003B613B69DB063B613B69DB0E3B613B6944
:1062D000012118460AF0C0FB0346FB830121202060
:1062E0000AF0BAFB03469AB2FB8B1343FB83FB789D
:1062F000002B08D0012140200AF0AEFB03469AB2E1
:10630000FB8B1343FB83FB78012B08D901218020F1
:106310000AF0A2FB03469AB2FB8B1343FB83FB7884
:10632000022B09D901214FF480700AF095FB034636
:106330009AB2FB8B1343FB83FB8AFA8B04217868A8
:10634000FFF784FEF860FB68002B01D0FB6858E083
:106350004FF44073FB8200214FF480700AF07CFB05
:106360000346FB83FB78042B09D901214FF400700D
:106370000AF072FB03469AB2FB8B1343FB83FB8A42
:10638000FA8B09217868FFF761FEF860FB68002B43
:1063900001D0FB6835E04FF40553FB82FB7803F036
:1063A0000103002B09D001214FF480700AF054FB47
:1063B00003469AB2FB8B1343FB83FB7803F0020383
:1063C000002B09D001214FF400500AF045FB034691
:1063D0009AB2FB8B1343FB83FB7803F00403002B7F
:1063E00008D0012140200AF037FB03469AB2FB8B0C
:1063F0001343FB83FB8AFA8B00217868FFF726FEA4
:10640000034618462037BD4680BD80B584B000AF36
:1064100078600B46FB704FF49053FB81FB78002BA8
:1064200001D0FA8900E00022FB8900217868FFF79B
:106430000DFE034618461037BD4680BD80B584B0BA
:1064400000AF786007F10A031A461A217868FFF74F
:10645000EBFDF860FB68002B09D17B8919464020D1
:106460000AF00CFB0346002B01D0012300E00023BF
:1064700018461037BD4680BD80B584B000AF786047
:1064800007F10A031A461A217868FFF7CDFD4FF08D
:10649000FF33FB60FB685B07FB60FB689B0DFB60E9
:1064A000FB687A89114618460AF0E8FA0346DBB21F
:1064B00018461037BD4680BD80B586B000AFF86085
:1064C000B9607A60BB681F2B02D96FF0150312E028
:1064D000FB681B6807F11202B9681846FFF7A4FDB4
:1064E00078617B69002B01D07B6904E07B8A1A46C6
:1064F0007B681A60002318461837BD4680BD80B5FA
:1065000084B000AFF860B9607A60BB681F2B02D915
:106510006FF0150308E0FB681B687A6892B2B968EF
:106520001846FFF76EFD034618461037BD4680BD7E
:1065300080B58CB002AFF860B9607A603B60FB68F0
:106540007B627B6A1B683B623B6B022B19D03B6B07
:10655000022B2CDC3B6B002B03D03B6B012B08D0B8
:1065600025E0386AFFF76AFF0346BB76BB7E7B6196
:1065700020E0386AFFF780FF0346FB76FB7E7B61F5
:1065800018E007F112031A460021386AFFF74CFDA4
:10659000F861FB69002B01D0FB6915E07B8A194685
:1065A0004FF480500AF06AFA03467B6102E06FF014
:1065B000150309E007F11403009301230122796810
:1065C000B86805F007FD034618462837BD4680BD6C
:1065D00080B588B000AFF860B9607A603B60002396
:1065E000FB61FB68BB61BB691B687B6107F1100243
:1065F00000230121B86805F03DFCF861FB69002B20
:1066000001DAFB694AE0BB6A022B31D0BB6A022B7C
:106610003ADCBB6A002B03D0BB6A012B1AD033E0F3
:106620004FF40053002217217869FFF70FFDF8613E
:10663000FB69002B01D0FB6930E03B69002B26D0C1
:106640004FF400534FF4005217217869FFF7FEFC16
:10665000F8611CE03B69052B02DD6FF015031DE0BE
:106660003B69DBB219467869FFF714FEF8610FE069
:106670003B69002B14BF01230023DBB21946786964
:10668000FFF7C3FEF86103E06FF0150306E000BFFB
:10669000FB69002B01D0FB6900E07B6818462037BE
:1066A000BD4680BDB0B586B000AF786039600821C6
:1066B000012008F083FF78617B69002B02D16FF025
:1066C0000B0329E03821012008F078FF38613B698D
:1066D000002B08D16FF00B03FB6000BF786908F056
:1066E0007BFFFB6818E03B690D4A1C4615460FCD41
:1066F0000FC40FCD0FC40FCD0FC495E8030084E87D
:1067000003007B693A695A603B681A687B691A60C2
:106710007B687A691A60002318461837BD46B0BDF9
:106720001801002080B586B000AFF860B9607A60CB
:10673000FB681B68BA68D1B207F11202184600F074
:1067400041FA78617B69002B01D07B6904E07B8A88
:106750001A467B681A60002318461837BD4680BD6C
:1067600080B584B000AFF860B9607A60FB681B68E0
:10677000BA68D1B27A6892B2184600F0EEF90346D0
:1067800018461037BD4680BD80B58CB002AFF860AA
:10679000B9607A603B60FB687B627B6A1B683B6226
:1067A0003B6B022B10D03B6B022B2DDC3B6B002B89
:1067B0001AD03B6B012B27D1386A00F0BFFB034690
:1067C000FB76FB7E7B6122E007F113031A46002172
:1067D000386A00F03EFBF861FB69002B01D0FB69D1
:1067E0001FE0FB7C7B6112E007F113031A460021D6
:1067F000386A00F09CFAF861FB69002B01D0FB6954
:106800000FE0FB7C7B6102E06FF0150309E007F10C
:1068100014030093012301227968B86805F0DAFBBC
:10682000034618462837BD4680BD80B588B000AF06
:10683000F860B9607A603B600023FB61FB68BB6174
:10684000BB691B687B6107F1100200230121B86856
:1068500005F010FBF861FB69002B01DAFB6933E0FE
:10686000BB6A022B1ED0BB6A022B24DCBB6A002B46
:1068700003D0BB6A012B09D01DE03B69DBB21A468D
:106880000321786900F009FAF86117E03B69002BF1
:1068900014BF01230023DBB21946786900F02CFBFA
:1068A000F8610BE03B69DBB21A460021786900F021
:1068B00077FAF86102E06FF0150305E0FB69002B41
:1068C00001D0FB6900E07B6818462037BD4680BDDB
:1068D000B0B586B000AF786039606FF00B037B61B4
:1068E0000821012008F06AFE38613B69002B02D1C3
:1068F0006FF00B0329E03821012008F05FFEF860FB
:10690000FB68002B08D16FF00B037B6100BF386977
:1069100008F062FE7B6918E0FB680E4A1C461546CB
:106920000FCD0FC40FCD0FC40FCD0FC495E80300DA
:1069300084E803003B69FA685A603B681A683B695F
:106940001A607B683A691A60002318461837BD46FA
:10695000B0BD00BFA001002080B586B000AF786058
:1069600039607B68002B02D03B68002B02D16FF0AE
:106970001503ADE00821012008F020FE38613B69D5
:10698000002B02D16FF00B03A2E03B691A1D3B689C
:10699000043319461046FEF747FF78617B69002BE8
:1069A00040F088803B681B68002B10D03A693B6838
:1069B0001B6819461046FEF7ECFB78617B69002BDB
:1069C00040F08180386900F0A1F8786103E038690F
:1069D00000F082F878617B69002B6DD107F10E031E
:1069E0001A463021386900F0EDF87861FB89B3F57B
:1069F000F75F08D0FB8941F6DF62934203D06FF066
:106A00000D037B6150E0FB89B3F5F75F14D144F2CD
:106A100004025021386900F0A0F8012000F0EBFCDE
:106A20004FF480425021386900F097F84FF400424B
:106A30000021386900F091F807F10E031A4614217D
:106A4000386900F0BFF807F10E031A4601213869D2
:106A500000F0B8F83B68197D3B685B7D1A463869E1
:106A600000F01BF978617B69002B18D13B68997D98
:106A70003B68DB7D1A46386900F092F978617B69E2
:106A8000002B0ED10121386900F036FA78617B695C
:106A9000002B08D17B683A691A60002318E000BF18
:106AA00002E000BF00E000BF3B695B681846FEF7EC
:106AB000F7FE02E000BF00E000BF3B691B6818461C
:106AC000FEF794FB00E000BF38690DF089F87B69A0
:106AD00018461837BD4680BD80B584B000AF7860D9
:106AE0004FF400434FF400423121786800F09EF8E3
:106AF000F860FB68002B01DAFB6803E0012000F07E
:106B00007AFC002318461037BD4680BD80B584B09E
:106B100000AF78607B681B6800211846FEF7AAFB6F
:106B2000F860FB68002B01D0FB6812E0642000F0E5
:106B300057FC7B681B6801211846FEF79BFBF86039
:106B4000FB68002B01D0FB6803E0012000F053FC40
:106B5000002318461037BD4680BD80B584B000AF15
:106B600078600B46FB7013463B80FB785B09FB7239
:106B7000FB7803F01F03BB72FB7A002B0AD07B6803
:106B80005868FB7A43F01003DBB21A461F21FEF768
:106B9000A7FEF8607B685B68B97A3A881846FEF70A
:106BA0009FFEF860FB7A002B07D07B685B681022A1
:106BB0001F211846FEF794FEF860FB681846103750
:106BC000BD4680BD80B586B000AFF8600B467A60E8
:106BD000FB72FB7A5B09FB74FB7A03F01F03BB7447
:106BE000FB7C002B0AD0FB685868FB7C43F0100349
:106BF000DBB21A461F21FEF773FE7861FB685B6803
:106C0000B97C7A681846FEF790FE7861FB7C002B11
:106C100007D0FB685B6810221F211846FEF760FE54
:106C200078617B6918461837BD4680BD80B586B04F
:106C300000AFF860084611461A460346FB720B4641
:106C40003B811346FB8007F11202FB7A1946F86874
:106C5000FFF7B8FF78617B69002B01D07B6918E0F2
:106C6000B7F90630DB431AB27B8A1BB213401BB262
:106C70009BB27B823A89FB8813409AB27B8A13438A
:106C80009BB27B827A8AFB7A1946F868FFF765FF28
:106C9000034618461837BD4680BD80B584B000AFA6
:106CA00078600B46FB701346BB70BB785B08DBB2A9
:106CB000FB81FB78032B34D1BB78052B02D8BB7842
:106CC000042B02D16FF085032DE00121802009F013
:106CD000C3FE0346BB814FF0FF33BB60BB689B071D
:106CE000BB60BB681B0CBB60BB68FA8911461846C9
:106CF00009F0B2FE03469AB2BB891343BB8101215E
:106D00004FF4006009F0A8FE03469AB2BB89134312
:106D1000BB81BB891A4612217868FFF71EFF034624
:106D200001E06FF0850318461037BD4680BD80B581
:106D300088B000AFF860B9607A6007F116031A46B0
:106D40001221F868FFF73EFFF861FB69002B01D0C4
:106D5000FB6921E0BB68002B02D0BB6803221A70DC
:106D60007B68002B17D04FF0FF33BB61BB699B07DB
:106D7000BB61BB691B0CBB61BB69FA8A1146184633
:106D800009F07CFE0346DBB25B00DBB243F001039B
:106D9000DAB27B681A70002318462037BD4680BDE2
:106DA00080B586B000AF78600B46FB701346BB70B1
:106DB000BB789BB203F00103FB82BB785B08DBB2BC
:106DC000BB82FB78002B3ED1BB78052B02D96FF03C
:106DD00085033AE01023002211217868FFF726FF8F
:106DE00038613B69002B01D03B692EE00121012075
:106DF00009F032FE0346FB81FB8A19464FF48050AE
:106E000009F02AFE03469AB2FB891343FB814FF037
:106E1000FF33BB60BB689B07BB60BB681B0DBB60DF
:106E2000BB68BA8A1146184609F016FE03469AB2A4
:106E3000FB891343FB81FB891A4604217868FFF71D
:106E40008CFE034601E06FF0850318461837BD46F7
:106E500080BD90B589B000AFF860B9607A60BB685A
:106E6000002B15D007F116031A461121F868FFF719
:106E7000A9FEF861FB69002B01D0FB6938E0FB8AB1
:106E80001946102009F0FAFD0346DAB2BB681A7001
:106E90007B68002B2BD007F116031A460421F868F3
:106EA000FFF790FEF861FB69002B01D0FB691FE042
:106EB0004FF0FF33BB61BB699B07BB61BB691B0D17
:106EC000BB61BB69FA8A1146184609F0D7FD034633
:106ED000DBB25B00DCB2FB8A19464FF4805009F04C
:106EE000CDFD0346DBB22343DAB27B681A70002380
:106EF00018462437BD4690BD90B585B000AF786088
:106F00000B46FB700121012009F0A6FD03469CB24F
:106F1000FB7819464FF4004009F09EFD03469BB2F2
:106F20002343FB81FA8948F2010304217868FFF7C3
:106F30007DFE034618461437BD4690BD80B584B02B
:106F400000AF786007F10A031A4601217868FFF75D
:106F500039FEF86007F10A031A4601217868FFF745
:106F600031FEF860FB68002B09D17B8919460420AB
:106F700009F084FD0346002B01D0012300E000232B
:106F800018461037BD4680BD80B586B000AF78602A
:106F900039603B68DB683B610821012008F00EFB8B
:106FA000F860FB68002B02D16FF00B0353E0042163
:106FB000012008F003FBB860BB68002B46D0FB68DB
:106FC0003A6911461846FEF7E4F878617B69002BB0
:106FD00037D1FB681A1D3B69143319461046FEF77A
:106FE000D8F878617B69002B24D1FB681B680021ED
:106FF0001846FEF73FF978617B69002B11D1FB68D9
:107000005B6801211846FEF735F978617B69002B32
:1070100009D1BB68FA68DA607B68BA681A60002335
:1070200019E000BF00E000BFFB685B681846FEF790
:10703000DDF800E000BFFB681B681846FEF7D6F8D5
:1070400000E000BFB86808F0C7FA00E000BFF868C9
:1070500008F0C2FA7B6918461837BD4680BD90B566
:1070600091B000AFF8607B600B46FB7213463B812A
:10707000FB68DB68BB63FB7A83F00103DBB287F854
:107080003730FB7A002B10D04FF0FF333B633B6B64
:10709000DB063B633B6BDB0A3B633B6B7968184663
:1070A00009F0ECFC0346DBB201E07B68DBB287F859
:1070B0002F304FF0FF33BB62BB6A9B07BB62BB6ADA
:1070C00097F837201146184609F0C6FC04464FF0E1
:1070D000FF337B627B6A9B077B627B6A9B087B62D8
:1070E0007B6A3A891146184609F0B6FC03461C43F0
:1070F0004FF0FF333B623B6ADB063B623B6A1B0996
:107100003B623A6AFB685B791946104609F0A4FCB9
:1071100003461C434FF0FF33FB61FB69DB06FB6159
:10712000FB695B0AFB61FB6997F82F201146184643
:1071300009F092FC03461C434FF0FF33BB61BB696F
:107140009B07BB61BB699B0BBB61BB6902211846F6
:1071500009F082FC034623437B61BB6B5B68012122
:107160001846FEF787F81F23FB630EE0BB6B1B6816
:1071700001211846FEF7A4F8BB6B1B6800211846D6
:10718000FEF79EF8FB6B013BFB63FB6B002BEDDA1C
:107190001F23FB631DE0BB6B58680122FB6B9A4009
:1071A0007B691340002B14BF01230023DBB2194677
:1071B000FEF786F8BB6B1B6801211846FEF780F8C6
:1071C000BB6B1B6800211846FEF77AF8FB6B013B8E
:1071D000FB63FB6B0F2BDEDC3B89012B02D03B8971
:1071E000002B2BD13B89002B02D17B689BB201E0A5
:1071F0003B6D1B887B820F23FB631BE0BB6B5868D6
:107200007A8AFB6B42FA03F3DBB203F00103DBB2D1
:107210001946FEF755F8BB6B1B6801211846FEF7AF
:107220004FF8BB6B1B6800211846FEF749F8FB6B53
:10723000013BFB63FB6B002BE0DA37E03B6D002288
:107240001A80BB6B5B681846FDF7F2FF0F23FB63E8
:1072500029E0BB6B5B6807F1110211461846FEF787
:1072600055F87B7C002B06D03B6D1B8843F0010357
:107270009AB23B6D1A80FB6B002B05D03B6D1B88CF
:107280005B009AB23B6D1A80BB6B1B6801211846EC
:10729000FEF716F8BB6B1B6800211846FEF710F8C6
:1072A000FB6B013BFB63FB6B002BD2DA0023184620
:1072B0004437BD4690BD80B588B002AFF860B96074
:1072C0001346FB80FB681B79002B04D0BB681F2B87
:1072D00001D9012300E00023FB75FB7D03F00103CE
:1072E000FB75FB7D002B0DD0F97D00230093BB685F
:1072F0000022F868FFF7B3FE38613B69002B01D02C
:107300003B6908E0F97DBB1D0093BB680122F8686A
:10731000FFF7A5FE034618461837BD4680BD80B569
:1073200088B002AFF860B9607A60FB681B79002B07
:1073300004D0BB681F2B01D9012300E00023FB759B
:10734000FB7D03F00103FB75FB7D002B0DD0F97D68
:1073500000230093BB680022F868FFF780FE3861C5
:107360003B69002B01D03B6908E0F97D7B68009305
:10737000BB680222F868FFF772FE0346184618370A
:10738000BD4680BD80B584B000AF78607B68DB68A7
:10739000FB60FB685B681846FDF728FFFB681B680D
:1073A0001846FDF723FFF86808F016F9786808F02A
:1073B00013F9002318461037BD4680BDB0B500AFA5
:1073C000FBF73AFB054BD3E90023541C43F10005BE
:1073D000024BC3E9004500BFB0BD00BFE819002063
:1073E00080B582B000AF78607868FBF74FFC00BFD3
:1073F0000837BD4680BD80B582B000AF78607B683D
:107400004FF47A7202FB03F31846FBF73FFC00BF10
:107410000837BD4680BD80B485B000AFF860B96064
:107420001346FB71FB79002B06D0FB681A68BB681A
:107430001A43FB681A6006E0FB681A68BB68DB4306
:107440001A40FB681A6000BF1437BD465DF8047B24
:107450007047000080B588B000AF786039603B6845
:10746000002B07D03B681B69002B03D03B685B688F
:107470001F2B02DD6FF0150394E01421012008F0AA
:107480009DF878617B69002B02D16FF00B0389E0D6
:107490000C21012008F092F838613B69002B03D1E0
:1074A0006FF00B03FB6179E03B681B69FB603B6895
:1074B0001B7A022B0CD0022B0DDC002B02D0012BEF
:1074C00003D008E00023BB6109E00123BB6106E0B3
:1074D0000223BB6103E06FF01503FB615BE03B68D7
:1074E0001B68032B03DD6FF01503FB6153E03B6862
:1074F0001B68002B13D03B681B68012B0DD03B6829
:107500001B68022B07D03B681B68032B01D1274B5C
:1075100006E0002304E0264B02E0264B00E0264B69
:107520003A6913603B685B68012202FA03F31A466A
:107530003B695A60BB69DAB23B695A723B69002207
:107540001A72FB681A783B699A723B681A687B6901
:107550001A603B685A687B695A603B681A7A7B6993
:107560001A727B693A691A613B681B681846F9F719
:1075700053FB7B691B691846F9F77AFBF861FB69D5
:10758000002B03D06FF01503FB6104E07B687A6980
:107590001A60002306E0386908F01EF8786908F0E0
:1075A0001BF8FB6918462037BD4680BD00B000407F
:1075B00000A00040009000400080004080B582B0F4
:1075C00000AF786039603B68002B04D17B680022F3
:1075D0001A60002304E039687868FFF73BFF034630
:1075E00018460837BD4680BD80B582B000AF7860D0
:1075F0007B68002B02D16FF0150308E07B681B69E4
:10760000184607F0E9FF786807F0E6FF0023184600
:107610000837BD4680BD80B584B000AF78607B6818
:10762000002B03D07B685B681F2B02DD6FF0150316
:1076300009E07B681B69FB60FB6800221A72F8682E
:10764000F9F716FB002318461037BD4680BD80B5FC
:1076500084B000AF78600B46FB707B68002B06D0CF
:107660007B685B681F2B02DCFB78012B02D96FF073
:10767000150330E07B681B69FB60FB681B68BB601F
:10768000FB6801221A72F868F9F7F2FA7B685B6806
:10769000012202FA03F301221946B868FFF7BBFE84
:1076A000FB78002B02D0012B0AD013E07B685B68CB
:1076B000012202FA03F31946B868F9F7C2FB09E0A0
:1076C0007B685B68012202FA03F31946B868F9F790
:1076D000ABFB00BF002318461037BD4680BD80B409
:1076E00085B000AF786039607B68002B03D07B6881
:1076F0005B681F2B02DD6FF015030EE07B681B69D2
:10770000FB60FB681B7A012B03D13B6801221A70D6
:1077100002E03B6800221A70002318461437BD4669
:107720005DF8047B704780B584B000AF78600B468D
:10773000FB707B68002B03D07B685B681F2B02DD2E
:107740006FF015033CE07B681B69FB60FB681B68FE
:10775000BB607B685B68012202FA03F301221946D1
:10776000B868FFF758FEFB78022B1AD0022B23DCF7
:10777000002B02D0012B0AD01EE07B685B6801223F
:1077800002FA03F31946B868F9F75BFB17E07B6868
:107790005B68012202FA03F31946B868F9F744FB63
:1077A0000DE07B685B68012202FA03F300221946B0
:1077B000B868FFF730FE02E06FF0150300E0002329
:1077C00018461037BD4680BD80B584B000AF7860E4
:1077D00039607B68002B03D07B685B681F2B02DD60
:1077E0006FF0150337E07B681B69FB60FB681B6863
:1077F000BB607B685B68012202FA03F30122194631
:10780000B868FFF708FEFB681B7A002B11D17B6874
:107810005B68012202FA03F31946B868F9F7F6FA31
:1078200002467B685B6822FA03F3DAB23B681A709F
:1078300010E07B685B68012202FA03F31946B8681E
:10784000F9F70CFB02467B685B6822FA03F3DAB2B5
:107850003B681A70002318461037BD4680BD0000F3
:1078600080B483B000AF03463960FB7197F90730ED
:10787000002B0BDA3B68DAB20C49FB7903F00F03FB
:10788000043B5201D2B20B441A7609E03B68DAB2EB
:10789000074997F907305201D2B20B4483F800230D
:1078A00000BF0C37BD465DF8047B704700ED00E07B
:1078B00000E100E080B586B000AF78607B687B6156
:1078C0007B695B681C4A934217D07B695B681B4AE3
:1078D000934210D07B695B68194A934209D07B6957
:1078E0005B68184A934201D1032307E04FF0FF334E
:1078F00004E0022302E0012300E000233B61124A7E
:107900003B6952F8233007F108017A69184608F0FC
:1079100025FCF860FB68002B0AD1BB689B68002B34
:1079200007D0BB689B68BA68D2681046984700E0E9
:1079300000BF1837BD4680BD008000400090004069
:1079400000A0004000B00040F019002080B500AF5A
:107950000020F9F7E3FA00BF80BD80B500AF012039
:10796000F9F7DCFA00BF80BD80B500AF0220F9F75F
:10797000D5FA00BF80BD80B500AF0320F9F7CEFA7D
:1079800000BF80BD80B584B000AF786039603B68CF
:10799000002B02D16FF0150331E00C21012007F01C
:1079A0000DFEF860FB68002B02D16FF00B0326E0A0
:1079B0003B681A68FB681A603B689A68FB689A60C3
:1079C0003B681B68104A52F82330002B0DD13B68EE
:1079D0001B689B000C4A13440C4A0321184608F00C
:1079E00021FAB860BB68002B04D17B68FA681A6082
:1079F000002304E000BFF86807F0EEFDBB681846FE
:107A00001037BD4680BD00BFF0190020258500104D
:107A100080B584B000AF78607B68002B06D16FF032
:107A200015031DE0FB68184607F0D6FD7B681B6850
:107A30000D4A52F8233007F10C021146184608F09F
:107A4000C6FB0346002BEDD07B681B68064A52F844
:107A50002330184608F02AFA786807F0BDFD0023A5
:107A600018461037BD4680BDF019002080B590B093
:107A700000AFF860B9607A6007F1280300221A604D
:107A80005A609A60DA60BB68BB62FB68002B02D068
:107A90007B68002B02D16FF01503AAE0FB681B681E
:107AA000564A52F8233007F1280207F138011846E8
:107AB00008F054FBF863FB6B002B40D01021012031
:107AC00007F07CFD0346BB63BB6B002B02D16FF05C
:107AD0000B038EE0BB6BBA681A60FB681B68002B57
:107AE00013D0FB681B68012B0DD0FB681B68022BB1
:107AF00007D0FB681B68032B01D1414B06E0002334
:107B000004E0404B02E0404B00E0404BBA6B536056
:107B1000BB6B7A685268DA60BB6B7A6812689A60ED
:107B2000FB681B68354A52F82330BA6B1146184679
:107B300008F01CFAF863FB6B002B26D054E0BB6BFB
:107B4000BA681A60FB681B68002B13D0FB681B68BF
:107B5000012B0DD0FB681B68022B07D0FB681B684C
:107B6000032B01D1264B06E0002304E0254B02E065
:107B7000254B00E0254BBA6B5360BB6B7A685268AB
:107B8000DA60BB6B7A6812689A60FB681B68002B2E
:107B900013D0FB681B68012B0DD0FB681B68022B00
:107BA00007D0FB681B68032B01D1154A06E00022B1
:107BB00004E0144A02E0144A00E0144A0121BB68C0
:107BC00001FA03F3184607F11C03002119605960FC
:107BD0009960FA613862BA6B07F11C030C491846C8
:107BE000F9F78DF9002304E0BB6B184607F0F4FCAD
:107BF000FB6B18464037BD4680BD00BFF019002022
:107C000000B0004000A00040009000400080004014
:107C1000B578001080B590B000AFF860B9607A60B8
:107C20000023BB6307F1280300221A605A609A60A0
:107C3000DA60BB68BB62FB68002B05D07B68002B59
:107C400002D0BB681F2B02D96FF0150344E0FB681C
:107C50001B68234A52F8233007F1280207F1380144
:107C6000184608F07BFAF863FB6B002B02D06FF02C
:107C7000120331E0FB681B68002B13D0FB681B6804
:107C8000012B0DD0FB681B68022B07D0FB681B681B
:107C9000032B01D1134A06E0002204E0124A02E05D
:107CA000124A00E0124A0121BB6801FA03F31846A8
:107CB00007F11C030021196059609960FA6138626C
:107CC00007F11C03002200211846F9F718F9BB6BD5
:107CD000184607F081FC002318464037BD4680BD9A
:107CE000F019002000B0004000A0004000900040CB
:107CF00000800040B0B590B000AFF860B9601346A6
:107D0000FB71244B07F120041D460FCD0FC42B68D7
:107D10002360FB68002B02D0BB681F2B02D96FF0D9
:107D2000150333E0FB681B68002B13D0FB681B684E
:107D3000012B0DD0FB681B68022B07D0FB681B686A
:107D4000032B01D1144A06E0002204E0134A02E0AA
:107D5000134A00E0134A0121BB6801FA03F31846F5
:107D600007F1340300211960596099607A63B863A0
:107D7000FB799B0040333B4453F8203CDAB207F1D7
:107D8000340311461846F9F777F8002318464037B0
:107D9000BD46B0BD1407021000B0004000A0004076
:107DA000009000400080004080B582B000AF786055
:107DB00039603B681F2B02D96FF0150321E07B6807
:107DC0001B68002B13D07B681B68012B0DD07B68D0
:107DD0001B68022B07D07B681B68032B01D10B4B60
:107DE00006E0002304E00A4B02E00A4B00E00A4BE5
:107DF00001213A6801FA02F211461846F9F74CF8E7
:107E0000002318460837BD4680BD00BF00B00040C3
:107E100000A00040009000400080004080B582B08B
:107E200000AF786039603B681F2B02D96FF01503F3
:107E300021E07B681B68002B13D07B681B68012B3B
:107E40000DD07B681B68022B07D07B681B68032B57
:107E500001D10B4B06E0002304E00A4B02E00A4B81
:107E600000E00A4B01213A6801FA02F21146184675
:107E7000F9F71FF8002318460837BD4680BD00BF3C
:107E800000B0004000A00040009000400080004092
:107E900080B584B000AF78607B681B68002B13D07E
:107EA0007B681B68012B0DD07B681B68022B07D0F9
:107EB0007B681B68032B01D10A4B06E0002304E01A
:107EC000094B02E0094B00E0094B4FF0FF32FA602A
:107ED000FA6811461846F8F7DFFF002318461037F6
:107EE000BD4680BD00B0004000A0004000900040B2
:107EF0000080004080B584B000AF78607B681B686C
:107F0000002B13D07B681B68012B0DD07B681B688E
:107F1000022B07D07B681B68032B01D10A4B06E0BC
:107F2000002304E0094B02E0094B00E0094B4FF04D
:107F3000FF32FA60FA6811461846F8F7BAFF0023D4
:107F400018461037BD4680BD00B0004000A000407C
:107F5000009000400080004080B586B000AFF8601F
:107F6000B9607A60FB681B68002B13D0FB681B6844
:107F7000012B0DD0FB681B68022B07D0FB681B6828
:107F8000032B01D13A2306E0002304E01A2302E088
:107F9000192300E018237B617B695BB2796818467E
:107FA000FFF75EFC002318461837BD4680BD000071
:107FB00080B483B000AF0346FB71FB7903F01F036D
:107FC000012202FA03F1064A97F907305B092033D0
:107FD00042F8231000BF0C37BD465DF8047B7047A4
:107FE00000E100E080B500AF0248F9F732FB00BFC6
:107FF00080BD00BF00D0014080B500AF0248F9F756
:1080000028FB00BF80BD00BF00E0014080B586B006
:1080100000AF78600B46FB707B68002B03D07B6859
:10802000012B07D00DE00E4A07F10C0307CA83E8C5
:10803000070009E00B4A07F10C0307CA83E80700B1
:1080400002E06FF0150307E0FB78BB7507F10C0346
:108050001846F8F70DFE002318461837BD4680BDB8
:108060007C0602108806021080B588B000AF7860E8
:1080700039607B68002B06D03B68002B03D03B683F
:108080001B69002B02D16FF01503C0E03B681B6831
:10809000012B02D96FF01503B9E01821012007F078
:1080A0008DFA02467B681A607B681B68002B02D140
:1080B0006FF00B03ABE00C21012007F07FFAB861F1
:1080C000BB69002B03D16FF00B03FB6199E03B68A8
:1080D0001B697B613B681B68002B07D03B681B68F2
:1080E000012B01D14C4B02E0002300E04B4B3B61E4
:1080F000BB693A691A607B681B683A6812685A6003
:108100003B685B68464A934204D87B681B68444AD4
:108110009A6021E03B685B68424A934204D87B68DE
:108120001B68404A9A6017E03B685B683E4A93428E
:1081300004D87B681B683C4A9A600DE03B685B682A
:108140003A4A934204D87B681B68384A9A6003E035
:108150006FF01503FB6151E07B681B683A68127A87
:108160001A737B681B68BA695A613B681B68304A9E
:1081700052F82330002B10D1BB691B681846F9F761
:108180007DF9002201213869F9F704F90346002B33
:1081900003D04FF0FF33FB6130E07B681B685A6807
:1081A0007B691B7819461046FFF730FFF861FB69C1
:1081B000002B01D0FB692AE03869F9F7ABF9F860C8
:1081C0007B681B689B68FA68934228BF1346FB6074
:1081D000F9683869F9F786F9F861FB69002B02DA6A
:1081E0006FF0150313E03B681B68114A52F8232017
:1081F00001320F4941F82320002308E0B86907F055
:10820000EBF97B681B68184607F0E6F9FB6918462E
:108210002037BD4680BD00BF00E0014000D00140D6
:10822000A0860100801A060040420F0040E13300A2
:10823000001A002080B584B000AF78607B685B696D
:10824000FB607B68002B02D16FF0150331E07B6887
:108250005B681A4A52F82320013A184941F8232052
:108260007B685B68154A52F82330002B1AD1FB68F3
:108270001B681846F9F702F9B860BB68002B01D0FB
:10828000BB6816E07B685B68002B07D07B685B6887
:10829000012B01D1242302E0002300E00D23184626
:1082A000FFF786FEF86807F097F9786807F094F909
:1082B000002318461037BD4680BD00BF001A0020BD
:1082C00080B590B000AFF860B96011461A460B4611
:1082D000FB711346BB71FB68002B03D0FB685B6925
:1082E000002B02D16FF0150352E0FB685B68002B96
:1082F00007D0FB685B68012B01D1274B02E000230C
:1083000000E0264BFB63FB685B69BB63BB79002B1A
:1083100029D1BB6BFA791A72BB6B5B68002B0BD04F
:10832000BB6B5B68FA79114618460BF023FF786344
:10833000BB6B7A6B5A600DE0FB79184607F032F997
:108340000246BB6B5A60BB6B5B68002B02D16FF0BF
:108350000B031DE0BB6B5B68FA79B96818460DF03A
:10836000EDF8002314E0FB6B7B61FB681B7BBB61BA
:10837000BB68FB61FB793B620023BB62BB687B622D
:108380000023FB6207F114031846F9F73AF9034694
:1083900018464037BD4680BD00E0014000D0014096
:1083A00080B590B000AFF860B96011461A460B4630
:1083B000FB711346BB71FB68002B03D0FB685B6944
:1083C000002B02D16FF0150346E0FB685B69FB638D
:1083D000FB685B68002B07D0FB685B68012B01D151
:1083E0001F4B02E0002300E01E4BBB63BB6B7B61B5
:1083F000FB681B7BBB6100233B620023FB61BB6806
:108400007B62FB79BB62BB79002B0CBF012300238D
:10841000DBB2FB62FB6B1B7A002B07D00023FB62F5
:10842000FB6B1B7A3B62FB6B5B68FB6107F1140320
:108430001846F9F7E6F87863FB6B1B7A002B0AD035
:10844000FB6B5B68184607F0C7F8FB6B00221A72DB
:10845000FB6B00225A607B6B18464037BD4680BDDF
:1084600000E0014000D0014080B483B000AF03467B
:10847000FB71FB7903F01F03012202FA03F1064AA4
:1084800097F907305B0942F8231000BF0C37BD464F
:108490005DF8047B704700BF00E100E080B483B06A
:1084A00000AF0346FB71FB7903F01F03012202FAC0
:1084B00003F1064A97F907305B09203342F823108D
:1084C00000BF0C37BD465DF8047B704700E100E05B
:1084D00080B483B000AF03463960FB7197F9073071
:1084E000002B0BDA3B68DAB20C49FB7903F00F037F
:1084F000043B5201D2B20B441A7609E03B68DAB26F
:10850000074997F907305201D2B20B4483F8002390
:1085100000BF0C37BD465DF8047B704700ED00E0FE
:1085200000E100E080B483B000AF786039607B6820
:108530001A683B681B68D31A18460C37BD465DF8AD
:10854000047B704780B485B000AF78600023FB6087
:108550001CE0FB68002B10D0FB68012B0BD0FB68E4
:10856000022B06D0FB68032B01D13A2306E000233F
:1085700004E01A2302E0192300E018237A689342EA
:1085800001D1012306E0FB680133FB60FB68032B8C
:10859000DFD9002318461437BD465DF8047B7047C9
:1085A00080B58AB000AF786007F1100300221A602E
:1085B0005A609A60DA607B68404A93425BD07B687D
:1085C0003E4A934203D07B683D4A934251D07B6838
:1085D0003A4A934207D07B68394A934203D07B687A
:1085E000384A934243D07B68344A93420BD07B682D
:1085F000334A934207D07B68324A934203D07B6868
:10860000314A934231D07B682C4A93420FD07B6829
:108610002B4A93420BD07B682A4A934207D07B684F
:10862000294A934203D07B68284A93421BD07B6837
:10863000224A934215D07B68214A934211D07B682D
:10864000204A93420DD07B681F4A934209D07B6831
:108650001E4A934205D07B681D4A934201D10A23EA
:108660000AE0002308E0092306E0082304E00723CA
:1086700002E0062300E005233B61164B7B627B6A28
:108680005B6807F1100207F10C01184607F066FD60
:1086900038623B6A002B0DD1FB689B68002B05D02C
:1086A000FB689B68FA68D268104698477868FAF7C2
:1086B000E1FD00E000BF2837BD4680BD000001405D
:1086C0000010014000200140003001400040014006
:1086D000005001401802002080B584B000AF7860DF
:1086E0007B68184A93420ED07B68174A934208D0A1
:1086F0007B68164A934201D1022305E04FF0FF3315
:1087000002E0012300E000235B01114A1344FB60F7
:108710007868FBF739F9FB681B68002B0ED0FB6803
:108720009B69002B03D1FB681B69002B03D1FB68FD
:10873000DB68002B02D0F868FBF7D2F800BF1037D7
:10874000BD4680BD0020044000300440004004408D
:10875000081A002080B500AF0248FFF7BDFF00BF38
:1087600080BD00BF0020044080B500AF0248FFF785
:10877000B3FF00BF80BD00BF0030044080B500AF34
:108780000248FFF7A9FF00BF80BD00BF00400440C2
:1087900080B500AF0248FFF703FF00BF80BD00BFF8
:1087A0000000014080B500AF0248FFF7F9FE00BFAE
:1087B00080BD00BF0010014080B500AF0248FFF748
:1087C000EFFE00BF80BD00BF0020014080B584B037
:1087D00000AFF9F7D7FF0346FB60124BBB60FB68A5
:1087E00003F04003002B19D04020F9F7D5FFBB68F8
:1087F0005B683A461146184607F062FC78607B6871
:10880000002B0ADB3B689B68002B07D03B689B680A
:108810003A68D2681046984700E000BF1037BD465E
:1088200080BD00BF0802002080B58AB000AF78602C
:1088300039607B681B683B4A934210D07B681B6899
:10884000394A934209D07B681B68384A934201D168
:10885000022305E04FF0FF3302E0012300E0002394
:108860003B6207F1080300221A605A609A60DA60DE
:108870003B6A002B0BD03B6A012B06D03B6A022BD4
:1088800001D1222304E0002302E00F2300E00E23A5
:10889000BB603B68002B02D0254B7B6218E07B68F5
:1088A000DA687B685B699A4206D17B68DB68002BDB
:1088B00002D0204B7B620BE07B681A697B689B6966
:1088C0009A4229D17B681B69002B25D01A4B7B6209
:1088D0007B6A5B6807F1080207F11801184607F088
:1088E0003DFCF861FB69002B18D1144A3B6A5B011F
:1088F000134400221A60BB699B68002B0FD0104BF9
:1089000001221A70BB699B68BA69D2681046984701
:108910000B4B00221A7002E000BF00E000BF2837B6
:10892000BD4680BD002004400030044000400440AB
:1089300000020020F0010020F8010020081A0020A9
:10894000681A002080B584B000AF786039603B6859
:10895000002B02D16FF0150316E00C21012006F068
:108960002DFEF860FB68002B02D16FF00B030BE0CB
:108970003B681A68FB681A603B689A68FB689A60F3
:108980007B68FA681A60002318461037BD4680BD20
:1089900080B584B000AF78607B68002B02D16FF0A7
:1089A000150326E00023FB601CE0BB68184606F0B8
:1089B00013FE124AFB68DB0013445B6807F10802F0
:1089C0001146184607F003FC0346002BEDD00B4A76
:1089D000FB68DB0013445B68184607F067FAFB6826
:1089E0000133FB60FB68062BE3D9786806F0F4FDE1
:1089F000002318461037BD4680BD00BFE8010020A7
:108A000080B58AB000AFF860B9607A6007F11003F2
:108A100000221A605A609A60DA60BB683B61B868ED
:108A2000FFF790FD0346002B02D06FF0570340E1A3
:108A3000FB68002B02D07B68002B02D16FF015037E
:108A400037E17B685B7A032B00F0C980032B00F3CE
:108A50002181012B02D0022B66D01BE17B681B7A9F
:108A6000964ADB0013445B68002B10D17B681B7AAD
:108A7000DB00924A13440433914A0321184607F05D
:108A8000D1F978627B6A002B01D07B6A11E17B68A7
:108A90001B7A8A4ADB0013445B6807F1100207F176
:108AA0002001184607F05AFB78627B6A002B2BD016
:108AB0001021012006F082FD03463B623B6A002B39
:108AC00002D16FF00B03F4E03B6ABA681A603B6AAC
:108AD0007A68D2685A603B6A7A6812689A603B6A20
:108AE0007A685268DA607B681B7A744ADB00134448
:108AF0005B683A6A1146184607F038FA78627B6A72
:108B0000002B00F0CA80CFE03B6ABA681A603B6A6B
:108B10007A68D2685A603B6A7A6812689A603B6ADF
:108B20007A685268DA60B8E0644B5B6A002B0AD15D
:108B3000634A0321634807F075F978627B6A002B6A
:108B400001D07B6AB5E05D4B5B6A07F120021146FC
:108B5000184607F0B5FA78627B6A002B26D0102100
:108B6000012006F02BFD03463B623B6A002B02D13D
:108B70006FF00B039DE03B6ABA681A603B6A7A6843
:108B8000D2685A603B6A7A6812689A603B6A7A686F
:108B90005268DA60494B5B6A3A6A1146184607F038
:108BA000B0F978627B6A002B0FD07DE03B6ABA682F
:108BB0001A603B6A7A68D2685A603B6A7A681268BF
:108BC0009A603B6A7A685268DA600220F9F7BAFD67
:108BD00078627B6A002B62D06FF00F0369E0374B3D
:108BE0005B6B002B0AD1364A0321374807F01AF98C
:108BF00078627B6A002B01D07B6A5AE07B681B7A23
:108C00002E4ADB0013445B6807F1100207F12001D4
:108C1000184607F0A3FA78627B6A002B2AD010214D
:108C2000012006F0CBFC03463B623B6A002B02D1DD
:108C30006FF00B033DE03B6ABA681A603B6A7A68E2
:108C4000D2685A603B6A7A6812689A603B6A7A68AE
:108C50005268DA607B681B7A184ADB0013445B6851
:108C60003A6A1146184607F081F978627B6A002B50
:108C700017D019E03B6ABA681A603B6A7A68D26812
:108C80005A603B6A7A6812689A603B6A7A685268EE
:108C9000DA6006E06FF015030BE000BF02E000BFF2
:108CA00000E000BF002304E03B6A184606F094FC95
:108CB0007B6A18462837BD4680BD00BFE80100200A
:108CC000258500100C0200201C02002080B58AB00F
:108CD00000AFF860B9607A6000233B6207F11003CF
:108CE00000221A605A609A60DA60BB683B61B8681B
:108CF000FFF728FC0346002B02D06FF0570332E049
:108D0000FB68002B02D07B68002B02D16FF01503AB
:108D100029E07B685B7A012B02D0022B04D009E0AA
:108D20007B68DB687B6105E0114B7B610220F9F712
:108D300019FD00BF7B681B7A0E4ADB0013445B6899
:108D400007F1100207F12001184607F0C2FA786215
:108D50007B6A002B02D06FF0120304E03B6A1846D6
:108D600006F03AFC7B6A18462837BD4680BD00BF36
:108D700000600040E801002080B485B000AFF860DA
:108D8000B9601346FB716FF0570318461437BD46A0
:108D90005DF8047B704780B483B000AF786062B642
:108DA00000BF002318460C37BD465DF8047B7047B2
:108DB00080B483B000AF786072B600BF002318465D
:108DC0000C37BD465DF8047B704780B582B000AFBC
:108DD000786039603B68502B02D96FF0150305E0CD
:108DE0003B685BB21846FFF73FFB00231846083785
:108DF000BD4680BD80B582B000AF786039603B6809
:108E0000502B02D96FF0150305E03B685BB21846A2
:108E1000FFF744FB002318460837BD4680BD80B5E8
:108E200084B000AFF860B9607A60BB68502B02D99B
:108E30006FF0150306E0BB685BB279681846FFF770
:108E400047FB002318461037BD4680BD80B584B06F
:108E500000AF786039603B68002B02D16FF01503DA
:108E600030E01021012006F0A9FBF860FB68002B20
:108E700002D16FF00B0325E03B681A78FB681A708B
:108E80003B685A68FB685A603B689A68FB689A605E
:108E90003B68DA68FB68DA60FB689B68002118466B
:108EA000F9F738FC0346002B08D06FF01503BB60C0
:108EB00000BFF86806F090FBBB6803E07B68FA68C7
:108EC0001A60002318461037BD4680BD80B582B0B9
:108ED00000AF786000BFF9F76FFC0346002BFAD1B2
:108EE000F9F704FC002318460837BD4680BD80B55D
:108EF00082B000AF786000BFF9F75EFC0346002B3C
:108F0000FAD1F9F7FDFB002318460837BD4680BDAE
:108F100080B584B000AF786039607B68002B02D1E7
:108F20006FF0150335E01D4BFB6000BFF9F744FC03
:108F30000346002BFAD1FB681B6943F40042FB682F
:108F40001A6100BFF9F738FC0346002BFAD17868A4
:108F5000FFF7CDFF00BFF9F72FFC0346002BFAD136
:108F6000FB683A681A6000BFF9F726FC0346002B3D
:108F7000FAD17868FFF7AAFF00BFF9F71DFC034696
:108F8000002BFAD1FB681B6923F40042FB681A61CD
:108F9000002318461037BD4680BD00BF006000406A
:108FA00080B582B000AF786039603868F9F78EFB21
:108FB000002318460837BD4680BD000080B586B046
:108FC00000AF78600B46FB707B68022B17D07B6884
:108FD000022B1BD87B68002B03D07B68012B07D0AA
:108FE00014E0124A07F10C0307CA83E8070010E0F7
:108FF0000F4A07F10C0307CA83E8070009E00D4A8E
:1090000007F10C0307CA83E8070002E06FF01503BD
:1090100007E0FB78BB7507F10C031846F7F728FE4D
:10902000002318461837BD4680BD00BF3406021025
:109030004C0602106406021080B586B000AFF860DE
:10904000B9607A6000237B61FB68002B05D0BB68A8
:10905000002B02D07B68002B02D16FF0150343E098
:10906000FB68DB68002B1FD000237B6116E0FB68E8
:10907000D868BA687B691344194606F0A9FD3861BF
:109080003B69002B07D07B69002B01D07B692BE06B
:109090006FF00A0328E07B6901337B617B687A69A2
:1090A0009A42E4D37B691FE0FB681B79002B0DD04B
:1090B000FB681B79012B07D0FB681B79022B01D1C0
:1090C0000B4B04E0002302E00A4B00E00A4B3A1D80
:1090D000B9681846FAF7D6FA38613B69002B02D016
:1090E0006FF0040300E07B6818461837BD4680BD6A
:1090F00000400440003004400020044080B588B0A7
:1091000000AFF860B9607A600023FB61FB68002B58
:1091100005D0BB68002B02D07B68002B4ED16FF0CE
:1091200015034FE07B68202B28BF20237B6100BF05
:10913000FB681B79002B0DD0FB681B79012B07D036
:10914000FB681B79022B01D1204B04E0002302E0D5
:109150001F4B00E01F4B1846FAF7A0FB034603F035
:109160004003002BE4D0FB681B79002B0DD0FB687B
:109170001B79012B07D0FB681B79022B01D1134B04
:1091800004E0002302E0124B00E0124BFA69B968D8
:10919000114407F114021846FAF784FAB8617B69A2
:1091A000FA691344FB617B691A467B689B1A7B60F2
:1091B000BB69002B02D06FF0040303E07B68002B37
:1091C000B0D1FB6918462037BD4680BD0040044041
:1091D000003004400020044080B586B000AFF86045
:1091E000B9607A60FB68002B05D0BB68002B02D009
:1091F0007B68002B02D16FF0150358E0FB681B79E8
:109200007B617B69002B0BD07B69012B06D07B69CE
:10921000022B01D1284B04E0002302E0274B00E0A1
:10922000274B28497A6952010A441360254A7B6911
:109230005B0113440833BA681A60224A7B695B01F8
:10924000134410337A681A601E4A7B695B01134429
:10925000043300221A601B4A7B695B0113440C3300
:1092600000221A60174A7B695B01134418330022FD
:109270001A60144A7B695B0113441C33124A1A605A
:10928000124B1B7883F00103DBB2002B0ED07B69FD
:109290005B010C4A13441846FAF722FB38613B691C
:1092A00013F1060F02D16FF00F0300E00023184600
:1092B0001837BD4680BD00BF004004400030044068
:1092C00000200440081A002029880010681A002095
:1092D00080B586B000AFF860B9607A60FB68002B9B
:1092E00005D0BB68002B02D07B68002B02D16FF049
:1092F000150358E0FB681B797B617B69002B0BD061
:109300007B69012B06D07B69022B01D1284B04E03D
:10931000002302E0274B00E0274B28497A695201DD
:109320000A441360254A7B695B0113440433BA681D
:109330001A60224A7B695B0113440C337A681A6015
:109340001E4A7B695B011344083300221A601B4AE2
:109350007B695B011344103300221A60174A7B6952
:109360005B011344143300221A60144A7B695B01C9
:1093700013441C33124A1A60124B1B7883F001030A
:10938000DBB2002B0ED07B695B010C4A13441846FC
:10939000FAF7A6FA38613B6913F1060F02D16FF0B4
:1093A0000F0300E0002318461837BD4680BD00BFFC
:1093B000004004400030044000200440081A00200F
:1093C00029880010681A002080B584B000AF78604A
:1093D0007B68FB60FB68DB68074A12781146184619
:1093E00006F017FC01220449F868FFF7F5FE00BFFC
:1093F0001037BD4680BD00BF691A002080B592B00D
:1094000000AF786039603B68002B03D03B689B69F4
:10941000002B02D16FF01503A3E11C21012006F0FF
:10942000CDF838633B6B002B02D16FF00B0398E152
:109430000421012006F0C2F8F862FB6A002B03D178
:109440006FF00B037B6488E13B6BFA6A9A613B68BF
:109450001B78002B0DD03B681B78012B07D03B6895
:109460001B78022B01D1944B04E0002302E0934BC4
:1094700000E0934BBB623B689B697B623B681A7858
:109480003B6B1A713B68DA683B6B1A613B685B7C2B
:10949000042B1CD801A252F823F000BFB194001095
:1094A000B7940010BD940010C3940010C99400102C
:1094B00000237B630FE003237B630CE004237B63C7
:1094C00009E002237B6306E001237B6303E06FF086
:1094D00015037B643EE13B681B7C032B16D801A27D
:1094E00052F823F0F5940010FB9400100195001041
:1094F000079500100523FB630CE00623FB6309E0DE
:109500000723FB6306E00823FB6303E06FF015030A
:109510007B641FE13B689B7C002B02D0012B03D0B6
:1095200005E000233B6406E001233B6403E06FF0A9
:1095300015037B640EE17B6A1B78022B0CD0022B97
:109540000DDC002B02D0012B03D008E00023BB630D
:1095500009E00123BB6306E00223BB6303E06FF075
:1095600015037B64F6E03B6B1B691946B86AF9F793
:10957000C3FE78647B6C002B03D06FF015037B6413
:10958000E8E03B6B1B791A467B6A5B78194610460C
:10959000FFF714FD78647B6C002B40F0D380F96BEF
:1095A000B86AF9F793FF78647B6C002B03D06FF0F7
:1095B00015037B64CBE07B6BDBB21946B86AF9F725
:1095C000A3FF78647B6C002B03D06FF015037B64E2
:1095D000BDE03B6CDBB21946B86AF9F785FF7864E9
:1095E0007B6C002B03D06FF015037B64AFE0BB6B8B
:1095F000DBB208221946B86AF9F796FF78647B6CEB
:10960000002B03D06FF015037B64A0E07B683A6BFE
:109610001A603B681B7A002B00F092803B6B0C3386
:10962000184606F07FFA78647B6C002B40F08C8043
:1096300007F1180300221A605A609A60214BFB61FF
:10964000FB6A07F1180211461846FBF7CBFF786456
:109650007B6C002B7AD11C4BBB603B6BFB60022305
:109660003B7401237B743B6B1B79002B0DD03B6B50
:109670001B79012B07D03B6B1B79022B01D10E4BC1
:1096800004E0002302E00D4B00E00D4B7B61FB6A20
:1096900018683B6B1B79002B18D03B6B1B79012B97
:1096A00007D03B6B1B79022B01D122230FE0002353
:1096B0000DE00F230BE000BF0040044000300440E9
:1096C0000020044060070210C99300100E2307F128
:1096D00008021946FBF7D3FF78647B6C002B26D178
:1096E000FB6A1A683B6B1B79002B0DD03B6B1B7917
:1096F000012B07D03B6B1B79022B01D1222304E005
:10970000002302E00F2300E00E2319461046FCF769
:1097100023F878647B6C002B0BD101221349386B42
:10972000FFF75AFD78647B6C002B09D002E000BF84
:1097300000E000BFFB6A1B681846FBF780FF06E0ED
:1097400000230EE000BF02E000BF00E000BFB86AE7
:10975000F9F75EFEF86A05F03FFF386B05F03CFF55
:109760007B6C18464837BD4680BD00BF691A002093
:1097700080B588B000AF786007F10C0300221A6052
:109780005A609A60DA6002233B7501237B757B681F
:109790001B79002B0DD07B681B79012B07D07B68D0
:1097A0001B79022B01D13A4B04E0002302E0394B34
:1097B00000E0394BBB617B68002B02D16FF01503D1
:1097C00062E07B689B69FB617B68DB68002B3CD0B7
:1097D000FB691A687B681B79002B0DD07B681B79AD
:1097E000012B07D07B681B79022B01D1222304E0D7
:1097F000002302E00F2300E00E2319461046FBF77A
:10980000CDFFFB6918687B681B79002B0DD07B6846
:109810001B79012B07D07B681B79022B01D12223F6
:1098200004E0002302E00F2300E00E2307F10C0206
:109830001946FBF748FF7B68DB68184606F00AFA12
:109840007B68DB68184605F0C7FE7B681B79002B38
:109850000DD07B681B79012B07D07B681B79022B0D
:1098600001D10B4B04E0002302E00A4B00E00A4B5D
:109870001846F9F7CDFD7B689B69184605F0ACFEEC
:10988000786805F0A9FE002318462037BD4680BD44
:1098900000400440003004400020044080B483B005
:1098A00000AF78606FF0570318460C37BD465DF87F
:1098B000047B704780B582B000AF78607B68002B76
:1098C0000BD0084A7B681360074B1B68986800231D
:1098D000022200210BF0ACF800E000BF0837BD46C3
:1098E00080BD00BF6C1A0020E410002080B582B05B
:1098F00000AF78607B68002B04DB7B68022B01DC07
:10990000002306E00BF0EAFB034609221A604FF041
:10991000FF3318460837BD4680BD80B582B000AF22
:1099200078607B68002B04DB7B68022B01DC012361
:1099300005E00BF0D3FB034609221A60002318460A
:109940000837BD4680BD80B584B000AFF860B9600F
:109950007A600BF0C3FB034609221A604FF0FF3315
:1099600018461037BD4680BD80B582B000AF786024
:1099700039607B68002B08DB7B68022B05DC3B68C9
:109980004FF400525A60002305E00BF0A7FB03469A
:1099900009221A60002318460837BD4680BD000022
:1099A00080B586B000AFF860B9607A60FB68002BC4
:1099B00015D1104B1B687A68B9681846FCF74CF84B
:1099C00078617B69002B08DA0BF088FB02467B6923
:1099D0005B4213604FF0FF3308E07B6906E00BF059
:1099E0007DFB034609221A604FF0FF3318461837F3
:1099F000BD4680BD6C1A002080B586B000AFF8600F
:109A0000B9607A60FB68012B02D0FB68022B15D18C
:109A1000104B1B687A68B9681846FCF74FF87861F4
:109A20007B69002B08DA0BF059FB02467B695B422D
:109A300013604FF0FF3308E07B6906E00BF04EFB4C
:109A4000034609221A604FF0FF3318461837BD4607
:109A500080BD00BF6C1A00202DE9B04F86B000AF6A
:109A6000F860C7E9002397F844300821184605F04C
:109A7000A5FD0246FB685A60FB685B68002B02D1BB
:109A80006FF00B034FE097F844300121184605F0C2
:109A900095FD0246FB689A60FB689B68002B0AD123
:109AA0006FF00B033B6100BFFB685B68184605F075
:109AB00093FD3B6937E000237B612AE07B69DA177D
:109AC00098469146BB6B09FB03F2FB6B08FB03F363
:109AD0001344BA6BA2FB08452B441D46FB685A6829
:109AE0007B69DB00D118D7E9002314EB020A45EBB0
:109AF000030BC1E900AB7B69D9B2FB689A687B694B
:109B0000134497F840200A44D2B21A707B6901339B
:109B10007B6197F844307A699A42CFDBFB6897F80B
:109B200044201A73002318461837BD46BDE8B08F8D
:109B300080B58AB004AF786039607B68002B02D0B2
:109B40003B68002B02D16FF01503CFE120210120EB
:109B500005F034FDF860FB68002B02D16FF00B03B9
:109B6000C4E13B681B78002B02D0012B06D00BE030
:109B7000954B3B61FB6806225A7009E0934B3B61B1
:109B8000FB6807225A7003E06FF015037B61A9E1BF
:109B90003B681A78FB681A703B685B78032B4FD8D8
:109BA00001A252F823F000BFB99B0010DB9B00100C
:109BB000FD9B00101F9C00101F2303932223029380
:109BC00073A3D3E90023CDE9002373A3D3E90023D2
:109BD000F868FFF741FF786135E02B2303931223E8
:109BE00002936FA3D3E90023CDE900236EA3D3E949
:109BF0000023F868FFF730FF786124E01023039317
:109C0000112302936AA3D3E90023CDE9002362A3C1
:109C1000D3E90023F868FFF71FFF786113E01123F1
:109C200003930A23029364A3D3E90023CDE900231D
:109C300063A3D3E90023F868FFF70EFF786102E021
:109C40006FF015037B617B69002B40F04A81FB6854
:109C500003F110023B68043319461046FBF799FAEA
:109C600078617B69002B40F03081FB6803F11402BE
:109C70003B68183319461046FBF78BFA78617B690D
:109C8000002B40F01B81FB6803F118023B682C336A
:109C900019461046FBF77DFA78617B69002B40F08E
:109CA0000681FB6803F11C023B68403319461046ED
:109CB000FBF76FFA78617B69002B40F0F180FB685D
:109CC0001B6901211846FBF7D5FA78617B69002BE7
:109CD00040F0C780FB685B6900211846FBF7CAFAB1
:109CE00078617B69002B40F0BE80FB689B69002196
:109CF0001846FBF7BFFA78617B69002B40F0B5800E
:109D0000FB68DB691846FBF793FA78617B69002BE7
:109D100040F0AD803969F86800F092FA78617B69AB
:109D2000002B40F0A6803B6893F854301946F86841
:109D300000F0D9FB78617B69002B40F09C803B6888
:109D400093F855301946F86800F039FB78617B6963
:109D5000002B40F092803B6893F860301946F86819
:109D600000F0B6FD78617B69002B40F088803B688D
:109D70001B78002B2CD13B6893F861301946F868AA
:109D800000F00BFE78617B69002B56D082E000BFAB
:109D900080B2E60E000000000095A9270D0000002B
:109DA000A06EA50F0000000040BFB4D50C0000005D
:109DB0000065CD1D0000000000BF2F200000000046
:109DC0000016C5530D000000A4070210BC070210C6
:109DD0003B6893F865301946F86800F099FF7861A0
:109DE0007B69002B4DD13B6893F861103B6893F879
:109DF00062301A46F86800F0E0FF78617B69002B5A
:109E000041D13B6893F863103B6893F864301A467D
:109E1000F86801F065F878617B69002B35D13B6803
:109E200093F866103B6893F867301A46F86801F0BB
:109E3000F0F878617B69002B29D13B6893F85430A6
:109E4000002B09D03B68D3E91623F86800F0FAFD2F
:109E500078617B69002B1CD17B68FA681A6000234B
:109E600044E000BF16E000BF14E000BF12E000BFF6
:109E700010E000BF0EE000BF0CE000BF0AE000BF32
:109E800008E000BF06E000BF04E000BF02E000BF42
:109E900000E000BFFB68DB691846FBF7A7F900E0AC
:109EA00000BFFB689B691846FBF7A0F900E000BF04
:109EB000FB685B691846FBF799F900E000BFFB6897
:109EC0001B691846FBF792F900E000BFFB685B686E
:109ED000184605F081FBFB689B68184605F07CFB83
:109EE00000E000BFF86805F077FB7B69184618377B
:109EF000BD4680BD80B584B000AF78607B685B688C
:109F0000184605F069FB7B6800225A607B689B68F5
:109F1000184605F061FB7B6800229A607B681B692C
:109F20001846FBF763F9F860FB68002B01D0FB686B
:109F300024E07B685B691846FBF758F9F860FB681A
:109F4000002B01D0FB6819E07B689B691846FBF782
:109F50004DF9F860FB68002B01D0FB680EE07B68D0
:109F6000DB691846FBF742F9F860FB68002B01D06B
:109F7000FB6803E0786805F02FFB002318461037D4
:109F8000BD4680BD80B483B000AF78607B68002B95
:109F900002D07B681B7800E0EA2318460C37BD46E8
:109FA0005DF8047B704780B586B000AF78600B46E3
:109FB000FB701346BB707B68002B02D16FF015035A
:109FC0006DE0BB783B614FF0FF33FB60FB689B06A5
:109FD000FB60FB689B0CFB60FB68FA781146184637
:109FE00006F03AFD02463B6913433B6101214FF401
:109FF000804006F031FD02463B6913433B614FF060
:10A00000FF33BB60BB685B07BB60BB689B0BBB607F
:10A01000BA687B685B781946104606F01DFD02465B
:10A020003B6913433B617B681B6900211846FBF7C2
:10A0300047F900237B6122E07B689A693B69DBB2C8
:10A0400003F00103DBB219461046FBF739F9012092
:10A05000FDF7C6F97B685B6901211846FBF730F90B
:10A060000120FDF7BDF97B685B6900211846FBF70D
:10A0700027F93B695B083B617B6901337B617B6945
:10A08000112BD9DD7B689B6900211846FBF718F975
:10A090007B681B6901211846FBF712F9002318465B
:10A0A0001837BD4680BD80B58AB000AFF8600B465A
:10A0B0007A60FB720023FB7500233B62FB68002B78
:10A0C00002D07B68002B02D16FF01503B4E04FF093
:10A0D000FF33FB61FB699B06FB61FB699B0CFB612A
:10A0E000FB69FA7A1146184606F0B6FC38624FF062
:10A0F000FF33BB61BB695B07BB61BB699B0BBB618A
:10A10000BA69FB685B781946104606F0A5FC024662
:10A110003B6A13433B62FB681B6900211846FBF74F
:10A12000CFF800237B6222E0FB689A693B6ADBB2CE
:10A1300003F00103DBB219461046FBF7C1F801201A
:10A14000FDF74EF9FB685B6901211846FBF7B8F88B
:10A150000120FDF745F9FB685B6900211846FBF714
:10A16000AFF83B6A5B083B627B6A01337B627B6AC8
:10A17000112BD9DDFB689B6900211846FBF7A0F87D
:10A18000FB681B6901211846FBF79AF80120FDF7CF
:10A1900027F9FB685B6901211846FBF791F801205C
:10A1A000FDF71EF9FB685B6900211846FBF788F88C
:10A1B0000120FDF715F97B6800221A70FB681B6906
:10A1C00000211846FBF77CF800237B622AE0FB683D
:10A1D0005B6901211846FBF773F80120FDF700F9D0
:10A1E000FB685B6900211846FBF76AF8FB68DB69CE
:10A1F00007F1170211461846FBF788F80120FDF712
:10A20000EFF87B681B785AB2FB7D19467B6A01FA2E
:10A2100003F35BB213435BB2DAB27B681A707B6AFA
:10A2200001337B627B6A072BD1DDFB681B6901214F
:10A230001846FBF745F8002318462837BD4680BD71
:10A2400080B588B000AF786039607B681B78012BDF
:10A2500006D10023FB610A23BB610F237B6106E06B
:10A260000123FB610D23BB610F237B6100BF35E040
:10A27000FA69BB699A4203DBFA697B699A4229DD74
:10A28000FB693A6813441B78FB73FB69DBB2FA7B0A
:10A2900019467868FFF787FE38613B69002B01DAC1
:10A2A0003B691FE0FB69DBB207F10F0219467868D2
:10A2B000FFF7F9FE38613B69002B01DA3B6911E0D9
:10A2C000FB693A6813441A78FB7B9A4203D06FF01B
:10A2D0000D0307E000BFFB690133FB61FB69172B2E
:10A2E000C6DD002318462037BD4680BD80B586B048
:10A2F00000AF78600B467B8013467B707B881B0A1F
:10A300009BB2FB757B88BB7507F10F02FB7D19467D
:10A310007868FFF7C8FE38613B69002B01D03B69C4
:10A320001CE097F91630DB435AB2FB7B5BB213405B
:10A330005BB2DBB2FB73BB7D7A781146184606F040
:10A340008BFB0346DAB2FB7B1343DBB2FB73FA7B76
:10A35000FB7D19467868FFF726FE03461846183736
:10A36000BD4680BD80B586B000AFF8600B467A6010
:10A370007B817B68002B02D16FF015031BE07B898A
:10A380001B0A9BB2DBB207F113021946F868FFF70C
:10A390008AFE78617B69002B01D07B690BE07B89A9
:10A3A000DBB2FA7C1146184606F068FB0346DAB2C7
:10A3B0007B681A70002318461837BD4680BD80B5EB
:10A3C00084B000AF78600B46FB707B681B78012B74
:10A3D00006D14FF41263FB814FF41463BB8106E096
:10A3E00040F20133FB8140F60123BB8100BFFA78C4
:10A3F000FB8919467868FFF779FFB860BB68002BC6
:10A4000001D0BB680AE0FB7883F00103DBB21A4697
:10A41000BB8919467868FFF769FF0346184610376D
:10A42000BD4680BD80B586B000AF786039607B687E
:10A430001B78012B06D14FF41263FB824FF4146397
:10A44000BB8206E040F20133FB8240F60123BB826F
:10A4500000BF07F10F02FB8A19467868FFF782FFF9
:10A4600038613B69002B01D03B691BE007F10E020C
:10A47000BB8A19467868FFF775FF38613B69002B86
:10A4800001D03B690EE0FB7B002B04D0BB7B002B93
:10A4900001D1012300E0002303F00103DAB23B689D
:10A4A0001A70002318461837BD4680BD80B584B0A9
:10A4B00000AF786039604FF0FF33FB60FB68DB066C
:10A4C000FB60FB68DB0EFB60FB689BB243F4D85378
:10A4D0009BB23A6819467868FFF744FF034618466E
:10A4E0001037BD4680BD80B584B000AF78600B46A4
:10A4F000FB706FF00D03FB607B681B78002B40F056
:10A50000A180FB7883F00103DBB21A464FF402719D
:10A510007868FFF7EBFEF860FB68002B01D0FB6862
:10A52000EDE0FB7883F00103DBB21A464FF40171D2
:10A530007868FFF7DBFEF860FB68002B01D0FB6852
:10A54000DDE0FB7883F00103DBB21A4640F2012123
:10A550007868FFF7CBFEF860FB68002B01D0FB6842
:10A56000CDE0FB7883F00103DBB21946802006F0D2
:10A5700073FA0346FB72FB7883F00103DBB21946E2
:10A58000402006F069FA0346DAB2FB7A1343FB7205
:10A59000FB7883F00103DBB21946202006F05CFA59
:10A5A0000346DAB2FB7A1343FB72FB7883F00103B4
:10A5B000DBB21946102006F04FFA0346DAB2FB7AF6
:10A5C0001343FB72FB7883F00103DBB219460820CA
:10A5D00006F042FA0346DAB2FB7A1343FB72FB78C9
:10A5E00083F00103DBB21946042006F035FA034676
:10A5F000DAB2FB7A1343FB72FB7883F00103DBB220
:10A600001946022006F028FA0346DAB2FB7A134311
:10A61000FB72FB7883F00103DBB21946012006F0E0
:10A620001BFA0346DAB2FB7A1343FB72FB7A1A4633
:10A6300004217868FFF7B7FCF860FB68002B56D060
:10A64000FB685CE0FB78002B01D0002300E0FF23D7
:10A65000FB72FB7A1A4600217868FFF7A4FCF860C9
:10A66000FB68002B01D0FB6849E0FB78194602200B
:10A6700006F0F2F90346FB72FB7883F00103DBB2CC
:10A680001946802006F0E8F90346DAB2FB7A134354
:10A69000FB72FB7883F00103DBB21946402006F021
:10A6A000DBF90346DAB2FB7A1343FB72FB7883F0E3
:10A6B0000103DBB21946102006F0CEF90346DAB2E8
:10A6C000FB7A1343FB72FB7883F00103DBB219467C
:10A6D000202006F0C1F90346DAB2FB7A1343FB727D
:10A6E000FB7A1A4601217868FFF75DFCF860FB7879
:10A6F0001A4641F202017868FFF7F8FD0346184652
:10A700001037BD4680BD80B586B000AF7860396037
:10A710006FF00D033B610123BB757B681B78002B39
:10A7200043D10121082006F097F90346FB7301216C
:10A73000042006F091F90346FB730121012006F085
:10A740008BF90346FB7307F10E031A460221786862
:10A75000FFF7A9FC38613B69002B01D03B69B3E0EE
:10A76000BA7BFB7B1340DBB2002B14BF0123002319
:10A77000FB7507F10E031A4604217868FFF793FC76
:10A7800038613B69002B01D03B699DE0FB7D002BCC
:10A7900004D0BB7B002B01D0012300E00023FB751C
:10A7A000FB7D03F00103FB7560E007F10E031A4621
:10A7B00000217868FFF777FC38613B69002B01D0F6
:10A7C0003B6981E0BB7B002B14BF01230023FB7599
:10A7D0000121102006F040F90346FB7301212020DF
:10A7E00006F03AF90346DAB2FB7B1343FB7301210F
:10A7F000402006F031F90346DAB2FB7B1343FB73CA
:10A800000121802006F028F90346DAB2FB7B1343CE
:10A81000FB7307F10E031A4601217868FFF743FC2A
:10A8200038613B69002B01D03B694DE0FB7D002B7B
:10A8300007D0BA7BFB7B1340DBB2002B01D0012396
:10A8400000E00023FB75FB7D03F00103FB75012194
:10A85000022006F001F90346FB73BA7BFB7B134031
:10A86000DBB2002B14BF01230023BB7507F10E03DD
:10A870001A4641F202017868FFF774FD38613B69BE
:10A88000002B01D03B691FE0BB7D002B04D0BB7BBC
:10A89000002B01D0012300E00023BB75BB7D03F03A
:10A8A0000103BB75FB7D83F00103DBB2002B04D0F9
:10A8B000BB7D002B01D0012300E0002303F0010346
:10A8C000DAB23B681A70002318461837BD4680BDBF
:10A8D00080B586B000AF78600B46FB707B681B7854
:10A8E000012B0ED14FF0FF333B613B691B073B61EE
:10A8F0003B691B0E3B613B699BB243F4A063FB8247
:10A900000EE04FF0FF33FB60FB681B07FB60FB684A
:10A910001B0EFB60FB689BB243F4E063FB8200BF4D
:10A92000FA78FB8A19467868FFF7E0FC0346184678
:10A930001837BD4680BD80B586B000AF78603960FD
:10A940007B681B78012B0ED14FF0FF333B613B69D5
:10A950001B073B613B691B0E3B613B699BB243F4A8
:10A96000A063FB820EE04FF0FF33FB60FB681B0728
:10A97000FB60FB681B0EFB60FB689BB243F4E0636B
:10A98000FB8200BFFB8A3A6819467868FFF7EAFC49
:10A99000034618461837BD4680BD80B584B000AF69
:10A9A00078600B46FB707B68002B02D16FF01503BB
:10A9B0001AE07B681B78002B02D06FF0570313E07E
:10A9C0004FF0FF33FB60FB681B07FB60FB681B0E4F
:10A9D000FB60FB689BB243F430639BB2FA78194684
:10A9E0007868FFF783FC034618461037BD4680BDE4
:10A9F00080B584B000AF786039607B68002B02D1ED
:10AA00006FF015031AE07B681B78002B02D06FF003
:10AA1000570313E04FF0FF33FB60FB681B07FB603D
:10AA2000FB681B0EFB60FB689BB243F430639BB278
:10AA30003A6819467868FFF795FC034618461037C0
:10AA4000BD4680BD80B58EB000AFF860C7E9002379
:10AA50004FF0FF33FB624FF0FF33BB62FB681B7BA1
:10AA6000013B7B630FE0FB685A687B6BDB001344A0
:10AA7000D3E90023D7E90001994208BF904206D0EC
:10AA80007B6B013B7B637B6B002BECDA00E000BF50
:10AA90007B6B002B02DA6FF01503A2E04FF0FF335F
:10AAA0007B627B6A5B067B627B6A5B0E7B627B6A96
:10AAB0009BB243F4A05399B2FB689A687B6B134432
:10AAC0001B781A46F868FFF711FC38623B6A002BC6
:10AAD00001D03B6A85E000233B633FE00023FB7528
:10AAE0004FF0FF33FB61FB695B06FB61FB695B0EAB
:10AAF000FB61FB699BB243F4B0539BB23A6BD2B299
:10AB00001946F868FFF7F2FB38623B6A002B01D068
:10AB10003B6A66E00120FCF76EFC07F117031A465A
:10AB200041F60801F868FFF71DFC38623B6A002B0C
:10AB300001D03B6A55E0FB7D002B06D03B6BBB622E
:10AB4000FB6A002B01DA3B6BFB62FB7D002B02D121
:10AB5000BB6A002B06DA3B6B01333B633B6B132B69
:10AB6000BCDD00E000BFBB6A002B02DA6FF00D0312
:10AB700037E04FF0FF33BB61BB695B06BB61BB696C
:10AB80005B0EBB61BB699BB243F4B05399B2FA6AE6
:10AB9000BB6A13440133DA0F13445B10DBB21A466D
:10ABA000F868FFF7A3FB38623B6A002B01D03B6AD1
:10ABB00017E00120FCF71FFC07F117031A4641F6C6
:10ABC0000801F868FFF7CEFB38623B6A002B01D022
:10ABD0003B6A06E0FB7D002B01D0002301E06FF013
:10ABE0000D0318463837BD4680BD80B586B000AF2E
:10ABF000786039607B68002B02D03B68002B02D163
:10AC00006FF015035FE007F10A031A4641F60801E9
:10AC10007868FFF7A7FB38613B69002B01D03B69DF
:10AC200051E0BB7A002B08D139684FF000024FF099
:10AC30000003C1E90023002345E04FF0FF33FB6030
:10AC4000FB685B06FB60FB685B0EFB60FB689BB20E
:10AC500043F4A0539BB207F10B0219467868FFF743
:10AC600081FB38613B69002B01D03B692BE07B689D
:10AC70001B7B013B7B610AE07B689A687B6913441C
:10AC80001A78FB7A9A4206D07B69013B7B617B692B
:10AC9000002BF1DA00E000BF7B69002B08DA39688D
:10ACA0004FF000024FF00003C1E9002300230AE047
:10ACB0007B685A687B69DB001344D3E90023396859
:10ACC000C1E90023002318461837BD4680BD80B473
:10ACD00085B000AFF860B9607A60FB68002B05D0E2
:10ACE000BB68002B02D07B68002B02D16FF01503EC
:10ACF00008E0FB685A68BB681A60FB681A7B7B68CF
:10AD00001A70002318461437BD465DF8047B70475F
:10AD100080B584B000AF78600B46FB707B68002B79
:10AD200002D16FF015031AE07B681B78012B02D06B
:10AD30006FF0570313E04FF0FF33FB60FB689B0796
:10AD4000FB60FB68DB0EFB60FB689BB243F40063B7
:10AD50009BB2FA7819467868FFF7C8FA0346184696
:10AD60001037BD4680BD80B584B000AF78603960D3
:10AD70007B68002B02D16FF015031AE07B681B780B
:10AD8000012B02D06FF0570313E04FF0FF33FB604D
:10AD9000FB689B07FB60FB68DB0EFB60FB689BB2FC
:10ADA00043F400639BB23A6819467868FFF7DAFA11
:10ADB000034618461037BD4680BD80B586B000AF4B
:10ADC00078600B46FB701346BB707B68002B02D18A
:10ADD0006FF015033CE07B681B78012B02D06FF00D
:10ADE000570335E0FB78032B02D8BB78032B02D93D
:10ADF0006FF015032CE04FF0FF337B617B699B07FD
:10AE00007B617B691B0F7B617B699BB243F4807321
:10AE10009BB2FA7819467868FFF768FA38613B699F
:10AE2000002B01D03B6913E04FF0FF33FB60FB6860
:10AE30009B07FB60FB689B0FFB60FB689BB243F4C6
:10AE400000739BB2BA7819467868FFF74FFA034649
:10AE500018461837BD4680BD80B588B000AFF86091
:10AE6000B9607A60FB68002B02D16FF0150333E004
:10AE7000FB681B78012B02D06FF057032CE04FF0DA
:10AE8000FF33FB61FB699B07FB61FB691B0FFB61E8
:10AE9000FB699BB243F480739BB2BA681946F868A9
:10AEA000FFF760FAB861BB69002B01D0BB6913E002
:10AEB0004FF0FF337B617B699B077B617B699B0F55
:10AEC0007B617B699BB243F400739BB27A6819463D
:10AED000F868FFF747FA034618462037BD4680BD9D
:10AEE00080B586B000AF78600B46FB701346BB7030
:10AEF0007B68002B02D16FF0150342E07B681B7862
:10AF0000012B02D06FF057033BE0FB78032B08D0F6
:10AF1000FB78062B05D8BB78032B02D0BB78062B19
:10AF200002D96FF015032CE04FF0FF337B617B6992
:10AF30005B077B617B691B0E7B617B699BB243F482
:10AF400000739BB2FA7819467868FFF7CFF9386139
:10AF50003B69002B01D03B6913E04FF0FF33FB60EE
:10AF6000FB685B07FB60FB68DB0EFB60FB689BB26A
:10AF700043F400739BB2BA7819467868FFF7B6F9C4
:10AF8000034618461837BD4680BD80B588B000AF6F
:10AF9000F860B9607A60FB68002B02D16FF015038E
:10AFA00033E0FB681B78012B02D06FF057032CE0D5
:10AFB0004FF0FF33FB61FB695B07FB61FB691B0E15
:10AFC000FB61FB699BB243F400739BB2BA681946FC
:10AFD000F868FFF7C7F9B861BB69002B01D0BB69FE
:10AFE00013E04FF0FF337B617B695B077B617B691B
:10AFF000DB0E7B617B699BB243F400739BB27A6882
:10B000001946F868FFF7AEF9034618462037BD46E3
:10B0100080BD80B586B000AF78600B46FB701346EC
:10B02000BB707B68002B02D16FF0150333E07B68A7
:10B030001B78012B02D06FF057032CE04FF0FF3349
:10B040007B617B699B077B617B691B0E7B617B69F5
:10B050009BB243F440739BB2FA7819467868FFF7C5
:10B0600045F938613B69002B01D03B6913E04FF093
:10B07000FF33FB60FB689B07FB60FB689B0EFB607C
:10B08000FB689BB243F440739BB2BA781946786868
:10B09000FFF72CF9034618461837BD4680BD80B52A
:10B0A00088B000AFF860B9607A60FB68002B02D10D
:10B0B0006FF0150333E0FB681B78012B02D06FF0B3
:10B0C00057032CE04FF0FF33FB61FB699B07FB61EB
:10B0D000FB691B0EFB61FB699BB243F440739BB29F
:10B0E000BA681946F868FFF73DF9B861BB69002BEB
:10B0F00001D0BB6913E04FF0FF337B617B699B0795
:10B100007B617B699B0E7B617B699BB243F44073DF
:10B110009BB27A681946F868FFF724F90346184687
:10B120002037BD4680BD80B586B000AFF860B960FD
:10B130007A60FB681B68BA68D1B207F1130218463F
:10B14000FEF7B1FF78617B69002B01D07B6904E0D9
:10B15000FB7C1A467B681A60002318461837BD46E8
:10B1600080BD80B584B000AFF860B9607A60FB68DC
:10B170001B68BA68D1B27A68D2B21846FEF713FFDC
:10B18000034618461037BD4680BD000080B592B01A
:10B1900002AFF860B9607A603B60FB68FB63FB6BF1
:10B1A0001B68BB63BB6C0E2B00F2FB8001A252F844
:10B1B00023F000BFF1B10010BDB2001011B20010B9
:10B1C000A3B3001043B200107DB200109FB2001074
:10B1D000DDB20010FBB2001019B3001019B300105B
:10B1E00047B3001047B3001075B3001075B30010DB
:10B1F00007F12B031946B86BFFF785FA78637B6B71
:10B20000002B01D07B6BD9E097F82B30FB62CBE0B1
:10B2100007F120031946B86BFFF7E7FC78637B6BF7
:10B22000002B01D07B6BC9E0D7E908014FF47A729B
:10B230004FF0000308F01AFB02460B461346FB6270
:10B24000B2E04FF0FF333B633B6B5B063B633B6B12
:10B250005B0E3B633B6B9BB243F4B0539BB207F175
:10B260001E021946B86BFFF77DF878637B6B002BE5
:10B2700001D07B6BA2E0BB7FFB6295E007F11D0371
:10B280001A4641F60801B86BFFF76CF878637B6BE0
:10B29000002B01D07B6B91E07B7FFB6284E007F1A8
:10B2A0001F031946B86BFFF746FB78637B6B002BD7
:10B2B00001D07B6B82E0FB7FFB6275E007F12B0323
:10B2C0001946B86BFFF7AEF878637B6B002B01D0A3
:10B2D0007B6B73E097F82B30FB6265E007F11F038F
:10B2E0001946B86BFFF784FB78637B6B002B01D0AA
:10B2F0007B6B63E0FB7FFB6256E007F11C031946A2
:10B30000B86BFFF730FD78637B6B002B01D07B6B54
:10B3100054E03B7FFB6247E007F11A0207F11B0391
:10B320001946B86BFFF798FD78637B6B002B01D053
:10B330007B6B43E0BB6C092B02D1FB7EFB6233E0ED
:10B34000BB7EFB6230E007F1180207F119031946D2
:10B35000B86BFFF71AFE78637B6B002B01D07B6B19
:10B360002CE0BB6C0B2B02D17B7EFB621CE03B7E96
:10B37000FB6219E007F1160207F117031946B86BD3
:10B38000FFF78DFE78637B6B002B01D07B6B15E0A4
:10B39000BB6C0D2B02D1FB7DFB6205E0BB7DFB622C
:10B3A00002E06FF0150309E007F12C03009301237D
:10B3B00001227968B86800F00DFE03461846403750
:10B3C000BD4680BD2DE9B04F8AB000AFF860B960CE
:10B3D0007A603B6000237B62FB683B623B6A1B68D0
:10B3E000FB6107F1180200230121B86800F042FD5B
:10B3F00078627B6A002B01DA7B6AFBE0BB6C0E2B68
:10B4000000F2EA8001A252F823F000BF49B4001014
:10B41000DBB4001061B40010D9B50010D9B500102C
:10B42000D9B50010CBB40010F3B4001003B5001070
:10B4300013B5001013B5001055B5001055B5001028
:10B4400097B5001097B50010BB69002B14BF0123FE
:10B450000023DBB21946F869FFF745F87862C3E0CC
:10B46000BB69DA179846914642464B464FF00000BA
:10B470004FF00001590141EAD261500102460B46EA
:10B48000B2EB080463EB09054FF000024FF0000334
:10B49000AB0043EA9473A20014461D4614EB080A5D
:10B4A00045EB090B4FF000024FF000034FEACB03CE
:10B4B00043EA5A734FEACA0292469B4652465B469B
:10B4C000F869FFF7BFFA78628EE0BB69DBB2194614
:10B4D000F869FFF7FDF9786286E0BB69002B14BFBD
:10B4E00001230023DBB21946F869FEF768FF786292
:10B4F0007AE0BB69DBB21946F869FFF74EFA786269
:10B5000072E0BB69DBB21946F869FFF701FC7862AB
:10B510006AE007F1160207F117031946F869FFF709
:10B520009BFC78627B6A002B59D1BB6C092B08D13C
:10B53000BB69DBB2BA7D1946F869FFF73EFC786259
:10B5400052E0FB7DBA69D2B21946F869FFF735FCC3
:10B55000786249E007F1140207F115031946F8690A
:10B56000FFF713FD78627B6A002B3AD1BB6C0B2B83
:10B5700008D1BB69DBB23A7D1946F869FFF7B0FC28
:10B58000786231E07B7DBA69D2B21946F869FFF77B
:10B59000A7FC786228E007F1120207F113031946AD
:10B5A000F869FFF77CFD78627B6A002B1BD1BB6CCE
:10B5B0000D2B08D1BB69DBB2BA7C1946F869FFF7DD
:10B5C00028FD786210E0FB7CBA69D2B21946F869AE
:10B5D000FFF71FFD786207E06FF015030AE000BF78
:10B5E00002E000BF00E000BF7B6A002B01D07B6A55
:10B5F00000E07B6818462837BD46BDE8B08F00BF25
:10B6000090B58DB000AFF860B9607A603B60002300
:10B610007B62FB683B623B6A1B68FB610023BB6289
:10B620003B6C032B02D06FF0150340E007F11702CB
:10B6300007F118031946F869FFF749FB78627B6A3E
:10B64000002B01D07B6A32E0002387F82F3028E0FE
:10B65000BA68BB6AD418BA6997F82F30DB00134474
:10B66000D3E900014FF47A724FF0000308F0FEF8BE
:10B6700002460B461346104A0C21204609F0AAFA4E
:10B6800003461A46BB6A1344BB62BA6A7B689A4295
:10B6900002D96FF006030AE097F82F30013387F8DC
:10B6A0002F30FB7D97F82F209A42D1D3BB6A1846E2
:10B6B0003437BD4690BD00BFD407021080B58AB0B4
:10B6C00002AFF860B9607A603B60FB68FB61FB69C0
:10B6D0001B68BB613B68DB78042B0BD107F11303BC
:10B6E0001946B869FEF7E2FE78617B69002B04D049
:10B6F0007B690DE06FF015030AE000BF07F113034B
:10B700000093012301227968B86800F063FC0346C6
:10B7100018462037BD4680BDB0B586B000AF786012
:10B7200039600821012003F049FF38613B69002B93
:10B7300002D16FF00B0343E03821012003F03EFFFC
:10B74000F860FB68002B36D0FB681F4A1C46154684
:10B750000FCD0FC40FCD0FC40FCD0FC495E803005C
:10B7600084E803003B69FA685A603A693B681B68E1
:10B7700019461046FEF7DCF978617B69002B15D17C
:10B780003B691B681846FEF7FDFB0346002B04D1FE
:10B790003B695B680D4ADA6003E03B695B680C4A11
:10B7A000DA607B683A691A60002309E000BFF86834
:10B7B00003F012FF00E000BF386903F00DFF7B6962
:10B7C00018461837BD46B0BD4C0400206C0200205E
:10B7D0002003002080B584B000AF78607B68002B28
:10B7E00001D1002313E07B681B681846FEF782FB3B
:10B7F000F860FB68002B01D0FB6808E07B685B68A1
:10B80000184603F0E9FE786803F0E6FE00231846C8
:10B810001037BD4680BD80B584B000AF7860396018
:10B820007B68DB6E07F10C021146184603F04BFFF4
:10B83000FB68032B02D86FF00A0307E07B68DB6E1E
:10B8400004223968184604F0FDF8034618461037FC
:10B85000BD4680BD80B582B000AF786039607B683E
:10B86000DB6E39460422184604F0DBF8034618461E
:10B870000837BD4680BD80B586B000AFF860B960BE
:10B880007A60FB681B687B617B695B6EFA68506855
:10B890007A68B9689847034618461837BD4680BD90
:10B8A00080B586B000AFF860B9607A60FB681B684D
:10B8B0007B617B699B6EFA6850687A68B9689847C3
:10B8C000034618461837BD4680BD000080B584B0D9
:10B8D00002AF786039603B6893F82130002B0FD0BD
:10B8E0003B681B791A46264B53F822203B68DB68DD
:10B8F000244951F823302449786809F0AFF93AE037
:10B900003B6893F82230002B2AD03B6893F8233011
:10B91000002B18D03B681B791A46194B53F822109C
:10B920003B6898683B681B791A46154B53F82230E0
:10B930003A68D2680192009303460A461349786830
:10B9400009F08CF917E03B681B791A460C4B53F849
:10B9500022203B689B680E49786809F07FF90AE06D
:10B960003B681B791A46064B53F822301A460949A0
:10B97000786809F073F900BF0837BD4680BD00BF85
:10B98000040C0210440C0210400902104809021075
:10B99000540902105C09021080B596B000AFF8603F
:10B9A000B9601346FB710023A7F8563036E0BB6838
:10B9B0009968B7F956201346DB0013449B00CA1858
:10B9C00007F1140311461846FFF780FF07F114032F
:10B9D0001946F86809F0E4FB0346002B17D1BB6851
:10B9E0009968B7F956201346DB0013449B000B44BB
:10B9F00093F82030FA799A4209D1BB689968B7F96F
:10BA000056201346DB0013449B000B440DE0B7F9AE
:10BA100056309BB201339BB2A7F85630B7F9563077
:10BA2000BA6892889342C2DB002318465837BD4655
:10BA300080BD80B584B000AF786039600023FB60C2
:10BA400018E07B681A6DFB68B02101FB03F3134417
:10BA50003968184609F0A4FB0346002B07D17B6820
:10BA60001A6DFB68B02101FB03F3134408E0FB6887
:10BA70000133FB607B685B6DFA689A42E1D3002377
:10BA800018461037BD4680BD80B584B000AF7860E1
:10BA900039600023FB601AE07B68996DFA681346F1
:10BAA0009B0013441B010B443968184609F078FBCE
:10BAB0000346002B08D17B68996DFA6813469B00FA
:10BAC00013441B010B4408E0FB680133FB607B68F7
:10BAD000DB6DFA689A42DFD3002318461037BD4663
:10BAE00080BD80B586B000AFF860B9607A60FB6851
:10BAF0001B687B61B9687869FFF79BFF0346002BE1
:10BB000002D16FF0120306E07B68012B02D06FF0C8
:10BB1000150300E0002318461837BD4680BD80B4E9
:10BB200083B000AF786039606FF0150318460C37AA
:10BB3000BD465DF8047B704780B483B000AF786089
:10BB400039606FF0150318460C37BD465DF8047B6D
:10BB50007047F0B589B002AFF860B9607A60FB70E9
:10BB60000023FB8216E0B7F9162013469B0013440E
:10BB70009B001A46BB6813441B681946786809F095
:10BB80000FFB0346002B12D0B7F916309BB20133DE
:10BB90009BB2FB82B7F9162013469B0013449B000F
:10BBA0001A46BB6813441B68002BDCD100E000BFC1
:10BBB000B7F9162013469B0013449B001A46BB6836
:10BBC00013441B68002B02D16FF0010363E0FB7884
:10BBD000002B30D0B7F9162013469B0013449B006E
:10BBE0001A46BB6813441B69002B02D16FF0010396
:10BBF00051E0B7F9162013469B0013449B001A46E8
:10BC0000BB6813441C69FB681868FB685968FB68CB
:10BC10009D68FB68DE68B7F9162013469B00134445
:10BC20009B001A46BB6813445B68009333462A4660
:10BC3000A04703462FE0B7F9162013469B00134494
:10BC40009B001A46BB681344DB68002B02D16FF0DF
:10BC5000010320E0B7F9162013469B0013449B0014
:10BC60001A46BB681344DC68FB681868FB685968AF
:10BC7000FB689D68FB68DE68B7F9162013469B00D9
:10BC800013449B001A46BB6813445B680093334619
:10BC90002A46A047034618461C37BD46F0BD0000A3
:10BCA00080B586B000AFF860B9607A6000233B6170
:10BCB000FB685B6D1B6BFA68506CFA68116D07F1DD
:10BCC0001002984778617B69002B01DA7B6906E0F6
:10BCD0003B69054A7968B86808F07CFF0346184656
:10BCE0001837BD4680BD00BF6009021080B588B01E
:10BCF00000AFF860B9607A6007F1100307F1140231
:10BD00001749B86808F0CAFF0346FB61FB69022BBC
:10BD10000DD1FB685B6D5B6BFA68506C79693A69B1
:10BD20009847B861BB69002B15DABB6914E007F1CD
:10BD300014031A460B49B86808F0B0FF0346FB61CC
:10BD4000FB69012B04D17A69FB681A657B6803E003
:10BD50006FF0150300E07B6818462037BD4680BDB4
:10BD6000640902106009021080B586B000AFF86067
:10BD7000B9607A60FB701E49F86809F009F97861CA
:10BD80007B69002B02D16FF015032CE0002200210B
:10BD9000786908F03BFC0246BB681A60FB78002B10
:10BDA0000DD01449002009F0F3F878617B69002B6D
:10BDB0000AD11149002009F0EBF8786104E00F493D
:10BDC000002009F0E5F878617B69002B02D16FF063
:10BDD000150308E00A220021786908F017FC0246E2
:10BDE0007B681A60002318461837BD4680BD00BF27
:10BDF0007009021074090210780902107C090210FF
:10BE000080B485B000AF786039607B68FB601DE06E
:10BE1000FB68174A82FB03129210DB17D31AFB60F0
:10BE20003B68134A82FB03129210DB17D31A3B6064
:10BE3000FB68002B11D03B68012B07DC7B680C4AA8
:10BE400082FB03129210DB17D31A7B603B68002B36
:10BE5000DED1FB68002BDBD100E000BF7B683A68D5
:10BE600002FB03F318461437BD465DF8047B7047A8
:10BE70006766666680B588B000AFF8607A603B6040
:10BE80000B46FB720023FB6100237B61FB7A013BC5
:10BE90000B2B00F2838001A252F823F0CDBE0010DC
:10BEA00009BF001035BF0010DDBE00109DBF00109F
:10BEB0009DBF00109DBF00109DBF00109DBF0010D2
:10BEC00061BF00109DBF00107DBF00100022002147
:10BED000F86808F09BFB0346BB6163E007F11402BE
:10BEE00007F118010123F868FFF73EFFF861FB69CD
:10BEF000002B01DAFB6962E07B6933491846FFF7E2
:10BF00007FFF03467B614DE007F1140207F1180142
:10BF10000023F868FFF728FFF861FB69002B01DABE
:10BF2000FB694CE07B6928491846FFF769FF034627
:10BF30007B6137E007F1140207F118010023F8686C
:10BF4000FFF712FFF861FB69002B01DAFB6936E0AD
:10BF50007B691E491846FFF753FF03467B6121E0CA
:10BF600007F1140207F118010023F868FFF7FCFE3F
:10BF7000F861FB69002B14DAFB6920E007F1130379
:10BF80001A461349F86808F089FE0346012B02D0CF
:10BF90006FF0150313E0FB7CBB6103E06FF015034A
:10BFA0000DE000BF7B68002B02D0BA697B681A6085
:10BFB0003B68002B02D07A693B681A60FB6918461F
:10BFC0002037BD4680BD00BF40420F0000CA9A3BEB
:10BFD000800902102DE9B04F98B002AF7863396341
:10BFE000BB62134687F82F30002387F857300023B1
:10BFF0003B650023FB6497F82F30013B0B2B00F2CD
:10C000005B8101A252F823F039C0001051C000102A
:10C010007FC000104BC0001095C20010B9C20010C4
:10C02000B9C20010B9C20010B9C200109BC0001004
:10C030003BC10010A5C20010BB6F1B68A14A396B41
:10C04000786B08F0C7FD034637E1012387F85730C6
:10C05000BB6F1A68BB6F04331B68194697F85730DB
:10C06000002B01D0984B00E0984B019300911346B0
:10C07000974A396B786B08F0ADFD03461DE1BB6F45
:10C080001A68BB6F04331B6800931346914A396BDF
:10C09000786B08F09FFD03460FE1BB6F1B68DA1752
:10C0A0003B617A618C4BD7E904452A4603FB02F2D7
:10C0B0000023214601FB03F31344874A2146A1FBD9
:10C0C0000212FA610A46BA61FA691344FB61BB6F56
:10C0D00004331B681A46D7E9060104F025FDC7E9B9
:10C0E0001001BB6F5B68BB6307F138037A4AD7E97D
:10C0F000100104F0F3FC02460B461346FB63FB6B96
:10C10000002B0DD1BB6B002B0ADABB6B002BB8BF29
:10C110005B42724A396B786B08F05CFD0346CCE0F9
:10C12000BB6B002BB8BF5B420093FB6B6C4A396B57
:10C13000786B08F04FFD0346BFE0BB6F1B68002B18
:10C140003ADABB6F1B68DA17BB60FA60654BD7E958
:10C1500002AB5A4603FB02F24FF0FF33514601FB9C
:10C1600003F313445F4A5146A1FB02127A620A4666
:10C170003A627A6A13447B62BB6F04331B68C3F173
:10C180002001B3F12002D7E908AB504620FA03F8AA
:10C19000584600FA01F148EA010804D4594641FA28
:10C1A00002F248EA02087A6A42FA03F90023D8F157
:10C1B000000463EB090528E0BB6F1B68DA173B60DE
:10C1C0007A60454BD7E900894A4603FB02F2002317
:10C1D000414601FB03F313443F4A4146A1FB02AB36
:10C1E0005B449B46BB6F04331B68C3F12001B3F172
:10C1F00020022AFA03F40BFA01F144EA010402D402
:10C200004BFA02F214434BFA03F5C7E9104507F164
:10C210003803314AD7E9100104F060FC02460B46AE
:10C220001346FB63FB6B002B0DD1BB6B002B0ADAB3
:10C23000BB6B002BB8BF5B42284A396B786B08F0A8
:10C24000C9FC034639E0BB6B002BB8BF5B420093CF
:10C25000FB6B234A396B786B08F0BCFC03462CE07F
:10C260007A6BFB6CD0183A6BFB6CD11A3B6D9B0060
:10C27000BA6F13441B681C4A08F0ACFC03461A460C
:10C28000FB6C1344FB64FA6C3B6B9A4207D23B6D28
:10C2900001333B653A6DBB6A9A42E1DB00E000BFC7
:10C2A000FB6C0AE0BB6F1B68DBB2104A396B786B22
:10C2B00008F090FC034600E0002318465837BD46BE
:10C2C000BDE8B08F84090210880902108C090210A1
:10C2D000900902109C09021000CA9A3BA80902109A
:10C2E000B0090210003665C4BC09021080090210B2
:10C2F00080B485B000AF0346B9607A60FB73FB7B06
:10C30000042B1CD801A252F823F000BF21C3001057
:10C3100031C3001039C3001039C3001029C3001005
:10C32000BB685B6D1B690BE0BB685B6DDB6807E09E
:10C33000BB685B6D5B6903E07B68DB6900E0002341
:10C3400018461437BD465DF8047B704780B483B04F
:10C3500000AF03463960FB71FB79042B03D13B68C6
:10C360009B6C5B6801E000BF002318460C37BD469C
:10C370005DF8047B7047000080B590B000AFF860B6
:10C38000B9607A603B600023FB63FB681B68B96897
:10C390001846FFF74EFBB863BB6B002B00F08480A0
:10C3A0007B681B78002B17D17B685B685A4918465D
:10C3B00008F0F6FE0346002B0ED1BB6B5B6D1B6BCA
:10C3C000002B06D0BA6C3968B86BFFF769FC0346DE
:10C3D0009DE06FF001039AE07B689B681B78002B5F
:10C3E0003AD07B681B78022B0CBF01230023DBB201
:10C3F00087F82F307B689868BB6B596D97F92F30A1
:10C40000002B14BF01230023DBB21A46FFF7C4FA46
:10C41000F863FB6B002B02D16FF0010377E097F913
:10C420002F30002B14BF01230023DBB287F822300A
:10C43000FB6B9B681BB23B84FB6B1B7987F823303B
:10C44000FB6B93F8233087F82430FB6B1B69BB62CE
:10C4500007F12003FB6101E00023FB613B687B6186
:10C46000BB6CBB61BB6B5B6C3B617B681B78FA6B25
:10C47000B96B1846FFF73CFF38637B685B681B7835
:10C48000002B07D107F11003396B1846FFF747FB64
:10C4900003463CE07B685A6807F110000023396BC3
:10C4A000FFF757FB034632E0FB681B68B968184684
:10C4B000FFF7EAFA78637B6B002B26D00023FB6141
:10C4C0003B687B61BB6CBB617B6B5B6C3B617B687E
:10C4D0001B78796B1846FFF739FF38637B685B6818
:10C4E0001B78002B07D107F11003396B1846FFF7B3
:10C4F00016FB03460BE07B685A6807F11000002327
:10C50000396BFFF726FB034601E06FF01203184674
:10C510004037BD4680BD00BFC409021080B590B051
:10C5200000AFF860B9607A603B600023FB63FB6892
:10C530001B68B9681846FFF77CFAB863BB6B002B21
:10C5400000F081807B681B78002B17D17B685B68CB
:10C550005849184608F024FE0346002B0ED1BB6B49
:10C560005B6D5B6B002B06D0BA6C3968B86BFFF75C
:10C57000BDFB03469AE06FF0010397E07B689B6880
:10C580001B78002B37D07B681B78022B0CBF012354
:10C590000023DBB287F82F307B689868BB6B596D3E
:10C5A00097F92F30002B14BF01230023DBB21A466A
:10C5B000FFF7F2F9F863FB6B002B02D16FF0010378
:10C5C00074E097F92F30002B14BF01230023DBB256
:10C5D000BB74FB6B9B681BB23B82FB6B1B79FB74D0
:10C5E000FB6B93F823303B75FB6B1B69BB6107F159
:10C5F0001003BB6201E00023BB623B683B62BB6C83
:10C600007B62BB6B5B6CFB617B681B78FA6BB96B05
:10C610001846FFF76DFE38637B685B681B78002B5C
:10C6200007D107F11C03396B1846FFF785FA03465B
:10C630003CE07B685A6807F11C000123396BFFF767
:10C6400088FA034632E0FB681B68B9681846FFF7B2
:10C650001BFA78637B6B002B26D00023BB623B6800
:10C660003B62BB6C7B627B6B5B6CFB617B681B78AA
:10C67000796B1846FFF76AFE38637B685B681B7846
:10C68000002B07D107F11C03396B1846FFF747FA57
:10C6900003460BE07B685A6807F11C000123396BE5
:10C6A000FFF757FA034601E06FF0120318464037D0
:10C6B000BD4680BDC409021080B584B000AF78606B
:10C6C00039603B68002B02D14FF0FF331DE000239F
:10C6D000FB6013E07B68996DFA6813469B00134476
:10C6E0001B010B443968184608F05AFD0346002B1D
:10C6F00001D1FB6809E0FB680133FB607B68DB6DFF
:10C70000FA689A42E6D34FF0FF3318461037BD4619
:10C7100080BD000080B588B000AFF860B9607A6075
:10C720003B60FB681B68FB61FB69DB6D002B02D182
:10C730006FF0010331E0B968F869FFF7A5F9B86156
:10C74000BB69002B02D06FF0010326E0B968F869DD
:10C75000FFF76FF978617B69002B02D16FF012034C
:10C760001BE07B69D3F8AC30B3F1FF3F04D17B68A9
:10C7700000221A70002310E0FB69996D7B69D3F8E1
:10C78000AC2013469B0013441B010B441B6C054A51
:10C790003968786808F01EFA034618462037BD4607
:10C7A00080BD00BF5C09021080B588B000AFF860A2
:10C7B000B9607A603B60FB681B68FB61FB69DB6DFD
:10C7C000002B02D16FF0010331E0B968F869FFF77F
:10C7D0005BF9B861BB69002B02D06FF0010326E062
:10C7E000B968F869FFF725F978617B69002B02D1F8
:10C7F0006FF012031BE07B681B78002B06D17B696E
:10C800004FF0FF32C3F8AC20002310E07968F869DC
:10C81000FFF752FF38613B69B3F1FF3F02D16FF080
:10C82000150304E07B693A69C3F8AC203B681846FD
:10C830002037BD4680BD80B584B000AF786000234E
:10C84000FB603CE07B681A6DFB68B02101FB03F3E1
:10C850001344BB60BB68D3F8AC30B3F1FF3F28D0C2
:10C860007B68996DBB68D3F8AC2013469B001344DA
:10C870001B010B4493F84C3083F00103DBB2002B17
:10C8800019D1BB685B6DDB6A002B15D0BB685B6D93
:10C89000DB6ABA684832104698477B68996DFA6837
:10C8A00013469B0013441B010B44002283F84C20C9
:10C8B00002E000BF00E000BFFB680133FB607B6863
:10C8C0005B6DFA689A42BDD300BF00BF1037BD460A
:10C8D00080BD80B485B000AF786039600023FB6014
:10C8E0000023BB601AE03B6803F00103002B0FD06C
:10C8F000BA681346DB0013449B001A467B68134456
:10C900009B699B78DB08DBB21A46FB681344FB602B
:10C910003B685B083B60BB680133BB603B68002B36
:10C92000E1D1FB6818461437BD465DF8047B7047BB
:10C9300080B58CB000AFF860B9607A603B60FB688E
:10C940001B68B9681846FFF774F838623B6A002B19
:10C9500002D16FF01203E5E03B6A93F8A83083F050
:10C960000103DBB2002B02D06FF01503DAE03B6A63
:10C970005B6D9B88C3F120034FF0FF3222FA03F373
:10C98000FB613A68FB6913403B603B68002B02D1B6
:10C990006FF00103C6E03B6A97F8382083F87020F7
:10C9A0003B6A00225A673B6A3A689A653B6A5B6D4C
:10C9B0009B6839681846FFF78CFF02463B6A1A6687
:10C9C0003B6A1B6E7A6803FB02F23B6ADA653B6ADC
:10C9D0007A685A663B6AD3F8A030002B22D03B6AB3
:10C9E000D3F8A430002B1DD03B6AD3F8A4203B6AB7
:10C9F000DB6D9A4202D26FF00B0393E03B6AD3F8EF
:10CA0000A4103B6AD3F8A4303A6AD26DB3FBF2F0BB
:10CA100000FB02F29B1ACB1A7B623B6AD3F8A03070
:10CA2000BB6221E03B6A93F8A930002B08D03B6A37
:10CA3000DB6F184602F0D0FD3B6A002283F8A92084
:10CA40003B6ADB6D7B623B6ADB6D0121184602F0BD
:10CA5000B5FDB862BB6A002B02D16FF00B0361E039
:10CA60003B6A012283F8A9203B6A78337A6AB96A63
:10CA7000184602F0BCFDF862FB6A002B0FDA3B6A35
:10CA800093F8A930002B08D03B6ADB6F184602F000
:10CA9000A3FD3B6A002283F8A920FB6A42E03B6ABF
:10CAA0005B6D1B6A002B1BD03B6A5B6D1B6A3A6A8D
:10CAB000526C396810469847F862FB6A002B0FDA0F
:10CAC0003B6A93F8A930002B08D03B6ADB6F18460D
:10CAD00002F082FD3B6A002283F8A920FB6A21E074
:10CAE000FB681B68BB613B6AD3F8AC30B3F1FF3F16
:10CAF00017D0BB69996D3B6AD3F8AC2013469B00F5
:10CB000013441B010B447B617B699B6C9B68002B6E
:10CB100007D07B699B6C9B687A69526C104698477A
:10CB2000F862FB6A18463037BD4680BD80B586B0D6
:10CB300000AF7860396000237B617B681B683968CF
:10CB40001846FEF776FF38613B69002B02D14FF0A3
:10CB5000FF334FE03B6993F8A83083F00103DBB269
:10CB6000002B02D06FF0150344E03B6993F8A93025
:10CB7000002B08D03B69DB6F184602F02DFD3B69A6
:10CB8000002283F8A9207B681B68FB603B69D3F80F
:10CB9000AC30B3F1FF3F1CD0FB68996D3B69D3F813
:10CBA000AC2013469B0013441B010B44BB60BB68C5
:10CBB0009B6CDB68002B0CD0BB689B6CDB68BA6895
:10CBC000526C1046984778617B69002B01D07B69D5
:10CBD00010E03B6900229A653B695B6D5B6A002B44
:10CBE00007D03B695B6D5B6A3A69526C10469847A7
:10CBF00078617B6918461837BD4680BD80B588B01E
:10CC000000AFF860B9601346FB71FB681B68B96838
:10CC10001846FEF70EFFB861BB69002B07D0BB6951
:10CC200093F8A83083F00103DBB2002B02D06FF041
:10CC3000150365E0BB69FA7983F86820BB695B6D11
:10CC40009B6A002B0ED0BB69D3F8AC30B3F1FF3F29
:10CC500008D1BB695B6D9B6ABA6948321046984738
:10CC600003464DE0FB79002B0AD1BB695B6D9B69E4
:10CC7000002B05D0BB69D3F8AC30B3F1FF3F0DD02A
:10CC8000FB79012B3BD1BB695B6DDB69002B36D097
:10CC9000BB69D3F8AC30B3F1FF3F30D1BB69583337
:10CCA0007B6107F110031946786900F0DAF8F86142
:10CCB000FB69002B01DAFB6922E0FB79002B0AD12A
:10CCC000BB695B6D9B69BA69506C39697A69D268D6
:10CCD0009847F86109E0BB695B6DDB69BA69506C24
:10CCE00039697A69D2689847F861FB69002B01DAE3
:10CCF000FB6905E0786900F0DCF8034600E00023FA
:10CD000018462037BD4680BD80B582B000AF786040
:10CD10003960012239687868FFF770FF03461846CA
:10CD20000837BD4680BD80B582B000AF78603960FD
:10CD3000002239687868FFF761FF03461846083714
:10CD4000BD4680BD80B588B000AFF860B9607A603C
:10CD50003B60FB681B68B9681846FEF76AFEF8611D
:10CD6000FB69002B07D0FB6993F8A83083F001031F
:10CD7000DBB2002B02D06FF0150327E0FB6978339C
:10CD800007F114021146184602F09DFCB861BB6918
:10CD9000002B01DABB6919E07B693A68934228BF2E
:10CDA00013463B603B68002B02D16FF00A030DE095
:10CDB000FB6978333A687968184602F043FEB86137
:10CDC000BB69002B01DABB6900E03B6818462037DD
:10CDD000BD4680BD80B588B000AFF860B9607A60AC
:10CDE0003B60FB681B68B9681846FEF722FEF861D5
:10CDF000FB69002B07D0FB6993F8A83083F001038F
:10CE0000DBB2002B02D06FF0150326E0FB6978330C
:10CE100007F110021146184602F055FCB861BB69D3
:10CE2000002B01DABB6918E0FB69DA6D3B69D31AA4
:10CE30007B613A687B69934228BF13463B60FB697C
:10CE400078333A687968184602F0EBFDB861BB693F
:10CE5000002B01DABB6900E03B6818462037BD466D
:10CE600080BD80B584B000AF786039607B68002BEE
:10CE700002D16FF0150318E07B681B7C002B0AD1F0
:10CE80007B6858697B68596807F10C033A6802F0BF
:10CE900086FD034609E07B6858697B68596807F19D
:10CEA0000C033A6802F08FFD034618461037BD4662
:10CEB00080BD80B582B000AF78607B68002B02D166
:10CEC0006FF0150310E07B681B7C002B06D17B689C
:10CED0005B69184602F08BFD034605E07B685B69E1
:10CEE000184602F091FD034618460837BD4680BD3E
:10CEF00080B588B000AF78607868FFF79CFC07F1D8
:10CF00000C0319467868FEF786FCF861FB69002B74
:10CF100001DAFB6911E07B681B68FA681146184664
:10CF200002F000FBF861FB6913F1800F04D0FB688D
:10CF300019467868FEF78EFCFB6918462037BD4617
:10CF400080BD000080B596B000AFF860B9607A602F
:10CF50007B68B3F1FF3F02D10023FB6401E07B68F3
:10CF6000FB64BB68002B02D107F11403BB600023F4
:10CF70007B65FB689B6CBB64BB6C002B35D00023CE
:10CF80003B652CE07B6DBA68D018FA6C7B6DD31AC8
:10CF900023EAE37319463B6DDB00BA6C13441B684C
:10CFA000144A07F017FE02467B6D13447B657B6DC8
:10CFB000BA68D018FA6C7B6DD31A23EAE37319466A
:10CFC0003B6DDB00BA6C13445B680B4A07F002FE52
:10CFD00002467B6D13447B653B6D01333B65FB680B
:10CFE000DB6C1A463B6D9342CCDB7B6D18465837A1
:10CFF000BD4680BDD8090210F8090210F0B59FB0F7
:10D0000006AFF860B9607A603B60BB6FB3F1FF3F79
:10D0100002D100233B6501E0BB6F3B653B68002B01
:10D0200002D107F114033B600023FB65FB6D3A68F6
:10D03000D0183A6DFB6DD31A23EAE3731946BB6827
:10D0400000937B68A14A07F0C5FD0246FB6D1344BF
:10D05000FB65FB689B68002B00F06C820023BB65BE
:10D0600061E2FB689968BA6D1346DB0013449B00CC
:10D070000B44FB6407F11403F96C1846FEF726FC19
:10D08000FB6D3A68D0183A6DFB6DD31A23EAE3734F
:10D09000194607F114038E4A07F09CFD0246FB6D0A
:10D0A0001344FB65FB6C1B68002B11D0FB6D3A68C9
:10D0B000D0183A6DFB6DD31A23EAE3731946FB6C63
:10D0C0001B68844A07F086FD0246FB6D1344FB652E
:10D0D000FB6D3A68D0183A6DFB6DD31A23EAE373FF
:10D0E0001946FB6C93F82030002B01D07A4B00E0FE
:10D0F0007A4B7B4A07F06EFD0246FB6D1344FB65DD
:10D10000FB6C9B69002B2FD0FB6D3A68D0183A6DF1
:10D11000FB6DD31A23EAE3739C46FB6C5969FB6CE5
:10D120009B691B79002B01D06E4B00E06E4BFA6CB3
:10D13000926912781446FA6C926952781546FA6C24
:10D14000926992781646FA6C9269D27804920396A4
:10D150000295019400930B46644A614607F03AFD3C
:10D160000246FB6D1344FB65FB6CDB69002B00F092
:10D17000C78100237B65B7E1FB6CD9697A6D1346E3
:10D180009B0013449B000B44BB64FB6D3A68D018B2
:10D190003A6DFB6DD31A23EAE3731946BB6C1B6827
:10D1A000534A07F017FD0246FB6D1344FB65FB6C09
:10D1B00093F82330002B00F0CC80BB6C1B7A032B40
:10D1C00000F27F8101A252F823F000BF95D2001037
:10D1D0003DD2001003D20010DDD10010FB6D3A6883
:10D1E000D0183A6DFB6DD31A23EAE3731946BB6C72
:10D1F0001B68404A07F0EEFC0246FB6D1344FB65DA
:10D200005FE1FB6D3A68D0183A6DFB6DD31A23EAE3
:10D21000E3731946FB6C93F82030002B01D0364A9B
:10D2200000E0364ABB6C1B6800931346344A07F093
:10D23000D1FC0246FB6D1344FB6542E1FB6D3A688D
:10D24000D0183A6DFB6DD31A23EAE3731D46FB6CCD
:10D2500093F82030002B01D0274C00E0274CFB6CCA
:10D260001B791A46274B53F82230FA6C1279114673
:10D27000244A52F82120B96C096802910192009366
:10D280002346214A294607F0A5FC0246FB6D1344BC
:10D29000FB6516E1FB6C93F8223083F00103DBB2EF
:10D2A000002B02D06FF015030FE2FB6D3A68D51822
:10D2B0003A6DFB6DD31A23EAE3739C46FB6C93F83B
:10D2C0002030002B22D00C4E21E000BF080A0210B3
:10D2D000240A0210380A0210440A02104C0A0210F2
:10D2E000540A0210640A0210680A02106C0A021042
:10D2F000A00A0210B80A0210C80A0210CC0A0210D2
:10D30000D00A0210040C0210E40A02108D4EFB6CCD
:10D310001B791A468C4B53F82230FA6C9268F96CE0
:10D3200009790846884951F82010F86CC068BC6C2F
:10D330002468049403900291019200933346834A37
:10D340006146284607F046FC0246FB6D1344FB6528
:10D35000B7E0BB6C1B7A032B00F2B38001A252F83A
:10D3600023F000BF1FD40010D5D300109BD30010B2
:10D3700075D30010FB6D3A68D0183A6DFB6DD31A67
:10D3800023EAE3731946BB6C1B68714A07F022FC61
:10D390000246FB6D1344FB6593E0FB6D3A68D018C1
:10D3A0003A6DFB6DD31A23EAE3731946FB6C93F8CD
:10D3B0002030002B01D0674A00E0624ABB6C1B683A
:10D3C00000931346644A07F005FC0246FB6D1344C4
:10D3D000FB6576E0FB6D3A68D0183A6DFB6DD31AA9
:10D3E00023EAE3731C46FB6C93F82030002B01D03A
:10D3F000584900E05349FB6C1B791A46524B53F8CD
:10D400002230BA6C1268019200930B46534A2146AF
:10D4100007F0E0FB0246FB6D1344FB6551E0FB6C3B
:10D4200093F82230002B27D0FB6D3A68D0183A6D64
:10D43000FB6DD31A23EAE3731D46FB6C93F820308F
:10D44000002B01D0434C00E03E4CFB6C1B791A468C
:10D450003D4B53F82230FA6C9268B96C096802911E
:10D460000192009323463E4A294607F0B3FB024649
:10D47000FB6D1344FB6523E0FB6D3A68D0183A6DF1
:10D48000FB6DD31A23EAE3731C46FB6C93F8203040
:10D49000002B01D02F4900E02A49FB6C1B791A466A
:10D4A000294B53F82230BA6C1268019200930B4654
:10D4B0002A4A214607F08EFB0246FB6D1344FB65AA
:10D4C00000BFFB6D3A68D0183A6DFB6DD31A23EAA2
:10D4D000E373244A194607F07DFB0246FB6D1344B3
:10D4E000FB657B6D01337B65FB6CD9697A6D1346F7
:10D4F0009B0013449B000B441B68002B7FF43CAE45
:10D50000FB6D3A68D0183A6DFB6DD31A23EAE373CA
:10D51000154A194607F05EFB0246FB6D1344FB6596
:10D52000BB6D0133BB65FB689B881A46BB6D93429C
:10D53000FFF697ADFB68DB68002B3FD00023BB658F
:10D5400031E000BFCC0A0210040C0210FC0A0210E9
:10D55000B80A0210C80A0210D00A0210180B0210F2
:10D560002C0B0210440B0210480B0210FB6D3A68A2
:10D57000D0183A6DFB6DD31A23EAE3731C46FB689F
:10D58000D968BA6D13469B0013449B000B441B687B
:10D59000504A214607F01EFB0246FB6D1344FB6513
:10D5A000BB6D0133BB65FB68D968BA6D13469B0040
:10D5B00013449B000B441B68002BD7D1FB681B69ED
:10D5C000002B2AD00023BB651CE0FB6D3A68D01805
:10D5D0003A6DFB6DD31A23EAE3731C46FB681969A5
:10D5E000BA6D13469B0013449B000B441B683A4AD8
:10D5F000214607F0EFFA0246FB6D1344FB65BB6D55
:10D600000133BB65FB681969BA6D13469B0013446F
:10D610009B000B441B68002BD7D1FB681B6B002BB6
:10D6200003D1FB685B6B002B0FD0FB6D3A68D01801
:10D630003A6DFB6DD31A23EAE373284A194607F0C3
:10D64000C9FA0246FB6D1344FB65FB685B69002B5E
:10D650002AD00023BB651CE0FB6D3A68D0183A6DF8
:10D66000FB6DD31A23EAE3731C46FB685969BA6D54
:10D6700013469B0013449B000B441B68184A214629
:10D6800007F0A8FA0246FB6D1344FB65BB6D01333E
:10D69000BB65FB685969BA6D13469B0013449B0038
:10D6A0000B441B68002BD7D1FB6D3A68D0183A6D3C
:10D6B000FB6DD31A23EAE3730A4A194607F08AFA84
:10D6C0000246FB6D1344FB65FB6D18466437BD468F
:10D6D000F0BD00BF540B02106C0B02108C0B02103B
:10D6E000BC0B0210DC0B0210B0B598B002AF786032
:10D6F00007F10C0338220021184607F0C3FB40F263
:10D70000F5333B654FF0FF3200217868FFF71AFCD4
:10D7100002463B6D13443B6500237B6519E07B6843
:10D720001A6D7B6DB02101FB03F313447B647B6CAA
:10D73000586D7B6C196C7A6C4FF0FF3300930023AB
:10D74000FFF75CFC02463B6D13443B657B6D013388
:10D750007B657B685B6D7A6D9A42E0D300237B65C5
:10D760001EE07B68996D7A6D13469B0013441B0184
:10D770000B44BB64BB6C9B6C5B68BB61BB6C196C82
:10D78000BA6C07F10C004FF0FF3300930023FFF752
:10D7900035FC02463B6D13443B657B6D01337B6575
:10D7A0007B68DB6D7A6D9A42DBD33B6D01330121DF
:10D7B000184601F003FF02467B681A647B681B6C05
:10D7C000002B02D16FF00B0378E07B683A6D5A644E
:10D7D0007B681B6C3B49184607F052FE40F2EB3366
:10D7E000FB647B681A6CFB6CD1183A6DFB6CD31A26
:10D7F0001A467868FFF7A6FB0246FB6C1344FB64ED
:10D8000000237B651FE07B681A6D7B6DB02101FBF7
:10D8100003F313447B647B6C586D7B6C196C7C6CDC
:10D820007B681A6CFB6CD5183A6DFB6CD31A0093AD
:10D830002B462246FFF7E2FB0246FB6C1344FB64D7
:10D840007B6D01337B657B685B6D7A6D9A42DAD3C1
:10D8500000237B6524E07B68996D7A6D13469B00FD
:10D8600013441B010B44BB64BB6C9B6C5B68BB61CA
:10D87000BB6C196CBC6C7B681A6CFB6CD5183A6D70
:10D88000FB6CD31A07F10C0000932B462246FFF7DE
:10D89000B5FB0246FB6C1344FB647B6D01337B6577
:10D8A0007B68DB6D7A6D9A42D5D37B681A6CFB6C12
:10D8B00013440549184607F0E3FD0023184658377E
:10D8C000BD46B0BD840400207008002080B588B03B
:10D8D00000AFF860B9607A60FB687A685A65FB68E7
:10D8E0005B6DB021184601F069FE0246FB681A65BF
:10D8F000FB681B6D002B02D16FF00B036CE0002363
:10D90000FB6164E0FA6913465B001344DB001A46CE
:10D91000BB681344BB61FB681A6DFB69B02101FB56
:10D9200003F313447B61BB699A687B695A657B6921
:10D93000FA692B49184607F091F9BB695B691946EA
:10D94000F868FEF7B9FE02467B69C3F8AC20BB69F4
:10D950005A687B695A64BB695A687B699A647B69B7
:10D9600003F158027B69DA64BB691A687B691A643F
:10D97000BB699B689B69002B0ED1BB699B68DB6907
:10D98000002B09D1BB699B689B6A002B04D1BB6942
:10D990009B68DB6A002B13D0BB69DA687B69C3F82C
:10D9A000A020BB691A697B69C3F8A4207B6903F1D5
:10D9B00078027B69DA667B69012283F8A82003E09C
:10D9C0007B69002283F8A820FB690133FB61FA69B7
:10D9D0007B689A4296D3002318462037BD4680BD07
:10D9E000E80B021080B588B000AFF860B9607A60CB
:10D9F000FB687A68DA65FB68DB6D5021184601F038
:10DA0000DDFD0246FB689A65FB689B6D002B02D129
:10DA10006FF00B032EE00023FB6126E0FA6913464A
:10DA20005B0013449B001A46BB681344BB61FB6850
:10DA3000996DFA6913469B0013441B010B447B61EB
:10DA4000BB695A687B695A64BB691A687B691A6446
:10DA5000BB699A687B699A647B69FA6907491846C9
:10DA600007F0FCF8FB690133FB61FA697B689A42B5
:10DA7000D4D3002318462037BD4680BDF80B0210D2
:10DA800080B590B000AF786039607B68002B02D021
:10DA90003B68002B02D16FF0150304E170210120D7
:10DAA00001F08CFDB863BB6B002B02D16FF00B0350
:10DAB000F9E03B68DA68BB6B9A643B681A69BB6B38
:10DAC000DA643B68D9693B681B6A1A46B86BFFF792
:10DAD00089FFF863FB6B002BC0F2D9803B68596962
:10DAE0003B689B691A46B86BFFF7F0FEF863FB6B67
:10DAF000002BC0F2D380B86BFFF7F6FDF863FB6B29
:10DB0000002BC0F2BD80BB6B04337B637B6B684A28
:10DB10001A627B6B674A5A627B6B674A9A627B6BBD
:10DB2000664ADA627B6B664A1A617B6B654A9A6168
:10DB30007B6B654A5A617B6B644ADA617B6B644A32
:10DB40009A607B6B634ADA607B6B634A1A607B6B1B
:10DB5000624A5A607B6B624A5A63BB6BBB627B6BE7
:10DB60007B62BB6B1B6CFB62BB6B5B6C3B63BB6B1D
:10DB700007F124021146184600F0BCFEF863FB6B67
:10DB8000002B76DBBB6B6C332C21184601F04BFD70
:10DB9000F863FB6B002B65DB3B681B78002B24D103
:10DBA000BB6B504A9A66BB6B4F4A5A663B685A68D1
:10DBB000BB6B1A66BB6B1B6E7B614C4BBB614FF43E
:10DBC0008053FB61BB6B1B6807F1200207F1140156
:10DBD000184600F019FFF863FB6B002B39DB3B6A3A
:10DBE0001946B86BFDF736FE2EE03B681B78012B1B
:10DBF00026D13B689B681A68BB6B5A663B689B687A
:10DC00005A68BB6B9A660023BB603B689B689B6845
:10DC1000FB603B689B68DB683B61BB6B1B6807F183
:10DC2000200207F10801184600F0EEFEF863FB6BD6
:10DC3000002B10DB3B6A1946B86BFDF70BFE03E0C7
:10DC40006FF01503FB6307E07B68BA6B1A60002373
:10DC500029E000BF00E000BFBB6BDB6E184601F09F
:10DC600017FD00E000BFBB6B1B68184600F091FE7B
:10DC700000E000BFBB6B1B6C184601F0ADFC00E080
:10DC800000BFBB6B9B6D184601F0A6FC00E000BF17
:10DC9000BB6B1B6D184601F09FFC00E000BFB86B2A
:10DCA00001F09AFCFB6B18464037BD4680BD00BFB3
:10DCB00079C300101DC5001015C70010A9C70010BA
:10DCC00045CD0010D5CD001027CD001009CD001096
:10DCD00031C900102DCB0010A1B8001077B800108A
:10DCE000E3BA0010BD5A0010595A0010701A0020F3
:10DCF00080B582B000AF78607B68002B02D16FF0F6
:10DD000015031CE07B68DB6E184601F0C1FC7B68E4
:10DD10001B68184600F03DFE7B681B6D184601F03D
:10DD20005BFC7B689B6D184601F056FC7B681B6CA6
:10DD3000184601F051FC786801F04EFC00231846AB
:10DD40000837BD4680BD000080B485B000AF786064
:10DD500039607B684FF4FA5202FB03F3094AA2FBD5
:10DD600003231B0CFB60FB68074AA2FB0323DB08B1
:10DD7000FA681344FB60FB6818461437BD465DF82B
:10DD8000047B7047C5B3A291CDCCCCCC80B586B016
:10DD900000AFF860B9607A603B60FB681B683A6866
:10DDA00079681846F7F78AFE78617B69002B01DAFB
:10DDB0007B6913E03B684FF4E1311846FFF7C4FF7D
:10DDC00038613869F9F717FBFB681B681846F7F7E5
:10DDD00015FEB968F868F7F7CDFD03461846183701
:10DDE000BD4680BDB0B5ADF5127D02AF07F510732D
:10DDF000A3F50F73186007F51073A3F5107319607E
:10DE0000314B07F50A741D460FCD0FC42B682360F4
:10DE10002E4B07F505741D460FCD0FC42B682360EC
:10DE20002B4A07F5037392E8030083E8030007F524
:10DE30001073A3F510731B68D96807F51073A3F569
:10DE400010731B681B7C9B0003F510733B4453F855
:10DE5000184C07F51073A3F510731B685B7C9B00CF
:10DE600003F510733B4453F82C2C07F51073A3F5FE
:10DE700010731B689B7C9B0003F510733B4453F8A5
:10DE8000343C07F10C000193009223460A461149E5
:10DE900006F0E4FE0346C7F83C32D7F83C3207F1FF
:10DEA0000C0207F51071A1F5107107F51070A0F5BF
:10DEB0000F7009680068FFF769FF0346184607F509
:10DEC0001077BD46B0BD00BFC00D0210F80D0210A6
:10DED000140E0210640C021080B5ADF5067D00AF83
:10DEE00007F50673A3F50373186007F50673A3F52A
:10DEF0000473196007F50673A3F505731A6007F537
:10DF00000673A3F5057307F114001A680D4906F0AE
:10DF1000A5FE0346C7F81432D7F8143207F11402ED
:10DF200007F50671A1F5047107F50670A0F50370F9
:10DF300009680068FFF72AFF0346184607F50677C9
:10DF4000BD4680BD1C0E021080B58AB000AF78605F
:10DF500039603B681B783B733B685B683B6101231E
:10DF60003B754FF4E133BB6103233B7700237B77A1
:10DF70000023BB773B685B693B623B689B697B62C4
:10DF800007F10C0319467868F7F7F4FC03461846C6
:10DF90002837BD4680BD84B080B592B000AF7860B0
:10DFA00007F1540080E80E00D7F88830FB63142195
:10DFB000012001F003FBB863BB6B002B02D16FF0B3
:10DFC0000B0314E1D7F88C20BB6BDA60D7F89020F4
:10DFD000BB6B1A6107F1540303F1180207F1080340
:10DFE00011461846FFF7B0FF38643B6C002BC0F2B7
:10DFF000EA8007F1540303F1180207F10803114600
:10E000001846FFF7EFFE38643B6C002BC0F2CD8062
:10E01000BA68BB6B1A6000233B73BB683B613B6E05
:10E020001821184601F0CAFA78637B6B002B03D1E4
:10E030006FF00B033B64BBE000237B6490E0F96D61
:10E040007A6C13465B001344DB0019447A6C134668
:10E050005B001344DB001A467B6B13440A681A60AA
:10E06000F96D7A6C13465B001344DB0019447A6C3B
:10E0700013465B001344DB001A467B6B13444A686B
:10E080005A60F96D7A6C13465B001344DB00194447
:10E090007A6C13465B001344DB001A467B6B134417
:10E0A0008A689A60F96D7A6C13465B001344DB0052
:10E0B00019447A6C13465B001344DB001A467B6BF1
:10E0C00013444A695A61F96D7A6C13465B00134434
:10E0D000DB000B44DB68002B08D0F96D7A6C13462B
:10E0E0005B001344DB000B44DB6807E0F96D7A6CDE
:10E0F00013465B001344DB000B441B693B633B6B23
:10E10000002B16D07A6C13465B001344DB001A46D2
:10E110007B6B13443A6B5268DA607A6C13465B008F
:10E120001344DB001A467B6B13443A6B12681A6186
:10E1300013E07A6C13465B001344DB001A467B6BDA
:10E1400013440022DA607A6C13465B001344DB0050
:10E150001A467B6B134400221A617B6C01337B648B
:10E160003B6E7A6C9A42FFF46AAF7B6B3B623B6E0C
:10E170007B627B6EBB62BB6EFB627B6DBB61BB6D0A
:10E18000FB61BB6B083307F10C0211461846FFF721
:10E1900077FC38643B6C002B09DB786B01F01CFAD0
:10E1A0007B68BA6B1A60002321E000BF00E000BF6B
:10E1B00007F1540303F1180207F10803114618464A
:10E1C000FFF7C2FE00E000BFB86B01F005FA07F1EF
:10E1D000540303F1180107F108033A6C1846FFF7DE
:10E1E0007BFE3864BB681846F7F708FC3B6C1846A2
:10E1F0004837BD46BDE8804004B0704780B584B064
:10E2000000AF78607B689B681846FEF771FEF86087
:10E21000FB68002B0ED0FB6813F10B0F0AD0FB68D4
:10E2200013F1800F06D0FB686FF4FA62934201D0BD
:10E23000FB680EE07B68DB68002BE3D07B68DB6863
:10E240007A68126910469847F860FB68002BD9D0AD
:10E25000FB6818461037BD4680BD80B584B000AF5E
:10E2600078607B681B681846F7F7C8FBF860FB68A6
:10E27000002B01D0FB680EE07B689B681846FFF717
:10E2800037FDF860FB68002B01D0FB6803E078687D
:10E2900001F0A2F9002318461037BD4680BD0000EA
:10E2A00080B584B000AF786039607B68002B02D104
:10E2B0006FF0150324E00023FB601CE0124AFB68AA
:10E2C00052F82330DB00114A1344BB60BB681B6863
:10E2D0001946786806F064FF0346002B08D10A4A05
:10E2E000FB6852F82330DAB23B681A70002307E06B
:10E2F000FB680133FB60FB680D2BDFD96FF0150362
:10E3000018461037BD4680BD080F02109008002047
:10E3100080B586B000AFF860B9607A607A6807F1BE
:10E3200014031946F86806F01BFA0246BB681A6027
:10E33000BB681B68002B06D17B691B78002B02D0C1
:10E340006FF0150300E0002318461837BD4680BD66
:10E3500080B586B000AFF860B9607A60FB68002BCA
:10E3600002D16FF0150340E0BB680C330A22194656
:10E37000F868FFF7CDFF78617B69002B01DA7B69D4
:10E3800033E07A681B49002006F03EFEF860FB6827
:10E39000002B02D16FF0150327E0BB680433102275
:10E3A0001946F868FFF7B4FF78617B69002B01DA42
:10E3B0007B691AE0BB6800221A767A680D49002052
:10E3C00006F022FEF860FB68002B0DD00A49F868C1
:10E3D00006F0E6FE0346002B03D1BB6801221A7645
:10E3E00002E06FF0150300E0002318461837BD4621
:10E3F00080BD00BF7C080020D40E021080B584B020
:10E4000000AFF860B9607A60FB68002B02D16FF052
:10E4100015031DE01049F86806F0C2FE0346002B04
:10E4200002D06FF0150313E07A680C49002006F063
:10E43000EBFDF860FB68002B02D16FF0150307E0DD
:10E44000BB6814330A221946F868FFF761FF0346D8
:10E4500018461037BD4680BDDC0E02107C08002037
:10E4600080B586B000AFF860B9607A60BB680422FE
:10E4700083F8D921FB68002B1FD000237B6119E0B2
:10E48000494A7B6952F823301946F86806F088FE3D
:10E490000346002B0BD17A684449002006F0B4FDF6
:10E4A000F8607B69DAB2BB6883F8D92105E07B6943
:10E4B00001337B617B69032BE2DDBB6893F8D931C3
:10E4C000032B04D0BB6893F8D931022B12D1FB681F
:10E4D000002B02D16FF0150361E0BB685933402275
:10E4E000F968184606F020FD7A683049002006F0E9
:10E4F0008BFDF860BB681B78082B3BD1FB68002BB9
:10E5000002D16FF015034AE0FB681B782F2B14D95A
:10E51000FB681B78392B10D8BB6899334FF4807295
:10E520000021184606F0AEFCBB6810330A221946DB
:10E53000F868FFF7EDFE034631E0BB6899334FF40E
:10E540008072F968184606F0EFFC7A6817490020D7
:10E5500006F05AFDF860FB68002B02D16FF015033E
:10E560001DE0BB6810330A221946F868FFF7D0FE99
:10E57000034614E0FB68002B08D0BB6899334FF4C6
:10E580008072F968184606F0CFFC07E0BB68993343
:10E590004FF480720021184606F074FC00231846E0
:10E5A0001837BD4680BD00BF800800207C080020D1
:10E5B00080B586B000AFF860B9607A607A68474984
:10E5C000F86806F021FD7861B9687869FFF768FEA0
:10E5D00038613B69002B01DA3B697AE07A683F4990
:10E5E000002006F011FD7861BB681B78032B02DC6C
:10E5F000002B03DA0DE0042B02D00AE0002368E0D0
:10E60000BB6808330A2219467869FFF781FE034682
:10E610005FE0BB68193340227969184606F084FC34
:10E620007A682E49002006F0EFFC7861BB681B7801
:10E63000053B082B4AD801A252F823F065E60010EA
:10E6400061E6001073E6001073E6001081E600102A
:10E6500081E6001061E6001093E60010BFE60010AE
:10E66000002336E07A68B9687869FFF771FE0346DF
:10E670002FE07A68B9687869FFF7F2FE034628E070
:10E68000BB6810330A2219467869FFF741FE03463A
:10E690001FE07B69002B08D0BB6803F2991340226E
:10E6A0007969184606F040FC07E0BB6803F299134D
:10E6B00040220021184606F0E5FB002309E07A68B5
:10E6C000B9687869FFF79AFE034602E000BF6FF071
:10E6D000150318461837BD4680BD00BF7C080020D2
:10E6E00080B485B000AFF860B9607A603B606FF0CD
:10E6F000150318461437BD465DF8047B704780B497
:10E7000083B000AF786039606FF0150318460C379E
:10E71000BD465DF8047B704780B485B000AFF860FB
:10E72000B9607A603B606FF0150318461437BD4638
:10E730005DF8047B704780B485B000AFF860B960C5
:10E740007A603B606FF0150318461437BD465DF8DC
:10E75000047B704780B485B000AFF860B9607A6020
:10E760003B606FF0150318461437BD465DF8047B17
:10E77000704780B483B000AF786039606FF01503E4
:10E7800018460C37BD465DF8047B704780B485B0F1
:10E7900000AFF860B9607A606FF01503184614375F
:10E7A000BD465DF8047B704780B483B000AF7860ED
:10E7B00039603B685B68002B03D03B681B68002B0B
:10E7C00002D16FF0150380E03B685A687B685A609D
:10E7D0003B681A687B681A603B689B68002B02D014
:10E7E0003B689B6800E03C4B7A6893603B68DB6861
:10E7F000002B02D03B68DB6800E0384B7A68D360BE
:10E800003B681B69002B02D03B681B6900E0344B5E
:10E810007A6813613B689B69002B02D03B689B6957
:10E8200000E0304B7A6893613B681B6A002B02D092
:10E830003B681B6A00E02C4B7A6813623B685B6A9A
:10E84000002B02D03B685B6A00E0274B7A6853627A
:10E850003B689B6A002B02D03B689B6A00E0204B20
:10E860007A6893623B68DB6A002B02D03B68DB6A04
:10E8700000E01C4B7A68D3623B681B6B002B02D014
:10E880003B681B6B00E0194B7A6813633B685B6B5A
:10E89000002B02D03B685B6B00E0154B7A6853633A
:10E8A0003B685B69002B02D03B685B6900E00B4B67
:10E8B0007A6853613B68DB69002B02D03B68DB69F7
:10E8C00000E0064B7A68D361002318460C37BD463A
:10E8D0005DF8047B704700BFE1E60010FFE6001022
:10E8E00037E7001055E7001019E7001073E7001034
:10E8F0008DE7001080B584B000AF786039607B6828
:10E90000002B06D03B68002B03D03B681B68002B14
:10E9100002D16FF0150338E041F6FC21012005F02B
:10E9200015F90346FB60FB68002B02D16FF00B0367
:10E930002BE0FB6803F5D55318333A68126811468B
:10E940001846FFF731FFB860BB68002B04DAF8689F
:10E9500005F046F9BB6818E03B689B68FA6802F569
:10E960008052C2F8F43A3B68DB68FA6802F58052DC
:10E97000C2F8F83A3B685B68FA6802F58052C2F860
:10E98000F03A7B68FA681A60002318461037BD46D3
:10E9900080BD80B582B000AF7860786805F020F95E
:10E9A00000BF0837BD4680BD80B582B000AF78603B
:10E9B0007B6808334FF4EE720021184606F062FAC5
:10E9C0007B6803F5F27314220021184606F05AFA08
:10E9D0007B6803F522730C220021184606F052FAD8
:10E9E0007B680022C3F8EC217B680022C3F8F02189
:10E9F0007B680022C3F87C227B68002283F8F82120
:10EA000000BF0837BD4680BD80B586B000AFF86056
:10EA1000B9607A60FB68002B02D07B68002B02D1C2
:10EA20006FF015033CE000237B6134E0FA687B69FA
:10EA30004FF42B7101FB03F3134404331B7883F071
:10EA40000103DBB2002B23D07B694FF42B7202FB56
:10EA500003F3FA6813443B614FF42B7200213869C9
:10EA600006F010FA3B6901221A71BB681A683B690B
:10EA70001A60BB685A683B69C3F88022BB689A6811
:10EA80003B69C3F884227B687A691A60002307E037
:10EA90007B6901337B617B69092BC7D96FF00F0359
:10EAA00018461837BD4680BDF0B587B002AFF86094
:10EAB000B9607A60BB681B780D2B65D801A252F84B
:10EAC00023F000BFFDEA001089EB001089EB001075
:10EAD00089EB001003EB001015EB001037EB001072
:10EAE00089EB001089EB001089EB001089EB001016
:10EAF00089EB001049EB001073EB00106FF0150369
:10EB000045E0FB681B6BBA689268114678689847C5
:10EB100003463CE0FB689C68BB6803F11901BB68D5
:10EB2000DA68BB685868BB681B7E00930346786848
:10EB3000A04703462BE0FB68DB68BA681932114630
:10EB400078689847034622E0FB68DC6ABB6803F1FB
:10EB50001905BB6803F29916BB6803F299131846AE
:10EB600006F08EFD0346324629467868A0470346E4
:10EB70000DE0FB685B6BBA6802F11901BA68526973
:10EB800078689847034602E000BF6FF01503184607
:10EB90001437BD46F0BD00BF80B58AB000AFF86045
:10EBA000B9607A60FB70FB6803F58053D3F8F03AE4
:10EBB0007B61BB681B68BB617B689A687B685B682C
:10EBC000D31A3B623B6A002B33D07B681A687B68A0
:10EBD0005B681344FB61FB7803F00103002B0BD04F
:10EBE000FB6803F58053D3F8B83A3A6A07F114008A
:10EBF000F969984778620AE0FB6803F58053D3F817
:10EC0000BC3A3A6A07F11400F969984778627B6A5E
:10EC1000002B01DA7B6A28E07B685A687B6A1A4419
:10EC20007B685A607A6A3B6A9A4202DA6FF00A039A
:10EC30001BE0FB7803F00203002B15D0FB6803F503
:10EC40008053D3F8B83A07F11400012209499847D4
:10EC500078627B6A002B01DA7B6A06E07B6A012B13
:10EC600002D06FF00A0300E0002318462837BD46A3
:10EC700080BD00BFEC0E021090B587B000AF786089
:10EC800039607B6803F58053D3F8F03ABB603B688A
:10EC90001B68FB603B68D3F89032002B2DD13B689A
:10ECA000D3F880223B68C3F888223B689A693B68A6
:10ECB000D3F88432934228BF13467B617B6803F507
:10ECC0008053D3F8C84A3B6803F121013B68D3F86D
:10ECD00088227B6907F10800A04738613B69002B57
:10ECE00001DA3B6933E03B697B617A693B68C3F8D1
:10ECF00090223B680022C3F88C223B68D3F88C2218
:10ED00003B68D3F890329A4220D23B6803F52272D6
:10ED1000012339687868FFF73FFF38613B69002BB2
:10ED200001DA3B6913E03B689A693B68D3F890329B
:10ED3000D21A3B689A613B680022C3F890223B6874
:10ED40009B69002B02D06FF00A0300E000231846F5
:10ED50001C37BD4690BD90B587B000AF7860396074
:10ED60007B6803F58053D3F8F03ABB603B681B68BF
:10ED7000FB603B68D3F89032002B16D13B68D3F888
:10ED800080223B68C3F888223B689A693B68D3F8C5
:10ED90008432934228BF13467B617A693B68C3F88B
:10EDA00090223B680022C3F88C223B68D3F88C2267
:10EDB0003B68D3F890329A420DD23B6803F5227239
:10EDC000042339687868FFF7E7FE38613B69002B58
:10EDD00001DA3B692AE07B6803F58053D3F8D04A17
:10EDE0003B6803F121013B68D3F888223B68D3F8E4
:10EDF000903207F10800A04738613B69002B01DA27
:10EE00003B6913E03B689A693B68D3F89032D21AA9
:10EE10003B689A613B680022C3F890223B689B697B
:10EE2000002B02D06FF00A0300E0002318461C37C5
:10EE3000BD4690BDB0B58CB002AF786039607B68DC
:10EE400003F58053D3F8F03ABB613B681B68FB6164
:10EE50003B6808333B623B6A93F8D9313B733B6AAA
:10EE600099333B613B6A59337B613B6A1B780D2BBD
:10EE700000F2298101A252F823F000BFB5EE001084
:10EE80000FEF001025EF00105FEF0010B5EE00103F
:10EE9000B5EE0010B5EE001071EF0010F7EF0010A6
:10EEA0004BF00010B3F0001071EF0010B5EE001041
:10EEB000B5EE00103B6A1B78052B0CD13B6A5A68F3
:10EEC0003B68C3F894223B6A1B7E002B03D03B684F
:10EED000012283F8A8223B6A1B78062B03D13B68EA
:10EEE000002283F8A8227B6803F5D553183307F175
:10EEF0001802396A1846FFF7D7FD03461A463B68E1
:10EF0000C3F8E4213B68012283F8E821DFE03B6895
:10EF10000022C3F8E4213B68012283F8E8216FF066
:10EF20007F03D5E07B6803F58053D3F8F82A3B686C
:10EF3000C3F8E4213B68012283F8E8217B6803F5EC
:10EF40008053D3F8F42A3B68C3F8EC217B6803F5BF
:10EF50008053D3F8F82A3B68C3F8F421B7E03B6844
:10EF60005D4AC3F8EC213B680B22C3F8F421AEE004
:10EF70003B6A1B78072B16D17B6803F58053D3F8C7
:10EF8000D84A3B6A03F119013B68D3F880523B68C9
:10EF9000D3F8843207F10C0207F1180000932B46D6
:10EFA000A047786211E07B6803F58053D3F8E04A0C
:10EFB0003B6A03F119013B68D3F880223B68D3F820
:10EFC000843207F11800A04778627A6A3B68C3F878
:10EFD000E4213B68012283F8E8217B6A002B75DB82
:10EFE0003B68D3F880223B68C3F8EC217A6A3B681F
:10EFF000C3F8F4216AE03B68D3F880223B6A1B69BE
:10F00000134400221A707B6803F58053D3F8DC4A5E
:10F010003B6A03F119013B68D3F880523B6A1B69D4
:10F0200007F10C0207F1180000932B46A047786205
:10F030003B680022C3F890227A6A3B68C3F8E42157
:10F040003B68012283F8E82141E03B68012283F814
:10F05000E8217B6803F58053D3F8CC3A3A6A02F191
:10F06000190107F118021046984778627B6A002B55
:10F0700004DA7A6A3B68C3F8E42128E03B6A1A693B
:10F080003B68C3F8E4213B6803F526703B68D3F87E
:10F090009432124A0A2105F09DFD78623B6803F51F
:10F0A00026723B68C3F8EC217A6A3B68C3F8F42106
:10F0B0000DE03B6A1A693B68C3F8E4213B68012212
:10F0C00083F8E82103E06FF0150301E000BF00239F
:10F0D00018462837BD46B0BDF00E0210FC0E0210D7
:10F0E00080B586B000AF786039607B6803F58053E7
:10F0F000D3F8F03ABB603B681B68FB6043E03B68B9
:10F1000003F2F9123B68D3F87C3213443B617B680D
:10F1100003F58053D3F8BC3A07F10800012239699E
:10F12000984778617B6913F10B0F02D07B69002B44
:10F1300002D16FF00A0335E07B69002B2CDB3B68C2
:10F14000D3F87C32002B08D13B691B780A2B1AD0EC
:10F150003B691B780D2B00D115E03B68D3F87C325E
:10F160005A1C3B68C3F87C223B691B780A2B0AD1E6
:10F170003B68D3F87C323A681344002283F8F921C3
:10F1800000237B6109E03B68D3F87C327E2BB6D943
:10F190006FF004037B6100E000BF3B680022C3F80E
:10F1A0007C227B6918461837BD4680BD80B586B085
:10F1B00000AF786039607B6803F58053D3F8F03A8C
:10F1C000FB603B681B683B613B6893F8F831062B9A
:10F1D00000F29F8101A252F823F000BFF9F1001064
:10F1E00083F20010A3F200109DF300103FF4001012
:10F1F00013F5001067F4001039687868FFF770FFA6
:10F2000078617B69002B01DA7B6984E13B6803F25A
:10F21000F9103B6803F108013B6803F529731A46AE
:10F22000FFF7C6F978617B69002B0CDA3B68012295
:10F2300083F8E8217A693B68C3F8E4213B6802223D
:10F2400083F8F8211BE03B681B7A082B13D13B683D
:10F25000D3F880223B68C3F888223B689A693B68F0
:10F26000C3F890223B680022C3F88C223B6804223A
:10F2700083F8F82103E03B68012283F8F82100239A
:10F2800049E139687868FFF7D5FD78617B69002B23
:10F2900001DA7B693FE13B68022283F8F821002311
:10F2A00039E13B6893F8E831002B33D03B68D3F861
:10F2B0009032002B18D13B6803F2F9123B68C3F877
:10F2C00088223B68D3F888023B68D3F8E4311A46B9
:10F2D000934905F0C3FC78617A693B68C3F89022D2
:10F2E0003B680022C3F88C223B68D3F88C223B6831
:10F2F000D3F890329A420DD23B6803F52272032371
:10F3000039687868FFF748FC78617B69002B01DA7F
:10F310007B6900E13B68D3F8EC31002B15D03B68EA
:10F32000D3F8F0213B68D3F8F4319A420DD23B6810
:10F3300003F5F672032339687868FFF72DFC7861CE
:10F340007B69002B01DA7B69E5E03B681B7A092BBE
:10F3500016D03B681B7A0A2B12D03B6893F8A83270
:10F36000002B08D03B681B7A052B04D03B68062293
:10F3700083F8F82110E03B68052283F8F8210BE0C0
:10F380003B6803F522730C220021184605F07AFD34
:10F390003B68032283F8F8210023BCE03B681B7A1A
:10F3A000092B05D139687868FFF766FC78613BE086
:10F3B00039687868FFF7CFFC78617B69002B33D11F
:10F3C0003B68012283F8E8217B6803F58053D3F87A
:10F3D000D43A3A6802F1210107F10C02104698472D
:10F3E00078617B69002B09DA7A693B68C3F8E4210C
:10F3F0003B68052283F8F82100238CE03B6803F585
:10F40000F6730C220021184605F03CFD3B689A6912
:10F410003B68C3F8E4213B6802221A723B6802226F
:10F4200083F8F821002376E07B69002B01DA7B6901
:10F4300071E03B68052283F8F82100236BE03B680C
:10F4400003F52272042339687868FFF7A5FB786119
:10F450007B69002B01DA7B695DE03B68012283F860
:10F46000F821002357E07B6803F58053D3F8D43AA2
:10F470003A6802F1210107F10C02104698477861C1
:10F480007B69002B19DA7A693B68C3F8E4217B6851
:10F4900003F58053D3F8C43A3A6802F1210107F129
:10F4A0000C02104698473B68052283F8F8213B6818
:10F4B000002283F8A82200232DE039687868FFF73E
:10F4C0000FFE78617B69002B01DA002323E03B68A3
:10F4D00003F2F9103B6803F108013B6803F5297357
:10F4E0001A46FFF765F878617B69002B0FDB3B68F4
:10F4F0001B7A062B0BD13B680022C3F890223B6895
:10F50000012283F8F8213B68002283F8A822002317
:10F5100001E06FF0150318461837BD4680BD00BFE7
:10F52000040F021080B584B000AF786039607B684A
:10F53000002B10D03B680A2B0DD87A683B684FF43B
:10F540002B7101FB03F3134404331B7883F0010395
:10F55000DBB2002B02D06FF015031FE03B684FF4C5
:10F560002B7202FB03F37A681344FB60F968786836
:10F57000FFF71CFEB860BB6813F10B0F01D1BB682D
:10F580000CE0BB68002B05DBFB6893F8F831052B1A
:10F5900000D0EBE7F868FFF707FABB6818461037AA
:10F5A000BD4680BD80B582B000AF7860786804F059
:10F5B0000FFB034618460837BD4680BD80B582B0B4
:10F5C00000AF786039603968786804F0BFFA0346A4
:10F5D00018460837BD4680BD80B582B000AF786060
:10F5E000786804F0FDFA00BF0837BD4680BD80B5DD
:10F5F00084B000AFF860B9607A60FB68002B02D17C
:10F600006FF015030BE028220021F86805F03AFCA2
:10F61000FB687A681A60FB68BA685A60002318466B
:10F620001037BD4680BD80B584B000AF78603960CA
:10F630007B68002B02D03B68002B02D16FF01503D2
:10F6400022E028210120FFF7B9FFF860FB68002BBA
:10F6500002D16FF00B0317E07B68FA681A60FB6851
:10F660003A681A6039680120FFF7A8FF0246FB6874
:10F670005A60FB685B68002B05D1F868FFF7ACFFA8
:10F680006FF00B0300E0002318461037BD4680BD25
:10F6900080B582B000AF78607B68002B02D14FF05C
:10F6A000FF330CE07B685B68002B04D07B685B68F1
:10F6B0001846FFF791FF7868FFF78EFF0023184682
:10F6C0000837BD4680BD80B485B000AF7860396032
:10F6D0007B68002B02D03B68002B02D16FF0150332
:10F6E00035E07B68DA687B68DB699A4206D97B681B
:10F6F000DA687B68DB69D31AFB6005E07B68DA684F
:10F700007B68DB69D31AFB60FB68002B0AD07B683F
:10F710001A687B689B681A447B689B69D21A3B68AD
:10F720001A6006E07B689A687B689B69D21A3B681E
:10F730001A603B681A687B681B689A4206D97B6826
:10F740001A683B681A606FF4FA6300E000231846F9
:10F750001437BD465DF8047B704780B588B000AFB4
:10F76000F860B9607A603B60FB68002B05D07B686D
:10F77000002B02D03B68002B02D16FF0150356E03E
:10F780000023FB6197F82830002B02D0FB68183368
:10F7900001E0FB680833BB61BB691B7A002B02D018
:10F7A0006FF00F0343E097F82830002B25D007F1C6
:10F7B00014031946F868FFF786FFF861FB696FF4D8
:10F7C000FA62934208D1FB68DB685A1EFB68DA6173
:10F7D000FB689A68FB689A617B69002B01D1002362
:10F7E00025E07B69BA68934228BF1346BB60BB68BB
:10F7F000002B02D16FF00A0319E0FB681A68BB699D
:10F800001B68D21ABB689A4228BF1A46BB69DA60E5
:10F81000BB69DA683B681A60FB685A68BB691B6899
:10F820001A447B681A60BB6901221A72FB69184688
:10F830002037BD4680BD80B485B000AF78600B46F0
:10F84000FB707B68002B02D16FF0150335E0FB786D
:10F85000002B02D07B68183301E07B680833BB6063
:10F86000BB681B7A83F00103DBB2002B02D04FF0A0
:10F87000FF3322E0BB681A68BB68DB681344FB6097
:10F880007B681B68FA689A420DD3BB685B685A1C98
:10F89000BB685A607B681A68FB68B3FBF2F101FB36
:10F8A00002F29B1AFB60BB68FA681A60BB68002210
:10F8B000DA60BB6800221A72002318461437BD466E
:10F8C0005DF8047B704780B58CB002AFF860B9601A
:10F8D0007A60FB7000237B61FB68002B05D0BB685E
:10F8E000002B02D07B68002B02D16FF0150352E091
:10F8F000002387F8233000237B6240E07A687B6A2C
:10F90000D11A07F1140007F11802FB78009303469F
:10F91000F868FFF722FFF861FB6913F1100FEDD0D3
:10F92000FB6913F10B0FE9D0FB696FF4FA629342A4
:10F9300002D1012387F823307B69002B02D14FF0DD
:10F94000FF3328E0FB78002B08D0BA687B6A1344A9
:10F95000B9697A69184605F0F1FD07E0B869BA6837
:10F960007B6A13447A69194605F0E8FDFB7819466D
:10F97000F868FFF760FF7B697A6A13447B627A6AF2
:10F980007B689A42BAD397F82330002B02D06FF4E9
:10F99000FA6300E0002318462837BD4680BD80B5D5
:10F9A00086B002AFF860B9607A603B6000230093D4
:10F9B0003B687A68B968F868FFF7CFFE03461846D7
:10F9C0001037BD4680BD80B586B002AFF860B96023
:10F9D0007A603B60012300933B687A68B968F868F5
:10F9E000FFF7BBFE034618461037BD4680BD80B505
:10F9F00082B000AF786000217868FFF71CFF0346F3
:10FA000018460837BD4680BD80B582B000AF78602B
:10FA100001217868FFF70FFF034618460837BD46F7
:10FA200080BD80B584B000AFF860B9607A60002313
:10FA30007A68B968F868FFF746FF0346184610373A
:10FA4000BD4680BD80B584B000AFF860B9607A6013
:10FA500001237A68B968F868FFF735FF034618464E
:10FA60001037BD4680BD80B485B000AF78600B46CE
:10FA7000FB707B68002B2DD00023FB8125E0FB89E8
:10FA80007B7300233B7311E097F90D30002B07DAED
:10FA90007B7B5B007B737A7BFB7853407B7302E05C
:10FAA0007B7B5B007B733B7B01333B733B7B072B97
:10FAB000EAD9B7F90E307A6813447A7B1A70B7F92D
:10FAC0000E309BB201339BB2FB81B7F90E30FF2B96
:10FAD000D5DD00E000BF1437BD465DF8047B7047FC
:10FAE00080B487B000AFF860B9607A60FB700DE059
:10FAF000BB681A78FB785340DBB27B61FA687B699C
:10FB000013441B78FB70BB680133BB607B685A1ED3
:10FB10007A60002BECD1FB7818461C37BD465DF8A7
:10FB2000047B704780B584B000AF78607B68002BA1
:10FB300002D16FF0150320E008210120FFF73EFD00
:10FB4000F860FB68002B02D16FF00B0315E04FF457
:10FB500080710120FFF732FD0246FB681A60FB68E6
:10FB60001B68002B05D1F868FFF736FD6FF00B031B
:10FB700003E07B68FA681A60002318461037BD4618
:10FB800080BD80B483B000AF78607B685B7901335F
:10FB90007A68127993420CBF01230023DBB2184626
:10FBA0000C37BD465DF8047B704780B483B000AF6E
:10FBB00078607B685A797B681B799A420CBF012375
:10FBC0000023DBB218460C37BD465DF8047B704756
:10FBD00080B582B000AF786039607868FFF7E5FFE4
:10FBE0000346002B02D04FF0FF330EE07B681B680A
:10FBF0007A68127913441A783B681A707B681B790B
:10FC00000133DAB27B681A71002318460837BD4603
:10FC100080BD80B582B000AF78600B46FB7078681D
:10FC2000FFF7AFFF0346002B02D04FF0FF330DE08C
:10FC30007B681B687A6852791344FA781A707B687B
:10FC40005B790133DAB27B685A71002318460837B2
:10FC5000BD4680BD80B582B000AF78607B68002B68
:10FC600008D07B681B68002B04D07B681B68184693
:10FC7000FFF7B2FC00BF0837BD4680BD80B483B03B
:10FC800000AF786039607A683B68D31A9B101846D9
:10FC90000C37BD465DF8047B704780B586B000AF79
:10FCA000F860B9607A600C210120FFF787FC786169
:10FCB0007B69002B01D1002309E07B69FA681A6097
:10FCC0007B69BA685A607B697A689A607B69184672
:10FCD0001837BD4680BD80B485B000AFF860B9600C
:10FCE0007A60FB68002B07D0BB68002B01D0BB6893
:10FCF00000E07B68FA689360BB68002B05D0BB68A6
:10FD0000FA685A60BB687A689A607B68002B07D0F3
:10FD1000BB68002B01D0BB6800E0FB687A685360C9
:10FD200000BF1437BD465DF8047B704780B485B0D2
:10FD300000AFF860B9607A60FB681B68BA689A42E5
:10FD40000CD1FB687A685A60BB68002B02D07B68D4
:10FD5000002B0FD1FB687A681A600BE0FB68BA6869
:10FD60001A607B68002B02D0BB68002B02D1FB68B5
:10FD7000BA685A6000BF1437BD465DF8047B70470F
:10FD800080B483B000AF78600B46FB70FB78012B2A
:10FD900011D0032B1FD17B681A4A1A607B681A4A5C
:10FDA0005A607B68194A9A607B68194ADA607B68F6
:10FDB000184A1A611FE07B68174A1A607B68124A6A
:10FDC0005A607B68114A9A607B68114ADA607B68E6
:10FDD000104A1A610FE07B680F4A1A607B680F4A6D
:10FDE0005A607B680A4A9A607B68084ADA607B68D6
:10FDF0000B4A1A6100BF00BF0C37BD465DF8047B9B
:10FE0000704700BFD7FF0010CF010110C1000110E3
:10FE10000F0101105D0001106DFF00105102011073
:10FE20008F00011080B586B000AFF8600B467A6095
:10FE3000FB72FB68002B02D14FF0FF332FE018213B
:10FE40000120FFF7BBFB78617B69002B02D14FF0EB
:10FE5000FF3324E01C210120FFF7B0FB38613B6930
:10FE6000002B05D17869FFF7B7FB4FF0FF3316E0A1
:10FE7000FB687A691A607B693A695A617B68002B72
:10FE800001D07B6800E0084B3A69D360FB7A1946E1
:10FE90007869FFF775FF3B693A695A610023184694
:10FEA0001837BD4680BD00BF7DFC001080B584B012
:10FEB00000AF78607B68002B02D14FF0FF331CE06D
:10FEC0007B685B69FB60FB681B69002B02D04FF00D
:10FED000FF3312E000BF07F108031946786800F00D
:10FEE00076F90346002BF6D07B685B691846FFF76E
:10FEF00073FB7868FFF770FB002318461037BD4688
:10FF000080BD80B586B000AF786039607B68002B1B
:10FF100002D14FF0FF3325E07B685B697B610023F2
:10FF20003B617B691B68FB60FA6839693868FFF7D9
:10FF3000B4FEB860BB68002B02D14FF0FF3311E074
:10FF4000FA68B9683869FFF7C6FE7B695B681A46CC
:10FF5000B9687869FFF7EAFE7B699B685A1C7B6980
:10FF60009A60002318461837BD4680BD80B586B01C
:10FF700000AF786039607B68002B02D14FF0FF330F
:10FF800025E07B685B697B617B695B683B61002383
:10FF9000FB60FA6839693868FFF77FFEB860BB68B4
:10FFA000002B02D14FF0FF3311E0FA68B9683869CD
:10FFB000FFF791FE7B691B68BA6819467869FFF7FD
:10FFC000B5FE7B699B685A1C7B699A6000231846C2
:10FFD0001837BD4680BD80B584B000AF7860396009
:10FFE0007B68002B02D14FF0FF3333E07B685B6905
:10FFF000BB60BB681B68FB600CE0BB68DB68FA6831
:020000041001E9
:1000000012683968104698470346002B06DCFB68E7
:100010009B68FB60FB68002BEFD100E000BFFB6832
:10002000002B0CD1BB685A68BB689A61BB6814335B
:1000300001223968184600F034FA03460AE0BB682A
:10004000FA689A61BB68143300223968184600F0D8
:1000500028FA034618461037BD4680BD80B485B0E7
:1000600000AF786039607B68002B02D14FF0FF331E
:1000700007E07B685B69FB60FB681B683A681A6095
:10008000002318461437BD465DF8047B704780B4E2
:1000900085B000AF786039607B68002B02D14FF0EB
:1000A000FF3307E07B685B69FB60FB685B683A686D
:1000B0001A60002318461437BD465DF8047B70476C
:1000C00080B485B000AF786039607B68002B02D0C7
:1000D0003B68002B02D14FF0FF3312E03B68002257
:1000E0001A607B685B69FB60FB681B68002B02D1B0
:1000F0004FF0FF3305E0FB681B681A683B681A6025
:10010000002318461437BD465DF8047B704780B461
:1001100085B000AF786039607B68002B02D03B6807
:10012000002B02D14FF0FF3312E03B6800221A602F
:100130007B685B69FB60FB685B68002B02D14FF05A
:10014000FF3305E0FB685B681A683B681A600023B0
:1001500018461437BD465DF8047B704780B586B0FD
:1001600000AFF860B9607A60FB68002B02D0BB6812
:10017000002B02D14FF0FF3325E0BB6800221A604C
:10018000FB685B697B617B69002B02D14FF0FF3319
:1001900019E0FB685B697B617B691A687B699A611E
:1001A0007B6914337968184600F0C3F80346002BC6
:1001B00002D04FF0FF3306E07B691433B96818466C
:1001C00000F04FF9034618461837BD4680BD80B58C
:1001D00086B000AF786039607B68002B02D03B6846
:1001E000002B02D14FF0FF332EE03B6800221A6053
:1001F0007B685B697B617B699B68002B02D14FF058
:10020000FF3321E07B691B683B613B695B68FB60F6
:100210003B699B68BB60BA680021F868FFF75BFD2B
:100220007B695B681A46B9687869FFF77FFD7B696F
:100230009B685A1E7B699A603B691A683B681A6022
:100240003869FFF7C9F9002318461837BD4680BD45
:1002500080B586B000AF786039607B68002B02D033
:100260003B68002B02D14FF0FF332EE03B680022A9
:100270001A607B685B697B617B699B68002B02D19C
:100280004FF0FF3321E07B695B683B613B695B6852
:10029000FB603B699B68BB60BA680021F868FFF7A8
:1002A0001AFD7B691B68FA6819467869FFF73EFDFD
:1002B0007B699B685A1E7B699A603B691A683B6838
:1002C0001A603869FFF788F9002318461837BD46C9
:1002D00080BD80B586B000AFF860B9607A60FB6819
:1002E000002B02D0BB68002B02D14FF0FF331CE083
:1002F000BB6800221A60FB685B697B617B691A68D6
:100300007B699A617B6914337968184600F011F8AB
:100310000346002B02D04FF0FF3306E07B69143315
:10032000B968184600F033F8034618461837BD463A
:1003300080BD80B584B000AF786039607B68BB60F9
:10034000BB68002B02D14FF0FF331CE0BB681B6879
:100350001B68FB6012E0BB681B68DB68FA68126808
:100360003968104698470346002B04D1BB68FA68E9
:100370005A60002307E0FB689B68FB60FB68002B6A
:10038000E9D14FF0FF3318461037BD4680BD80B528
:1003900084B000AF786039607B68BB60BB68002BBD
:1003A00006D0BB685B68002B02D03B68002B02D1F3
:1003B0004FF0FF3351E0BB685B685868BB685B680F
:1003C0009B681A460021FFF786FCBB685A68BB6829
:1003D0001B681B689A420BD1BB681868BB685B68D6
:1003E0009968BB681B685B681A46FFF79FFC11E0C1
:1003F000BB685A68BB681B685B689A420AD1BB68D5
:100400001868BB681B681968BB685B685B681A463C
:10041000FFF78CFCBB681B689A68013A9A60BB685E
:100420005B681A683B681A60BB685A68BB681B68DF
:100430005B689A4204D1BB685B685B68FB6003E061
:10044000BB685B689B68FB60BB685B681846FFF72E
:10045000C3F8BB68FA685A60002318461037BD46D7
:1004600080BD80B485B000AF786039607B68FB6088
:10047000FB68002B06D0FB685B68002B02D03B6852
:10048000002B02D14FF0FF3305E0FB685B681A6870
:100490003B681A60002318461437BD465DF8047B9C
:1004A000704780B58CB000AFF860B9601346FB713F
:1004B000FB68BB62BB6A002B02D14FF0FF3355E0F3
:1004C000FB681B687B62FB79002B0ED0BB6A5A6805
:1004D000BB6A1B685B689A4207D107F11003B968D1
:1004E0001846FFF743FD034640E0FB7983F0010324
:1004F000DBB2002B0ED0BB6A5A68BB6A1B681B6854
:100500009A4207D107F11003B9681846FFF7F9FCC2
:1005100003462BE0FB79002B0AD0BB6A5968BB6A03
:100520005B689B681A46B868FFF7B7FBF86209E09A
:10053000BB6A5B685968BB6A5B681A46B868FFF7B4
:10054000ACFBF862FB6A002B02D14FF0FF330DE0E9
:10055000FB6A5868FB6A9B681A46F96AFFF7BBFB9F
:10056000BB6A1B689A6801329A60002318463037CC
:10057000BD4680BD80B483B000AF786000BF0C374B
:10058000BD465DF8047B704780B483B000AF7860EF
:1005900000BF0C37BD465DF8047B704780B483B064
:1005A00000AF786000BF0C37BD465DF8047B704734
:1005B00080B483B000AF786000BF0C37BD465DF8F3
:1005C000047B704784B02DE9B04382B000AF7860FF
:1005D00007F1240080E80E007B68002B02D16FF049
:1005E000150331E0FA6B3B6C9A4202DA6FF01503A7
:1005F0002AE038210120FEF7E1FF02467B681A60FD
:100600007B681B68002B02D16FF00B031CE07B683A
:100610001B6803F1100407F124050FCD0FC40FCDA3
:100620000FC42B6823607B6C7A681268D9179846D0
:100630008946C2E902897B681B6800221A607B68D0
:100640001B6800225A60002318460837BD46BDE8E3
:10065000B04304B0704700002DE9B04FB0B000AF18
:10066000C7F89400C7F89010C7F88C20C7F88830F6
:10067000D7F89430002B03D0D7F88830002B02D164
:100680006FF0150383E1D7F894302033C7F8BC30FE
:10069000D7F894302833C7F8B830D7F89020D7F877
:1006A0008C30D31AC7F8B430D7F8B430002BB8BFA9
:1006B0005B421A46D7F89430DB699A42C0F05E81FB
:1006C000D7F894301B6900223B677A67D7F8B430BB
:1006D000DA1798469146D7E91C010B4608FB03F24E
:1006E000034603FB09F313440246A2FB08452B44CF
:1006F0001D46C7E92A45C7E92A45D7F8BC301A681C
:10070000D7F8BC305B689A421CDDD7F894301A6881
:10071000D7F8BC301B689A4206DDD7F8BC301A689F
:10072000D7F894301A600DE0D7F894301A68D7F8EB
:10073000BC305B689A4205DAD7F8BC305A68D7F803
:1007400094301A60D7F894305B690022BB66FA6671
:10075000D7F894301B68DA173B667A66D7E91A45F2
:100760002B46D7E91889424602FB03F24B46214645
:1007700001FB03F3134422464146A2FB0112C7F8D2
:1007800084200A46C7F88020D7F884201344C7F88D
:100790008430D7E92034C7E92834C7E92834D7F8AA
:1007A00094309B690022BB65FA65D7F894305A688B
:1007B000D7F8B430D31ADA173B657A65D7E916450E
:1007C0002B46D7E91489424602FB03F24B462146E9
:1007D00001FB03F3134422464146A2FB0112FA67D0
:1007E0000A46BA67FA6F1344FB67D7E91E34C7E9B4
:1007F0002634C7E92634D7F89430D3E90245224697
:100800002B464FF000004FF00001590141EAD26140
:10081000500102460B46B2EB040A63EB050B4FF0A6
:1008200000024FF000034FEA4B2343EADA534FEA4A
:100830004A2292469B461AEB0403BB604BEB05032E
:10084000FB604FF000024FF00003D7E902894946F0
:100850008B01414643EA916341468A014146511A60
:100860003960494663EB01037B60D7E900120B4610
:100870001B19BB64134645EB0303FB64D7E92A014C
:10088000D7E9282384183C6441EB03037B64D7E950
:100890002623D7E9104521468918B963294643EB39
:1008A0000101F963D7E912452346D7E90E01024653
:1008B0009B1A3B632B460A4663EB02037B63364A73
:1008C0004FF00003D7E90C0102F080FF02460B460F
:1008D000D7F89410C1E90223D7F8B8301A68D7F8CE
:1008E000B8305B689A423ADDD7F89430D3E90223F6
:1008F000D7F8B8100968C817B962F862D7E90A458D
:1009000021469142294699410CDAD7F8B8301B6844
:10091000DA173B627A62D7F89430D7E90812C3E954
:1009200002121CE0D7F89430D3E90223D7F8B810AC
:100930004968C817B961F861D7E9064521468A4276
:1009400029468B410BDAD7F8B8305B68DA173B6180
:100950007A61D7F89430D7E90412C3E90212D7F8C4
:1009600094301A68D7F8B4301A44D7F894301A6023
:10097000D7F89430D7F8B4205A6000E000BFD7F819
:100980009430D3E90223D7F888301A600023184640
:10099000C037BD46BDE8B08F40420F0080B483B081
:1009A00000AF786039607B68002B02D16FF01503CF
:1009B00003E07B683A68DA61002318460C37BD46CD
:1009C0005DF8047B704780B483B000AF78607B68CB
:1009D000002B02D16FF0150306E07B6800221A603D
:1009E0007B6800225A60002318460C37BD465DF82C
:1009F000047B704780B582B000AF78607B68002BC5
:100A000002D16FF0150305E07868FEF7E5FD0023DD
:100A10007B60002318460837BD4680BD80B485B092
:100A200000AF78600023FB600CE07B6803F00103FB
:100A3000002B01D0FB6809E07B685B087B60FB68EA
:100A40000133FB607B68002BEFD12023184614375D
:100A5000BD465DF8047B704780B582B000AF78601A
:100A600039607868FFF7DAFF02463B6803FA02F262
:100A70007B68134018460837BD4680BD90B583B0EB
:100A800000AF786039603A687B6802EA03047868EE
:100A9000FFF7C4FF034624FA03F318460C37BD469C
:100AA00090BD80B485B000AF0346FB710023FB60AE
:100AB0000AE0FB7903F00103002B02D0FB6801334D
:100AC000FB60FB795B08FB71FB79002BF1D1FB68C4
:100AD00018461437BD465DF8047B70472DE9B043D6
:100AE00084B000AFC7E902017A603B607B68DA1727
:100AF00098469146D7E9020142464B4602F066FE0F
:100B00003B681A607B68DA171C46154622462B465E
:100B1000D7E9020102F05AFE02460B46104619467A
:100B20001037BD46BDE8B08380B586B000AFC7E9D9
:100B300002017A6007F114037A68D7E90201FFF72E
:100B4000CDFF02460B46104619461837BD4680BDFC
:100B500080B483B000AF03463960FB803B6801334B
:100B6000FA88D2B21A70FB881B0A9BB2DAB23B68D1
:100B70001A7000BF0C37BD465DF8047B704700005B
:100B800080B582B000AF42494248F4F702FB78607A
:100B90007B68002B01D07B6876E03F493F48F4F743
:100BA000F8FA78607B68002B01D07B686CE03C49E8
:100BB0003C48F4F7EEFA78607B68002B01D07B6844
:100BC00062E039493948F4F7E4FA78607B68002B31
:100BD00001D07B6858E036493648F4F7DAFA786095
:100BE0007B68002B01D07B684EE033493348F4F733
:100BF000D0FA78607B68002B01D07B6844E03049F4
:100C00003048F4F7C6FA78607B68002B01D07B6827
:100C10003AE02D492D48F4F7BCFA78607B68002B48
:100C200001D07B6830E01B4B1B6800211846F4F7AD
:100C300021FB1A4B1B6800211846F4F71BFB194BCC
:100C40001B6800211846F4F715FB184B1B680021A0
:100C50001846F4F70FFB174B1B6800211846F4F7F2
:100C600009FB164B1B6800211846F4F703FB154BD4
:100C70001B6800211846F4F7FDFA144B1B6800218D
:100C80001846F4F7F7FA002318460837BD4680BD2A
:100C9000FC0B0020782A0020100C00207C2A002069
:100CA000380C0020702A0020240C0020742A002018
:100CB0004C0C0020842A0020600C0020802A002098
:100CC000740C0020882A0020880C00208C2A002028
:100CD00080B582B000AF0346FB71054B1B68FA7903
:100CE00011461846F4F7ECFA00BF0837BD4680BD40
:100CF000782A002080B582B000AF0346FB71054B17
:100D00001B68FA7911461846F4F7DAFA00BF08377B
:100D1000BD4680BD7C2A002080B582B000AF03466E
:100D2000FB71054B1B68FA7911461846F4F7C8FAAF
:100D300000BF0837BD4680BD742A002080B582B050
:100D400000AF0346FB71054B1B68FA791146184644
:100D5000F4F7B6FA00BF0837BD4680BD702A002000
:100D600080B582B000AF0346FB71054B1B68FA7972
:100D700011461846F4F7A4FA00BF0837BD4680BDF7
:100D8000802A002080B582B000AF0346FB71054B7E
:100D90001B68FA7911461846F4F792FA00BF083733
:100DA000BD4680BD842A002080B582B000AF0346D6
:100DB000FB710D4B1A68FB7903F00103DBB2194696
:100DC0001046F4F77DFA094B1A68FB795B10DBB229
:100DD00003F00103DBB219461046F4F771FA00BFC5
:100DE0000837BD4680BD00BF882A00208C2A00201D
:100DF00080B584B000AF786039600023FB602AE0E2
:100E00000120FFF765FF0120FFF774FF0120FFF7C6
:100E100083FF0120FFF7A4FF3A687B68B2FBF3F37E
:100E20005B081846F6F7E7FA0020FFF751FF0020AD
:100E3000FFF760FF0020FFF76FFF0020FFF790FF34
:100E40003A687B68B2FBF3F35B081846F6F7D3FA0F
:100E5000FB680133FB60FB687A689A42D0D800BF18
:100E600000BF1037BD4680BD80B584B000AF78604C
:100E70007B68FB601F4B1B78DBB283F00103DBB2A6
:100E8000002B01D0002330E00023FB72FB685B687D
:100E90001B6807F10B0241F608011846F9F762FAE0
:100EA000FB7A002B14BF01230023DBB21846FFF7A7
:100EB0000FFF0023FB72FB689B681B6807F10B02A6
:100EC00041F608011846F9F74DFAFB7A002B14BFDA
:100ED00001230023DBB21846FFF70CFFF86800F08F
:100EE00023FF044B00221A70002318461037BD461A
:100EF00080BD00BF902A002080B582B000AF78602E
:100F0000054B01221A7000217868F8F701F800BF3C
:100F10000837BD4680BD00BF902A002080B58EB046
:100F200000AF07F1240300221A605A609A60DA6069
:100F300007F1240207F1200311461846F7F786FF50
:100F400078637B6B002B01D07B6B57E03B6A012100
:100F50001846F8F725F878637B6B002B01D07B6B84
:100F60004CE007F1100300221A605A609A60254B8A
:100F70007B6107F1100207F11C0311461846F4F7D4
:100F800031FB78633B4600221A605A609A60DA604F
:100F90001D4B3B603B6A7B6004233B7202237B72E8
:100FA000FB693A4603211846F4F769FB78637B6BCB
:100FB000002B01D07B6B21E0FB6901220321184645
:100FC000F4F70EFC78637B6B002B01D07B6B15E094
:100FD000FB6903211846F4F7BFFB78637B6B002B9A
:100FE00001D07B6B0AE03B6A1846F7F76FFF786326
:100FF0007B6B002B01D07B6B00E000231846383759
:10100000BD4680BD60070210F90E01102DE9F041C8
:10101000ADF5387D0EAF6B469846052387F89F32B5
:10102000FF23A7F89C32B7F89C32C7F89832B7F87C
:101030009C32013300221C4615464FF000024FF04F
:101040000003EB0043EA5473E200B7F89C3201332B
:101050000022184611464FF000024FF00003CB006B
:1010600043EA5073C200B7F89C3201330733DB0800
:10107000DB00ADEB030D0EAB0033C7F89432072154
:10108000D048FEF7F0FCD04B07F510741D460FCD8D
:101090000FC495E8070084E807004FF4E133C7F870
:1010A0004C3207F5107207F5217311461846F4F714
:1010B00061FCC7F8A402D7F8A432002B03D0D7F8FC
:1010C000A43200F068BDD7F884321846F8F7F2FB76
:1010D0004222BE49BE4803F043FC07F51C73BD49DC
:1010E0001846F4F756F8C7F8A402D7F8A432002B34
:1010F00040F01385D7F870321846F4F799F8C7F81E
:10110000A402D7F8A432002B40F00985D7F870323A
:1011100007F2772211461846F4F7F8F8C7F8A40248
:10112000D7F8A432002B40F0FC8497F87732002BDC
:1011300001D0012200E0022297F89F3207F51E70CD
:10114000A54903F08BFD07F51E731946A34803F06C
:1011500007FCFFF715FDC7F8A402D7F8A432002B4F
:1011600040F0E18407F51A739D491846F3F792FFA2
:10117000C7F8A402D7F8A432002B40F0D68407F5B4
:101180001B7398491846F4F704F8C7F8A402D7F877
:10119000A432002B40F0CB84D7F86C321846F4F719
:1011A00047F8C7F8A402D7F8A432002B40F0C18456
:1011B000D7F86C3207F2762211461846F4F7A6F8F3
:1011C000C7F8A402D7F8A432002B40F0B48497F8F3
:1011D0007632002B66D100BF834803F021FCD7F89C
:1011E0006802B7F89C3201339BB2D7F894224FF4CF
:1011F0007061F3F7A5FFC7F8A402D7F8A432002B5B
:1012000003D0D7F8A43200F0C6BCB7F89C22A523BF
:10121000D7F894126B48FEF763FC034687F89332C5
:10122000B7F89C32D7F89422D35C97F893229A426D
:101230001DD1D7F86802B7F89C3201339BB2D7F8BA
:1012400094220021F3F753FFC7F8A402D7F8A43281
:10125000002B03D0D7F8A43200F09DBC634803F004
:10126000DFFB40F6B8310A20FFF7C2FD1AE0B7F8FD
:101270009C32D7F89422D35C194697F893321A46D9
:101280005B4803F06DFB5B4803F0CAFBB7F89C3288
:101290001A465949D7F8940204F050F9574803F018
:1012A000BFFB3EE0564803F0BBFBD7F86802B7F837
:1012B0009C3201339BB2D7F894220021F3F740FF10
:1012C000C7F8A402D7F8A432002B03D0D7F8A43271
:1012D00000F061BCB7F89C22A523D7F894123948D6
:1012E000FEF7FEFB034687F89332B7F89C32D7F837
:1012F0009422D35C97F893229A420FD0B7F89C328D
:10130000D7F89422D35C194697F893321A46384896
:1013100003F026FB3B4803F083FB5DE73A4803F00C
:101320007FFBD7F89432C7F88C3297F89F32012BA5
:1013300002D0032B04D007E06423C7F8A03208E0F2
:101340006423C7F8A03204E04FF47A73C7F8A032E0
:1013500000BFD7F8A02207F5187107F519731846D2
:1013600001F00EFFC7F8A402D7F8A432002B40F01A
:10137000E4830023C7F82432244BC7F828325A23C9
:1013800087F82C32224BC7F83032012387F83832E5
:1013900007F50E73C7F8343207F50973C7F83C3206
:1013A00007F50F7207F5177311461846F3F736FE67
:1013B000C7F8A402D7F8A432002B2BD0D7F8A43258
:1013C000E9E300BF942A0020980A0020400F021091
:1013D000600F0210D40B0020780F0210840F02104F
:1013E000B80C0020E80B0020980F0210BC0F021070
:1013F000E00F021010100210901102103C100210A9
:101400006C10021098100210CC100210A08601007F
:1014100050070210DF4BC7F8E831D7F88C3293F849
:10142000363087F8EC31D7F88C32D3F83730C7F83C
:10143000F031D7F88C32D3F83B30C7F8F431D7F815
:101440008C3293F83F3087F8F831D7F88C321B6C28
:10145000C7F8FC31D7F88C325B6CC7F80032D7F88C
:101460008C3293F8483087F80432D7F88C3293F8EE
:10147000493087F8053297F877321A4613469B00B1
:1014800013449B004833D7F88C2213440233C7F827
:10149000083297F89F3287F80C3297F87732002B92
:1014A00014BF01230023DBB287F80D32BA4BC7F813
:1014B0001032D7F86832C7F81432D7F864321B6894
:1014C000C7F81832D7F860321B68C7F81C3207F526
:1014D000F47207F508731146184601F071FCC7F85D
:1014E000A402D7F8A432002B40F02983D7F8203289
:1014F000184600F02DFEC7F8A402D7F8A432002B3E
:1015000040F01F8307F52A73A3F5987318466823E4
:101510001A46002103F0B6FC07F52A73A3F5987369
:1015200000221A7007F52A73A3F5987301225A70E6
:1015300007F52A73A3F59873984A1C1D15460FCD1D
:101540000FC42B68236007F52A73A3F59873944A98
:1015500003F1180415460FCD0FC42B68236007F55F
:101560002A73A3F598738F4A03F12C0415460FCD07
:101570000FC42B68236007F52A73A3F598738A4A72
:1015800003F1400415460FCD0FC42B68236097F874
:101590007732D7F88C220E33DB00D118D1F8032034
:1015A000D1F8073007F52A71A1F59871C1E9162322
:1015B000D7F88C3293F8722007F52A73A3F5987345
:1015C00083F8542007F52A73A3F59873012283F852
:1015D0005520D7F88C3293F8832007F52A73A3F5AA
:1015E000987383F86020D7F88C3293F8842007F53D
:1015F0002A73A3F5987383F8612007F52A73A3F57E
:101600009A7307F5BC721A6007F5BA7207F5F273A0
:1016100011461846FAF780F8C7F8A402D7F8A432A2
:10162000002B40F0908297F89F32052B41D1D7F8DC
:10163000E43118684FF0FF33C7F88832D7F88832A2
:101640001B07C7F88832D7F888321B0FC7F88832D3
:10165000D7F888329BB243F480739BB208221946B4
:10166000F8F744FEC7F8A402D7F8A432002B40F0E4
:101670006C82D7F8E4311B6800224FF401711846E0
:10168000F8F734FEC7F8A402D7F8A432002B40F0D4
:101690005E82D7F8E4311B68002240F2022118462E
:1016A000F8F724FEC7F8A402D7F8A432002B40F0C4
:1016B000508207F52A73A3F5D073184668231A469B
:1016C000002103F0DFFB07F52A73A3F5D073012295
:1016D0001A7007F52A73A3F5D07301225A7007F523
:1016E0002A73A3F5D0732D4A1C1D15460FCD0FC4C8
:1016F0002B68236007F52A73A3F5D073284A03F1FA
:10170000180415460FCD0FC42B68236007F52A7304
:10171000A3F5D073234A03F12C0415460FCD0FC453
:101720002B68236007F52A73A3F5D0731F4A03F1D2
:10173000400415460FCD0FC42B68236097F877320D
:10174000D7F88C221033DB00D118D1F80620D1F85D
:101750000A3007F52A71A1F5D071C1E91623D7F82F
:101760008C3293F8852007F52A73A3F5D07383F89C
:10177000542007F52A73A3F5D073012283F855206E
:10178000D7F88C3293F8962007F52A73A3F5D07317
:101790000EE000BFBC0A0020942A0020D00A0020DE
:1017A000E40A0020F80A00200C0B0020200B002087
:1017B00083F86020D7F88C3293F8982007F52A73C5
:1017C000A3F5D07383F86120D7F88C3293F8992071
:1017D00007F52A73A3F5D07383F86220D7F88C320B
:1017E00093F89A2007F52A73A3F5D07383F8632042
:1017F000D7F88C3293F89B2007F52A73A3F5D073A2
:1018000083F86420D7F88C3293F8972007F52A7371
:10181000A3F5D07383F8652007F52A73A3F5D07379
:10182000002283F8662007F52A73A3F5D0730022FF
:1018300083F8672007F52A73A3F5D27307F584723E
:101840001A6007F5827207F5B87311461846F9F762
:1018500063FFC7F8A402D7F8A432002B40F07B81C5
:10186000D7F82032D7F8E4215A60D7F8203207F5AC
:101870002A72A2F59C7212689A60FFF74FFBC7F8B4
:10188000A402D7F8A432002B40F0678107F52A7331
:10189000A3F50D73184690231A46002103F0F2FABF
:1018A00007F52A73A3F50D73BE4A1A60D7F8E42131
:1018B00007F52A73A3F50D735A60D7F8E4315A6817
:1018C00007F52A73A3F50D739A6007F52A73A3F53C
:1018D0000D73B54A9A6107F52A73A3F59C731A68CC
:1018E00007F52A73A3F50D73DA6107F52A73A3F5DB
:1018F0009C731B685A6807F52A73A3F50D731A6267
:1019000007F52A73A3F50D73A84A1A63D7F82022A6
:1019100007F52A73A3F50D735A63D7F820321A68B6
:1019200007F52A73A3F50D739A6307F52A73A3F5D8
:101930000D739F4A9A64D7F8642207F52A73A3F5BA
:101940000D73DA64D7F864325A6807F52A73A3F581
:101950000D731A6507F52A73A3F50D73954A1A6678
:10196000D7F8602207F52A73A3F50D735A66D7F8E6
:1019700060325A6807F52A73A3F50D739A6607F566
:101980002A73A3F50D738C4A9A67D7F85C2207F582
:101990002A73A3F50D73DA67D7F85C325A6807F536
:1019A0002A73A3F50D73C3F8802007F52A73A3F5F6
:1019B0001973824A1A6007F52A73A3F5197307F59C
:1019C0001E725A6007F52A73A3F519737C4A9A6050
:1019D000D7F88C2207F52A73A3F51973DA6007F597
:1019E0002A73A3F51973774A1A61D7F88C329A1CB7
:1019F00007F52A73A3F519735A6107F52A73A3F53E
:101A00001973714A9A61D7F88C3203F1110207F504
:101A10002A73A3F51973DA6107F52A73A3F519730D
:101A20006A4A1A62D7F88C3203F1250207F52A7345
:101A3000A3F519735A6207F52A73A3F51973644A5B
:101A40009A62D7F88C3203F1270207F52A73A3F5BF
:101A50001973DA6207F52A73A3F529731846402330
:101A60001A46002103F00EFA07F52A73A3F529732D
:101A700007F144021A6007F52A73A3F529730622B9
:101A80005A6007F52A73A3F5297307F174029A6067
:101A900007F52A73A3F529730622DA6007F52A737E
:101AA000A3F529734B4A03F1180415460FCD0FC453
:101AB00095E8070084E8070007F52A73A3F5297362
:101AC000454A9A63D7F8202207F52A73A3F52973AC
:101AD000DA6307F52A73A3F52976BC466D4606F14D
:101AE0000C040FCC0FC50FCC0FC50FCC0FC523684E
:101AF0002B6096E80E006046FCF74DFAC7F8A4028A
:101B0000D7F8A432002B2AD107F52A73A3F52A733C
:101B10001B681846FCF772FB22E000BF20E000BF04
:101B20001EE000BF1CE000BF1AE000BF18E000BFCD
:101B300016E000BF14E000BF12E000BF10E000BFDD
:101B40000EE000BF0CE000BF0AE000BF08E000BFED
:101B500006E000BF04E000BF02E000BF00E000BFFD
:101B6000D7F8A4121D4802F0FBFE07F52A73A3F56F
:101B70002A731B681846FCF770FBD7F8E431184647
:101B8000F9F728FE07F52A73A3F59C731B6818461E
:101B9000F9F720FE0023C546184607F52A77BD460B
:101BA000BDE8F081F4100210FC10021004110210C4
:101BB0000811021014110210201102102811021035
:101BC00034110210401102104C1102105C1102106D
:101BD0006C110210980A0020690E01107C1102108D
:101BE00080B487B000AFF860B9607A60BB68132B2F
:101BF00002D96FF015031EE0B968124BA3FB012355
